S02B0000433A2F4D4A42432F496E7465726E616C2F755461736B6572426574612F4170706C69636174696F6E73
S20C00200000000120A1D400003D
S214002008C0B2482832D00CD8372837D004D8312860
S21400201824D0322814D127E0382829D045280FD1D3
S21400202812E052280ED004D84E2811D04F2807D1D7
S2140020380CE0582802D06E2802D121E0202031E09A
S214002048002224E040202DE002202BE0042029E096
S214002058154B1B689B8B13F0060F16E0124B1B687C
S2140020689B8B13F0180F10E010201BE0082019E0D7
S2140020780D4B1B689B8B13F0010F06E0012011E047
S214002088094B1B689B8B13F0600F0AD102220B1EAC
S21400209818BF0123002A0CBF002303F0010303B175
S2140020A80A70002070470000E0060020C0B24428EE
S2140020B80BD002D8412806D10BE0462807D0532873
S2140020C801D1012017E000220AE0082013E00220D0
S2140020D811E0094B1B681B8813F0030F0AD1022274
S2140020E80B1E18BF0123002A0CBF002303F00103B0
S2140020F803B10A7000207047E006002010B50F4BA9
S214002108186890F8202012F0080F13D012F0200F4D
S2140021180CBF032407240A492230042203F04EF891
S21400212808B144F0080407480749084A234606F059
S214002138B9FC01E006F0A2FC10BD0000E006002095
S214002148E4050100F1270000BD2500005921000024
S214002158F0B515468AB29C46002A40F08781037877
S214002168441C413B342B00F27D81DFE813F07B00F2
S2140021787B017B017B014F010A017B015D01A50004
S2140021887B013F007B01EA0035007B017B017B0178
S2140021987B0100017B01890005017B0125017B018C
S2140021A87B017B017B017B017B017B017B016B0053
S2140021B87B017B017B0155017B017B017B017B0158
S2140021C87B017B017B0152007B017B011C017B01AB
S2140021D87B0139007B019500DD4B00211A68BCE0C5
S2140021E820786138C0B205F029FE17E1D948DA49E7
S2140021F803F012F8207801F0DDF910B1D748D84975
S21400220801E0D648D74903F007F84FF015032B80AE
S21400221816E02378682B07D0732B08D0662B40F07F
S214002228948104F0A3FA04E004F094FA01E004F0C0
S21400223883FAC84A822102F037FF4FF006022A8046
S214002248C44C83E1207801216138C0B204F00EFD49
S214002258C54B98421CD0BF4C214607F097FD001B83
S214002268288073E1207800216138C0B204F0FEFCB3
S214002278BD4B984268D14FF004022A80BB4C65E1FA
S2140022882378302B04D1B34C204601F063FCE6E7F4
S2140022984FF004032B80F1E7AD4B196801F12604D3
S2140022A801F1270212F8013C0132262BFAD8C1EBBD
S2140022B80203283B2B8049E12378672B19D007D8DF
S2140022C8532B3CD0642B19D0472B40F03E8129E095
S2140022D86D2B1CD0732B07D0692B40F036819C4B96
S2140022E81B6803F10800B6E7994B1B6803F10C005E
S2140022F8B1E7974B1B6803F11000ACE79C4B1B68D3
S2140023081B7A13F0020F18BF9A48A4D112E0984B14
S2140023181B681B7A13F0020F0ABF042396482B800B
S2140023280BD098E7924B1B681B7A13F0020F18BF66
S214002338924890D14FF004022A808B4C06E19048D0
S21400234889E7834B18680230824C214607F05CFD0B
S2140023586FEA0403C01883E7013102EB010393F820
S21400236836307C480B54002BF6D12980EBE0794CAC
S214002378204601F0CDFB72E7824C4FF008032B8015
S214002388E4E02378482B724B0BBF1B681B6893F856
S2140023984B0093F84C0000216E4A03F013F96D4A7F
S2140023A8C2EB0003AFE02378542B01D00020F6E7F9
S2140023B8674B1B68D88BEEE72378303B042B1DD879
S2140023C8DFE803F00303080D1200614B1B6803F1F6
S2140023D8520417E05E4B1B6803F1740412E05C4B72
S2140023E81B6803F193040DE0674B00211878594CDD
S2140023F8421C1A70574A03F0E5F803E04FF0000352
S2140024082B80A2E0204602F017FF29E75F4802F07B
S21400241813FF5E4C288099E05D4B18884D4C0021D0
S214002428224603F0CFF81AE7DCF8080020B18178D6
S21400243811B10088012302E00A200A21002322782D
S214002448312A0DD0322AA6D0302A7ED113B141487F
S214002458504901E03F48504902F0DEFE01389EE749
S214002468084698E74FF000022A806EE028B9986878
S2140024780021042202F08EFE67E00078302845D15D
S2140024889F682FB902238CF840304FF00003BEE651
S214002498B9783B8801FB03F39BB29A4207D9002917
S2140024A853D102234FF000028CF84030C7E6531E83
S2140024B89BB293FBF1F202FB01F15B1A01329EB26A
S2140024C894B24EB9012C07BF2248344921483449F2
S2140024D802F0A2FE421E07E01E48324902F09CFEA9
S2140024E806FB0443421E9CB20021204603F06AF80D
S2140024F8BB78B3420CBF2C492C4902F08DFE154A16
S2140025086FEA0203034414462B801FE031287FF449
S21400251897AE93F84030B2F5004F43F008038CF8B6
S214002528403012D8002322481B540133B3F5807F6D
S214002538F9D12B80B2F5004F02BF9CF8403043F02B
S21400254804038CF84030044600E000242046F0BD22
S214002558E00600207F060020BCE30000900600206E
S214002568D0E30000D8E30000E4050100DDE3000046
S214002578DC060020050A0020090A00200D0A0020B3
S214002588E4060020B0E300007E0600201C050020BC
S2140025987C050020BCE20000F8E200002CE3000006
S2140025A85CE300008CE300009CE30000A8E3000066
S2140025B87E05002030B5002381B08DF803300378FF
S2140025C8451C423B2C2B00F2ED80DFE813F053004D
S2140025D8EB004C006700EB00EB00EB009700EB000D
S2140025E8EB00EB00A500F1009B00A100EB00EB0060
S2140025F87500EB005E00EB00EB00EB00EB00EB0079
S214002608EB00EB00EB00EB00EB00EB002D003B00D3
S214002618EB004500EB00EB00EB00EB00EB00EB00FB
S214002628EB00EB00F100F100634C644920680422DB
S214002638223002F0C3FD002800F0BA802068294640
S214002648223001E05E492846042202F0B7FDD0F1A8
S214002658010038BF0020ACE02846FFF7ABFF002893
S21400266840F0A2809EE02846FFF7A4FF002800F06E
S2140026789B8097E0504B2A781B68413A93F82130A4
S2140026889A4214BF0020012093E04B4B28781B6821
S2140026980DF103019C8BFFF7B3FC07E0464B287847
S2140026A81B680DF103011C88FFF700FD044208BFF4
S2140026B89DF803007DD079E03F4B28781B684628B4
S2140026C893F8202016D004D8412809D0442869D188
S2140026D808E054280CD0732806D0532862D105E0A9
S2140026E8202308E0022306E0012304E0402302E05A
S2140026F8102300E004231A4258D153E0287800F04B
S21400270811FF4EE0287800F00DFF00284ED049E073
S214002718287800F0F7FE44E02B78303B062B41D8AB
S214002728DFE803F0040C11191E2A3900224B23494E
S21400273818680622023002F041FD2EE01E4B2149A1
S2140027481868083003E01C4B1F4918680C30042230
S21400275802F034FD25E0184B1C4918681030F6E7DF
S214002768154B1B4A196813785278098843EA0223DE
S214002778C81A18BF012014E00F4B1B6893F82020D6
S214002788144B02F002021B681B7A03F00203D01AED
S21400279818BF012005E000F0C1FAD0F1010038BFEB
S2140027A8002018B9002004E0032002E0022000E020
S2140027B8012001B030BD0000E0060020E40501005D
S2140027C8E2E300001D0A0020210A0020250A002056
S2140027D8150A0020DC06002000B561202821832287
S2140027E804F08AF800BD0000C0B2532870B50E4643
S2140027F8144600F0D1802BD8482800F0498213D818
S214002808422800F0138105D8002870D0412840F0EF
S214002818698275E0452800F02281462800F0C281CA
S214002828442840F05F825BE14E2800F0878106D896
S214002838492800F058814D2840F05482BDE15028C0
S21400284800F09381C0F09A81522840F04B8244E110
S2140028586F2800F08F8114D85A2800F0A08106D877
S214002868552800F0EA80582840F03C82F1E16528B7
S21400287800F0FE806E2800F07181632840F03282F6
S2140028884CE1752800F0E28006D8702800F07F81B9
S214002898732840F02782A3E0FD280BD0FE2813D02B
S2140028A8FB2840F01F82DFF84034928A187802F03E
S2140028B8C7FD17E2DFF83434536040F285135361DE
S2140028C8002382F820300FE0002382F8203092F8A8
S2140028D84230532B40F00682DFF8143453604FF42E
S2140028E8EB735361FFF778FF6FF00100FBE1DFF849
S2140028F804344FF000021870FF4B1A80FF4B6DE04F
S2140029084B78313B032B43D8DFE803F020023740EF
S214002918FB4B02201968F74B91F820201B7802F031
S214002928020243F008031A4381F8202001F092F9C6
S21400293820B1012001F08EF9FFF74EFFFFF7DEFB0E
S2140029483C2001F095F801F0D1F9CBE10021ED4BE0
S214002958CA5CEB4B1B680B440131262A83F82620F9
S214002968F5D10021E84BCA5CE54B1B680B440131E6
S214002978262A83F82E200BD0F4E701F053F902201C
S21400298801F068F920B1012001F064F9FFF724FF8F
S21400299801F0D6F9002220E00878D64B46281B78A6
S2140029A818D004D8412809D0442809D10AE0542868
S2140029B80ED0732808D0532802D107E020220AE058
S2140029C8002208E0022206E0012204E0402202E09B
S2140029D8102200E0042243EA0202C64B1A7081E184
S2140029E8C74B30781A68462892F8201018D004D8B2
S2140029F8412809D0442809D10AE054280ED0732863
S214002A0808D0532802D107E020230AE0002308E074
S214002A18022306E0012304E0402302E0102300E03E
S214002A28042381EA030382F820305BE1B44B1A687A
S214002A384B78413B82F8213054E1AF4D887800212D
S214002A482C88FFF7DDFA04432C804BE1AC4B0420BE
S214002A581A68A94B1B88938300F028FA42E1A74D11
S214002A68487800212C78FFF721FB04432C7039E1C5
S214002A78087871282BD005D853286BD06D2840F0DD
S214002A88318105E0722825D0732840F02B815BE061
S214002A9800F044F9A8B99A4B984A19680B8823F0AD
S214002AA80B030B80127813430B80924B91F820206F
S214002AB81B7802F0550243F008031A4381F82020D9
S214002AC811E1022003F0B4FD00F03CFA0AE101F03F
S214002AD88DF907E101F034F904E105F0F1F901E1B7
S214002AE804F0E6F8FEE00B78692B05D0732B08D0C7
S214002AF8672B40F0F78009E0814B1B6803F108015B
S214002B0808E07F4B1B6803F10C0103E07C4B1B6855
S214002B1803F11001B01C07F051F9E3E0784C7B494B
S214002B2820680622023002F049FB002840F0DA80CE
S214002B382168701C023107F07FF9D3E0704B013131
S214002B481868363009F024FC022001F083F80028C3
S214002B5800F0C880012001F07DF820E00B78542BA7
S214002B6840F0C0800231072024E00878897800F019
S214002B78E9FCB7E0087800F063FDB3E0337801229B
S214002B88303B9A405B490B7813430B70AAE0594CCC
S214002B980021207800F0AEFD00232370A2E0FFF7A6
S214002BA81BFE9FE016F8023B482B314601D1032056
S214002BB800E0042000F06EFF94E05549B01C01E0E8
S214002BC801F8012C10F8012C0131B2F1200318BFCE
S214002BD80123262A0CBF002303F001030130002B33
S214002BE8EED14C48012400F1FF3C01F8013C20E0FE
S214002BF8252B14D19CF801200CF10103303A03F17F
S214002C08010C5B78D1B2303B0929DAB201D9CB1F67
S214002C18D9B2092A01D9D31FDAB242EA011300F859
S214002C28013C10F8013C0CF1010C402B08BF0024B5
S214002C3801309CF80030002BDAD100F8013C002C5B
S214002C4850D1002000F09AF8334A138801331380D5
S214002C5848E00B78303B032B44D8DFE803F0020744
S214002C680C11274B1B6803F152000DE0244B1B6820
S214002C7803F1690008E0224B1B6803F1740003E0C7
S214002C881F4B1B6803F19300B11C09F081FB29E078
S214002C9893681BB9042003F0A5FDA0603378A468E8
S214002CA8312B0DD1B01C02F065FAC0B2A07010B975
S214002CB80123A37017E00C2814D90C23A37011E085
S214002CC8322B0FD1B01C02F055FA80B2208018B90A
S214002CD84FF00103238006E0B0F57A7F84BF4FF4F7
S214002CE87A722280002070BD4D050020E8E30000BF
S214002CF870E50000D7060020D8060020D60600207B
S214002D08E0060020C4060020BB060020E4050100FB
S214002D181C0500201D0500207C050020034B1868B4
S214002D28042814BF0020012070470000E806002091
S214002D380549064B0A781A7010B9054B1B7801E04E
S214002D484FF0FF330B7070474D05002045050020F7
S214002D58FC090020024B1A78024B1A7070470000D4
S214002D68450500204D05002070470000024A1368FC
S214002D7883F0020313607047FC53024010B50E49F7
S214002D88044604220D4802F019FA0D4B28B91868B3
S214002D980C49933004F074FE08E01B68074893F863
S214002DA82010094A01F0010107F05EFB14B9074B31
S214002DB802221A7010BD0000E4050100E406002097
S214002DC8E0060020D92D00000D2E00000007002088
S214002DD8C0B2012800B50DD10422074802F0E2F976
S214002DE8064B05481B68064A93F8201001F00101B7
S214002DF807F03AFB00BD0000E4060020E0060020CD
S214002E080D2E0000C0B2013800B5072826D8DFE826
S214002E1800F00612170419080D3218482CE0184856
S214002E282AE0184B1B6803F1520025E0154B1B6877
S214002E3803F1690020E0134B1B6803F174001BE0E4
S214002E48114819E00888CA2884BF00230B8012D8C6
S214002E58C0F1CB030B800D4BC0180DE004220C48C4
S214002E680C4902F09FF90C4A137823B1013B137002
S214002E780120FFF783FF002000BD000050E8000097
S214002E8840E80000E00600201C05002064E800007A
S214002E98E4060020E40501000007002000B502490A
S214002EA8182202F07FF900BD50E9000010B5002393
S214002EB884B08DF808301D4BC1B21A68002092F80D
S214002EC821301B4C8DF80B304FF04003ADF8043022
S214002ED84FF48073ADF8063061238DF80C3092F805
S214002EE84B308DF80D3092F84C308DF80E30938BB1
S214002EF86A46009302F072FC207090B10521002209
S214002F0801F0FCFF009B13F0400F0AD040F204418A
S214002F180022207801F0F2FF20788121002201F0BB
S214002F28EDFF034B187804B010BD0000E006002043
S214002F38FC09002000B5024803F00EFA00BD0000A8
S214002F4830E90000044B012200B51A60612003F046
S214002F58ADFCFFF7EFFF00BDE8060020182210B50D
S214002F6848F20400134903F0A7FB0028A8BF4FF453
S214002F78004013DA042018220E4903F09DFB0028AF
S214002F8801DB00200AE00B48FFF788FF0A4B0B49D5
S214002F981868A02202F006F9002408E0064B04464A
S214002FA840F01C0080B21968A02203F085FB20467A
S214002FB810BD0000FD090020DC060020A0E7000088
S214002FC830B5012886B0224C20D1182221496846FF
S214002FD802F0E8F8FFF7C2FF182205461D492068E8
S214002FE802F0E0F81C4B1B681B7A13F0020F15D092
S214002FF804A90422194802F0D5F803A9042218489F
S21400300802F0D0F8174802A9042205E0FFF7A6FF49
S214003018104905462068182202F0C4F80C4C1822FD
S2140030282168114802F0BEF80B4B20681968183062
S214003038A02202F0B7F82068037E092B04D01830C7
S2140030480A49A02202F0AEF8284606B030BD0000B5
S214003058E0060020FD090020DC0600200D0A0020FE
S214003068090A0020050A0020150A0020A0E700002B
S214003078182200B548F204000C4903F01DFB00288E
S21400308809DA04201822094903F016FB002802DA98
S2140030980648FFF703FF054B1A78597842EA0122DB
S2140030A842F004021A70120A5A7000BDFD09002088
S2140030B880B2134B202800B518800BD002D8D8B1A0
S2140030C8082805E0802817D0B0F5807F09D040286A
S2140030D815D111E0612041F27071062203F00CFC54
S2140030E80DE0062261204FF4966103F005FC054BBF
S2140030F81A78054B1A7002E0612003F0D7FB00BD72
S21400310814070020FC0900204D05002000B5044BDC
S2140031180021187801F056FF024B01221A6000BD04
S214003128FC090020E806002000B5C9B282B00129D3
S21400313896461FFA83FCBDF810200BD1074B714644
S21400314893F90000039B009261220192083B6246B5
S21400315808F082FE002002B000BD0000F80600203D
S21400316800B5002387B00093032302930C23039330
S21400317803F1005303F5FE43F433049306238DF856
S2140031881630084B0222069368464FF002038DF865
S21400319804208DF80520ADF8143009F047FE07B076
S2140031A800BD00000207002070B5974C92B0236857
S2140031B8867B002B40F0E980A02003F013FB934B9E
S2140031C81860B82003F00EFB914B18600020FFF73C
S2140031D8F7FEB0F5004F08D161204FF416610322C0
S2140031E803F08AFB0423236003E001232360FFF730
S2140031F8A1FE00F09FFA6D20042103F0B7FB032020
S214003208FFF754FE002800F0FC80824B82481A78AC
S214003218824B1A7002F0C0F97D4B1B6893F8203079
S21400322813F0020F03D06FF01E0004F033F8FEF719
S21400323865FF3C2000F01CFC10200322784908F0AB
S21400324851FF784BC0B2187040B2002809DB42F232
S2140032580F7108F0C7FD4FF4037003F0C3FA724B02
S21400326818606A4B18681E3006F018FEFFF778FFDD
S2140032786E4801230371022383724FF00B03C38049
S2140032880023036003896433038109F0CFFD7CE0E3
S2140032989DF80B20012A1ED002D3412A6FD152E096
S2140032A89DF80C30032B03D1032003F0C1F90AE084
S2140032B8062B06D1574B5E491878162202F0C0F83E
S2140032C863E0832B02D10AF065F85EE06C2B5CD1D4
S2140032D8FFF746FF59E09DF80C30DE2B55D0DF2B64
S2140032E802D0DB2B09D105E047490B68082B08BF3D
S2140032F80A604AE003F098FF47E05E2B45D14D4848
S21400330802F04AF94C4802F047F94C4D00244C4864
S21400331802F042F900210022204602F053F94948FB
S21400332802F03AF90134822135F8020B02F03CF932
S214003338082CECD1444802F02FF9612064216C2255
S21400334803F0DAFA21E09DF80C203046214601F019
S214003358F1FD9DF80830042B17D1324B4FF400725C
S21400336893F90000304B39491B680092612201929C
S21400337802F51A5202332E3208F06EFD05E09DF86B
S2140033880C203046214601F0D5FD02AC30462146D9
S214003398052201F0CFFD00287FF47AAF1A4B1B6890
S2140033A813F0370F2DD01B4B187801F0DBFDF0B962
S2140033B827E02846214600F045FD254B1B888BB99B
S2140033C828462146002201F0DDFB80B14FF48070CC
S2140033D800F07AFE02280AD130781E49172202F039
S2140033E82FF804E028462146002201F0CBFB094EC0
S2140033F802AD30782946402201F09CFD044600289C
S214003408D7D112B070BD0000E8060020DC06002008
S214003418E0060020FC09002048E700004D050020D3
S21400342831310000F8060020FC060020EC060020DB
S21400343880E900006CE700007CE700000207002037
S21400344888E70000F4F100002CF200004605002092
S2140034581407002068E90000013103E001319A42B0
S2140034680FD1013011F8013C0278002BF6D1202A42
S21400347807D8013010F8013C0130202BFAD002386A
S21400348800E000207047000000B503685A1C02E000
S21400349803680133036012F8013C0132202BF7D091
S2140034A8511E4FF0000C4FF0030E15E0303BDAB219
S2140034B8092A01D9D31FDAB24FEA0C139BB202F0DD
S2140034C80F0243EA020C03680EF1FF3E0133013196
S2140034D8BEF1FF3F036003D011F8013C2F2BE5D85F
S2140034E8604600BD013010F8012C01300F2A14BFC9
S2140034F800230123202A08BF43F00103002BF2D142
S21400350802387047064BC0B231381A68C0B2012379
S2140035188340DBB21A420CBF00200120704700002F
S214003528FC530240064BC0B231381A68C0B20123B9
S2140035388340DBB21A4214BF002001207047000007
S21400354800540240C0B2C9B2303864295FFA80FC21
S2140035580AD002D8612904D124E0692904D06F2949
S2140035680DD04FF0FF301EE0BCF1030F1AD8012231
S21400357802FA0CF20C48036823EA020308E0BCF1DE
S214003588030F0FD8012202FA0CF207480368134308
S214003598064903600B6813430B60054B02681B68FB
S2140035A883F84D2000207047005402401C55024006
S2140035B8E0060020C0B261380F2809D8DFE800F01E
S2140035C80A0C0E10121416181A1D2125292D31352D
S2140035D800202FE0184B0EE0174B0FE0164B11E0BB
S2140035E8154B13E0144B15E0134B17E0124B19E07C
S2140035F8114B1BE0114B1B681AE0104B1B685B084D
S21400360816E00E4B1B689B0812E00C4B1B68DB0889
S2140036180EE00A4B1B681B090AE0084B1B685B098F
S21400362806E0064B1B689B0902E0044B1B68DB0997
S21400363803F0010070470000FC530040FC630040A4
S214003648C0B2A0F161030F2B41D8DFE803F0080AE7
S2140036580C0E10121416181D22272C31363B224A3F
S2140036680EE0214A11E0204A14E01F4A17E01E4ADD
S2140036781AE01D4A1DE01C4A20E01B4A23E01B4AAC
S214003688136883F0010321E0184A136883F00203E5
S2140036981CE0164A136883F0040317E0134A1368FD
S2140036A883F0080312E0114A136883F010030DE054
S2140036B80E4A136883F0200308E00C4A136883F068
S2140036C8400303E0094A136883F080031360084B3D
S2140036D8A0F16102196801239340B1F85020002038
S2140036E85340A1F850307047FC530040FC6300403C
S2140036F8E0060020C0B251B10A4A136843F020031E
S2140037081360C03A136823F02003136002E0064BE8
S2140037181B681840054B18601A68054B1B6883F829
S2140037284E20704708E10F4000540240FC53024008
S214003738E006002070B5C14901250A68302492F8D1
S2140037484E3092F84D6006EA030382F84E300B6856
S214003758012193F84E00FFF7CDFF2E4214BF6F21CC
S214003768692120460134FFF7EDFE382C02D06B00A5
S214003778DDB2F2E7B24A0121136843F0060313608C
S214003788AE4B1B68B3F8500008425FD0802931D092
S21400379810D808292ED005D802292BD0042929D0DC
S2140037A8012904E0202925D0402923D0102940F0FB
S2140037B8BD801FE0B1F5006F2FD00AD8B1F5007FA5
S2140037C821D0B1F5806F23D0B1F5807F40F0AE8070
S2140037D814E0B1F5005F2AD004D8B1F5805F40F058
S2140037E8A5801FE0B1F5804F26D0B1F5004F40F018
S2140037F89D8026E0934A13680B438DE0924A13682F
S21400380843F0010388E0904A136843F0020383E01C
S2140038188D4A136843F004037EE08B4A136843F02E
S214003828080379E0884A136843F0100374E0864A70
S214003838136843F020036FE0834A136843F040039D
S2140038486AE0814A136843F080036DE080293CD023
S21400385810D8082931D006D802292AD004292AD017
S214003868012963D123E020292BD040292BD0102909
S2140038785CD124E0B1F5006F3BD009D8B1F5007FE4
S2140038882DD0B1F5806F2FD0B1F5807F4ED121E0D5
S214003898B1F5005F37D003D8B1F5805F46D12DE08B
S2140038A8B1F5804F34D0B1F5004F3FD138E0654AC6
S2140038B811E0644A14E0634A17E0624A1AE0614A73
S2140038C81DE0604A20E05F4A23E05E4A136823F062
S2140038D8800321E05C4A136823F001031CE05A4A7F
S2140038E8136823F0020317E0574A136823F004030B
S2140038F812E0554A136823F008030DE0524A13688D
S21400390823F0100308E0504A136823F0200303E06E
S2140039184D4A136823F0400313604B0099B233E70F
S214003928494A136823F08003136004E04B0099B2F9
S21400393800297FF429AF414B62211B68A3F8500089
S21400394810E04B1CD9B24B1EDBB2613B0F2B71D873
S214003958DFE803F0080A0C0E1012141618232E3986
S214003968444F5A65394A0EE0384A17E0374A20E08D
S214003978364A29E0354A32E0344A3BE0334A44E0E6
S214003988324A4DE0324A136843F001031360A2F549
S2140039988E72136843F001034BE02D4A136843F018
S2140039A802031360A2F58E72136843F0020340E028
S2140039B8274A136843F004031360A2F58E7213684F
S2140039C843F0040335E0224A136843F00803136003
S2140039D8A2F58E72136843F008032AE01C4A13689F
S2140039E843F010031360A2F58E72136843F01003B9
S2140039F81FE0174A136843F020031360A2F58E727F
S214003A08136843F0200314E0114A136843F0400398
S214003A181360A2F58E72136843F0400309E00C4A5F
S214003A28136843F080031360A2F58E72136843F0A0
S214003A3880031360702984D970BD0000E00600205A
S214003A4808E10F40FC530040FC6300401C55004052
S214003A581C65004000B5054B84468AB293F9000001
S214003A686146112307F0AAFA00BD00004C050020A5
S214003A7800B5074B80B21B6893F8201011F0040FAE
S214003A8803D0C90904F0C6FA01E004F0AFFA00BD95
S214003A98E006002030B50246481C10F8013C01300C
S214003AA82B2BFAD00238042A16D0072A27D0032A46
S214003AB82AD1164C256801F05DFB85F84B00246872
S214003AC894F84B30632B01D9632302E0092B1BD8EB
S214003AD80A2384F84B3017E00C4C256801F04AFBA3
S214003AE885F84C00246894F84C30632B01D963237E
S214003AF802E0092B08D80A2384F84C3004E0034B6C
S214003B081C6801F037FBE08330BD0000E0060020AB
S214003B1810B50F4B024619688B78CC78C87904EB39
S214003B2803248B7991F804C000EB03204B7902211B
S214003B381B0403EB0C63C01801F044FDA4B2024654
S214003B482D2302F8013B2046022101F03BFD10BD63
S214003B58E00600202A4B70B519682AA318CBA1FBEB
S214003B6803562AA318CB35090246A5FB03010C0CFD
S214003B782046002101F026FD04EB44044FF0200CFB
S214003B880246442302F801CBC4EB041443706123B5
S214003B985370511C7923C4EB04144B70481C7323D0
S214003BA8A5EBC415421C43701AA318CBA5FB03014A
S214003BB8CC0A82F801C000210232204601F002FD3C
S214003BC8C4EB0414C4EB0414A5EB0415024613A3B3
S214003BD818CBA5FB03013A264C0902F8016B022113
S214003BE8204601F0EFFCC4EB04140246A5EB84055E
S214003BF802F8016B2846022101F0E4FC70BD0000C3
S214003C08400A0020CDCCCCCCFFFFFFFF07452EC2D4
S214003C18FFFFFFFFC5B3A291FFFFFFFF89888888D3
S214003C28FFFFFFFF10B5084C2068FFF737F920683C
S214003C3806220230054901F0B5FA20680449183012
S214003C48A02201F0AFFA10BDE0060020FF09002010
S214003C58A0E70000022830B50546214C11D1214BBB
S214003C6820681B6890F820201B7A02F0020203F0F6
S214003C7802039A4221D11C49182201F09FFAE0B9A2
S214003C881DE01822216848F2040002F0F3FC2168BF
S214003C98A022183148F21C0002F0ECFC012D0AD0D4
S214003CA8022002F0C5FC0F4BA02218680C4B1968BE
S214003CB8183101F077FA002010E001200EE0084CD9
S214003CC81822216848F2040002F0D4FC2168A022D9
S214003CD8183148F21C0002F0CDFCE1E730BD0000C8
S214003CE8E0060020DC060020150A002010B50F4B61
S214003CF881B01A680E4C92F8203013F0100F09D0D5
S214003D080C4BD08B782100930022002307F080FE0E
S214003D18207009E094F9000007F0AEFE064B4FF05D
S214003D2800021A80054B1A7001B010BDE00600208C
S214003D384C050020E14C0000180700201A07002058
S214003D48284B10B51868284B828B19688B889A42BE
S214003D5812D190F84B2091F833309A420CD190F853
S214003D684C2091F834309A4206D190F821204B7AAC
S214003D78D41A18BF012400E0012490F82000097A1C
S214003D8800F0280201F028039A4200F0040201F02D
S214003D98040318BF44F002049A4200F0100201F02F
S214003DA8100318BF44F004049A4218BF44F00804ED
S214003DB80120FFF705F914F0010F02D00420FFF7E1
S214003DC875F814F0020F01D0FEF798F914F0040FF6
S214003DD802D03C20FFF74CFE14F0080F01D0FFF786
S214003DE885FF10BDE0060020DC060020F0B5144B69
S214003DF881B01B68002693F84D70B3F85030012543
S214003E08009331242046FFF77DFB00B12E43013492
S214003E18392C02D06B00DDB2F4E7FFF791FF084AB1
S214003E280020136883F84D70136883F84E60136893
S214003E38009AA3F85020FFF70DFF01B0F0BD000070
S214003E48E0060020114B00B51B888446B3F5007FBA
S214003E588AB214D00E4B1B78052B10D10378082B8A
S214003E6804D10C4B0C49187803220BE03A2B094B6B
S214003E7815BF0A49187818786146012202E0054BF2
S214003E886146187801F0DCFA00BD0000180700202B
S214003E981A070020FC09002058FA000018EE000057
S214003EA810B5CCB201F078FB094801F075FB094B58
S214003EB81B6893F820301C4204D0074801F06CFBBE
S214003EC8012003E0054801F067FB002010BD000054
S214003ED81CEE0000E006002020EE00002CEE00009D
S214003EE810B50278437842EA032313F0010F01D095
S214003EF8002404E013F0020F0CBF02240124084833
S214003F0801F04AFB074B04EB8400C01801F044FBA1
S214003F18054801F041FB02210448FFF7C1FF10BD28
S214003F2838EE00000AFC00002CF2000044EE000008
S214003F3810B5C0B2022884B002D0042825D11EE0ED
S214003F48134801F029FB6846FFF7E2FD684601F0D2
S214003F5823FB104801F020FB0F4801F01DFB0F481B
S214003F6801F01AFB0B4801F017FB0D4801F014FB93
S214003F780C4B6C461868363001F00EFB05E0094B12
S214003F8814221868363001F00DF904B010BD000090
S214003F9850EE000050F0000064EE0000B0E30000B1
S214003FA878EE0000E0060020F0B53C4A3C4E137858
S214003FB888B003EB43039B0003EB06029C59137976
S214003FC8074655790DF1050020211B22009301F0C4
S214003FD8E1F84FB1002201E00C340132C2EB0503D0
S214003FE8BB42F9DC1D464FE02E4801F0D5FA2B4AB5
S214003FF8137803EB430306EB8303986801F0CCFAC7
S21400400829483FE03078402141F26D0200F076FF03
S21400401811E0264B1B88202B12D0254B1B88B3F5A6
S214004028805F0DD0234B244993F9000042220823D1
S21400403806F0C4FF60B9214B6A1C01201A602AE00A
S2140040481F4E00213078422201F0FAF90028D9D014
S21400405854F80C0C01F0A0FA009E0346B0420DF18D
S2140040680501174A02DB1078012204E0009E10784A
S214004078C3EB060292B201F0E3F954F8080C01F01B
S2140040888BFA104801F088FA0C34013DC1D20B4B6C
S21400409800221A60002008B0F0BD00001D070020AE
S2140040A85CFA000090EE000094EE00001407002072
S2140040B8160700204C050020A4FA00002007002060
S2140040C84D05002050F0000080B2B0F5807F00B5A6
S2140040D808D1174B1B8843BB164B1B882BBBFEF718
S2140040E8E7FF03E0134B4FF400721A80124B1B884D
S2140040F8B3F5807F03D12020FEF7DAFF09E00D4BE9
S2140041084FF004021A800D4B032193F9000007F0C4
S21400411833FC02200021FFF70BFF094B00221A7020
S2140041280020FFF741FF002000E0022000BD00004D
S2140041381607002018070020140700204C0500204A
S2140041481D07002030B5C0B282B00091072866D897
S214004158DFE800F004294E55155A5F3F6846FFF71A
S21400416893F905466846FFF78FF902A901F8010D8D
S2140041780122284602F07EFA2A486C464DE0684638
S214004188FFF782F904466846FFF77EF944F40044D0
S21400419802A9A4B201F8010D0122204602F06AFA2B
S2140041A821486D4639E06846FFF76EF901220DF1A1
S2140041B8070102F081FA0028B8BF1C482DDB1C480E
S2140041C801F0EAF99DF80700012101F0EDF9194818
S2140041D823E0194C19491822206800F0E3FF2068EC
S2140041E8174B18301968A02200F0DCFF154814E0B9
S2140041F8FFF718FD0020FFF72DFD13480DE00120FE
S21400420802F016FA114808E0022002F011FA1048E7
S21400421803E00020FFF71EFD0E4801F0BDF902B0CE
S21400422830BD0000ACEE0000C0EE0000F0EE00006E
S214004238D8EE000050F00000E0060020FD0900203F
S214004248DC06002014EF000038EF000058EF0000EE
S21400425874EF000094EF000043B2B3F1FF3F00B5DF
S2140042680AD180216D22054805F0FAFAB0F1FF3F21
S21400427802D1034801F090F900BD00004C07002069
S214004288ACEF000010B585B00DF10204214605F02C
S214004298BBFD204601F080F905B010BD10B584B00E
S2140042A8694605F073FD68466C4601F075F904B07A
S2140042B810BD000010B504460F4801F06DF904F172
S2140042C80800FFF7EBFF0D4801F066F9A01CFFF7A2
S2140042D8D9FF0B4801F060F904F10C00FFF7DEFF88
S2140042E81034084801F058F92046FFF7D7FF06486B
S2140042F801F052F910BD0000C8EF0000D8EF00002A
S214004308ECEF000000F000002CF2000030B5044688
S214004318CDB21048214600F065FF48B10E48214648
S21400432800F060FF58B10D4801F036F901200FE0A3
S2140043380B4B1A6892F8203045EA030305E0084B51
S2140043481A6892F8203023EA050382F82030002005
S21400435830BD000018F0000020F0000028F0000033
S214004368E0060020F0B5C0B285B01546C9B20728E9
S21400437800F28283DFE810F008002800F20015013A
S2140043881A01D40115031A0329B1042907D10122F9
S214004398DFF8EC361A700020FFF706FE6DE30529F5
S2140043A801D10222F4E7062901D10322F0E7072902
S2140043B801D10422ECE7092901D10522E8E70D29F5
S2140043C840F05A830022E3E70C2900F25583DFE821
S2140043D811F01E010D009E0053038800560053037B
S2140043E853035303530333003F008500DFF8940656
S2140043F801F0D2F8DFF8900601F0CEF8DFF88C0668
S21400440801F0CAF802F0B2F9822101F0CDF8DFF81F
S214004418800601F0C1F802F09DF9822101F0C4F887
S214004428DFF8700601F0B8F802F086F9822101F08C
S214004438BBF8DFF864061DE36846FFF78BFB00232E
S2140044480370DFF8580601F0A7F86C46684611E3D3
S2140044582B78313BDBB2032B88BFDFF8440600F22B
S2140044680983DFF8400601F097F82878FFF75AF82E
S21400447810B9DFF83406FDE2DFF83006FAE22878ED
S214004488A0F13103DBB2032B30D8FFF74BF810B19D
S214004498DFF81C06EEE20027012631242046FFF747
S2140044A831F800B137430134352C02D07300DEB240
S2140044B8F4E7284600F044FEC0B2013801238340E2
S2140044C8681CDCB200F03CFE01280CBF47EA04007A
S2140044D827EA04000021FFF70DF9CDE2FFF786FC76
S2140044E8CAE22B78313BDBB2032B02D9DFF8C405CE
S2140044F8C0E2DFF8C40501F04FF82878FFF702F8A5
S21400450810B1DFF8B805B5E2DFF8B405B2E2284620
S21400451800F016FE2B780246202B18BF284605D139
S2140045282846013009E0202BFBD001300378002B09
S214004538F9D1F6E70130202904D110F8011C00292A
S214004548F8D108E039B102F12F00C0B2FEF7FAFF41
S214004558002800F09182DFF86C058BE2C8B250B1F3
S214004568032840F08982DFF8603528461C6800F08A
S21400457801FEE08380E2DFF854452388042B07D148
S214004588DFF84C0501F008F84FF01002228073E2BD
S214004598DFF840354FF000021A800020FEF788FD4D
S2140045A86AE208462946FFF7CDFD65E20A2900F2C9
S2140045B86382DFE801F006102F344C436A8DB2158B
S2140045C83C002846DFF8101505F0F8FB4FF0FF30E2
S2140045D8FFF742FE50E2DFF8F0341968083122E0AF
S2140045E8DFF8F804DFF8F814062200F0E7FD38B91B
S2140045F8DFF8D43428461968023105F01DFC10B9D6
S214004608DFF8E00436E206200021FFF79BFD08F0FD
S214004618C1FE31E2DFF8B03419680C3103E0DFF888
S214004628A83419681031284605F0C8FB24E2DFF8DC
S214004638B804FFF73FFEDFF8B00405E0DFF888446B
S2140046482068FFF737FE2068FFF74AFC14E2DFF819
S2140046589C0400F0A1FFDFF898540024DFF89404C7
S21400466800F09AFF284600F097FFDFF88C0400F069
S21400467893FF204603F0E2FB01340021002200F0FD
S214004688A1FF1335122CE9D1F3E1DFF83C34DFF84B
S2140046986C641C6800273046294600F0A3FD88B9DC
S2140046A823884FF6FC7203EA020222801FB1012F0C
S2140046B840F0E28102E042F0010301E042F002032A
S2140046C82380D9E101370536032F00F0C281E2E7DF
S2140046D8DFF82C0400F060FF00250121284602F0D0
S2140046E8C5FAFF490422044600F068FD80B1DFF8E9
S2140046F8140400F051FF2046FFF7D0FDDFF8080449
S21400470800F04AFF0021284602F0B0FAFFF7BAFD8B
S2140047180135082DE1D1FD48ACE102F0C9FAABE15C
S214004728CCB2162C00F2A881DFE814F017005E0061
S21400473828003D007F00A601A601A601A601A60145
S214004748A601A601A601A601A601A601A601A0002B
S214004758A601A601A6011E011E01DB4BEC4E1F6832
S21400476800243046294600F03DFD002800F00F8161
S214004778013407360C2C00F06E81F2E728783728CB
S21400478805D1D14B1A68938B43F0010309E038280A
S21400479818BFE04840F06E81CB4B1A68938B23F025
S2140047A801039383F9E0C84BDB4E1C6800273046AC
S2140047B8294600F017FD88B9A38B4FF6F97203EA6D
S2140047C80202A2831FB1012F40F0E78002E042F008
S2140047D8040301E042F00203A383DEE00137053656
S2140047E8032F00F03A81E2E7B74BCC4E1C6800274F
S2140047F83046294600F0F6FC88B9A38B4FF6E772D8
S21400480803EA0202012FA28303D0022F40F0C580DC
S21400481802E042F00803DFE742F01003DCE7013766
S2140048280436032F00F01B81E2E7A74BBC4E1C683A
S21400483800273046294600F0D5FC88B9A38B4FF6EA
S2140048489F7203EA0202012FA28303D0022F40F0D0
S214004858A48002E042F04003BEE742F02003BBE734
S21400486801370836032F00F0FC80E2E7AD4800F079
S21400487893FEAD4800F090FE934B1B6893F82130EA
S2140048880B2B97BFC3EBC300A848A14BC01800F07A
S21400489883FE984800F080FE8B4B1B689B8B13F0BA
S2140048A8010F14BFA248A34800F076FEA24800F005
S2140048B873FE854B1B689B8B13F0020F01D00123F8
S2140048C804E013F0040F0CBF0223002303EB83005D
S2140048D8914BC01800F060FE984800F05DFE7A4BD9
S2140048E81B689B8B13F0100F01D0022302E0DB0835
S2140048F803F00103894800EB830000F04DFE904862
S21400490800F04AFE704B1B689B8B13F0400F01D0DB
S214004918012404E013F0200F00F0A5800224894843
S21400492800F03AFE7E4800EBC40000F035FE664C08
S214004938704800F031FE844800F02EFE23680021FF
S21400494893F84B00002200F03DFE804800F024FE5D
S2140049587F4800F021FE2368002193F84C000022CF
S21400496800F030FE794885E0284600F003FCC0B227
S214004978632801D9632002E0002808BF0120524BB3
S214004988152C04BF1B6883F84B0006D002E087F896
S214004998214002E01B6883F84C000420FEF786FAE4
S2140049A86AE008462946FFF7C3FA65E0062963D891
S2140049B8DFE801F0040D101F2B221A0028461021EC
S2140049C8FFF7A4FC002857D1FFF790F954E02846D3
S2140049D802210BE028460421FFF798FC00284BD15B
S2140049E83C20FFF745F847E028464021FFF78EFCB5
S2140049F842E02846082101E028462021FFF786FCE9
S214004A08002839D1FDF77AFB36E0524800F0C4FD9D
S214004A1840215148FFF744FA04215048FFF740FA6E
S214004A284F480821FFF73CFA18B14E482021FFF7F7
S214004A3837FA4D481021FFF733FAE8B14B4800F033
S214004A48ABFD214B00211B680022D88B00F0BAFD75
S214004A580FE047480EE047480CE047480AE047485A
S214004A6808E0474806E0374800F096FD2C4800F076
S214004A7893FD204800F090FD002005B0F0BD000032
S214004A881D0700203CF0000054F000006CF0000009
S214004A987CF0000084F0000050F0000098F0000061
S214004AA8C0F00000D4F00000E8F00000F4F00000C9
S214004AB80CF10000FCF000001CF100002CF10000D6
S214004AC830F1000034F10000E0060020180700204E
S214004AD83CF10000160700204C070020FF090020C4
S214004AE8E405010048F10000FD09002064F100001B
S214004AF8B4FA00002CF20000F4F100000AFC0000F2
S214004B087CF1000094F10000A4F10000B4F100006C
S214004B1819FC0000BCF100006DFC00007CFC0000E5
S214004B2888FC0000D4F10000F0F10000F8F1000065
S214004B3804F2000008F200000CF2000014F2000074
S214004B4820F2000030F2000040F200004CF20000B4
S214004B5850F200005CF2000074F2000088F20000D8
S214004B6894F20000A0F20000BCF20000CCF20000B4
S214004B78E8F2000000F300001CF3000030F3000029
S214004B8848F30000F0B589B283B000250290009281
S214004B98019182E0029B1A78082A09D1454A1378BF
S214004BA8002B7AD0013B1370434800F0F5FC74E004
S214004BB8D2F1010338BF00230A2A14BF1F4643F068
S214004BC80107002F69D13B4C3C4E21787254029A5B
S214004BD813780D2B57D10A2300987354FEF7A8F8BC
S214004BE8237837490133D8B2364B1B7803EB430397
S214004BF89B0003EB01025D58731EC754009B527955
S214004C0833B9314B1B88002B33D013F4806F30D167
S214004C1800282BD0144611E029682848FEF71CFC0B
S214004C28024650B1287A697AFFF79CFB10B92748E4
S214004C3800F0B2FC009AE2B913E00C35013CEBD266
S214004C48234C1E482168FEF707FC024670B1207AFE
S214004C58617AFFF787FB10B91C4800F09DFC009BA3
S214004C683BB9194B1888FEF723FA02E0194800F0FA
S214004C7893FCFEF76FF80F4B00221A70029A012574
S214004C880132029209E04B1C029ADBB20132272B52
S214004C982370029201D927232370019A531E9BB2D0
S214004CA80193019A4FF6FF739A427FF473AF284632
S214004CB803B0F0BD1B07002059FA000024070020A7
S214004CC85CFA00001D0700201407002038F10000D9
S214004CD8A8FA000034F10000C9B2023930B59BB218
S214004CE81446062965D8DFE801F01E3C59332C64C3
S214004CF80400314D314928680422223000F05EFA5B
S214004D0838B1286821462230042200F057FA0028D5
S214004D184DD12B4B1B8813F4917F48D1294B4FF06C
S214004D280101198045E0284B00221A70254B4FF0E8
S214004D3840021A80254B002193F9000006F01CFE5D
S214004D4838E0234A1378FF2B02BF224B1B781370D8
S214004D581C4B4FF000021A801F4B1A701F4B1A701C
S214004D6827E0184B1B88402B12D11949194B0A7893
S214004D784FF400701A704FF0FF330B70FFF7A4F96A
S214004D88012805D1114B022193F9000006F0F4FD25
S214004D980C4B1B88102B0CD108200BE0204619461C
S214004DA80122FFF7EFFE003818BF012002E00220BC
S214004DB800E0002030BD0000E0060020E405010009
S214004DC81407002018070020500700204C05002074
S214004DD84D0500201C0700201A0700201B0700208E
S214004DE830B53B4B88B093F90030857B002B65DAED
S214004DF8FEF77CFF62E09DF80330412B1DD0692B3F
S214004E083DD0012B9DF8042054D1DF2A56D1314BD2
S214004E18186810B1FFF7C8F850E02F4A137813F057
S214004E28010F4BD023F001031370294B4FF4807108
S214004E3893F9000005F0F6FC40E09DF804202846AB
S214004E48694600F077F89DF80030042B12D1234805
S214004E5800F0A2FB9DF90100002802DAFFF7FCF932
S214004E682CE01B4B002193F900000022042306F0D7
S214004E78A5F823E0032B08BF194818D01EE09DF8B4
S214004E8804202846694600F055F89DF80030012BA6
S214004E9814D19DF90130B3F1FF3F18BF114806D170
S214004EA8114800F079FB1148FFF7F8F9104800F0B0
S214004EB873FB03E02846694600F03CF82846694636
S214004EC805226C4600F036F8002894D108B030BDAC
S214004ED84C050020200700205007002064F300003F
S214004EE878F30000A8F3000094F300004C070020B5
S214004EF82CF2000000B507F025FB00BD10B50C4BE2
S214004F08C0B201381FFA81FCC0B219684FEA001E09
S214004F180EEB01031B7B81B0009092B25EF8014055
S214004F281846114602236246A04701B010BD00008D
S214004F385407002010B50A4BC0B20138D3F800C099
S214004F48C0B24FEA001E0EEB0C031B7B81B000902C
S214004F5892B25EF80C4018460423A04701B010BD74
S214004F685407002010B5094BC0B201381A68C0B201
S214004F78010101EB02031B7B81B000908C58184698
S214004F88002100220523A04701B010BD54070020C9
S214004F9810B50B4BC0B201385FFA81FCC0B2196875
S214004FA84FEA001E0EEB01031B7B81B000905EF8F3
S214004FB801401846114607236246A04701B010BDB7
S214004FC85407002010B50A4BC0B20138C0B2CAB2A6
S214004FD819684FEA001C0CEB01031B7B81B000909C
S214004FE85CF80140184600210623A04701B010BD12
S214004FF85407002010B50B4BC0B20138C0B24AB2F5
S21400500819684FEA001C0CEB01031B7B81B000906B
S2140050185CF8014092B2184600210823A04701B068
S21400502810BD00005407002010B50B4BC0B2013865
S2140050381FFA81FCC0B219684FEA001E0EEB010386
S2140050481B7B81B000905EF80140184611460A2383
S2140050586246A04701B010BD5407002000B5104BAB
S214005068C9B293F800E00F4B4FF0000C1B6803F131
S214005078100210E052F8103C834207D112F8043CA4
S2140050888B4203D10CF10103D8B207E00CF10103FF
S2140050985FFA83FC1032F445ECD1002000BD000016
S2140050A85807002054070020C9B211F0100F10B599
S2140050B89446044602D020230CF8013B11F0800FDA
S2140050C808D06346302203F8012B78228CF801209A
S2140050D803F1010C01F00703042B28BF042301F099
S2140050E820004FEA430E0CF1010210E04FEA8E034F
S2140050F834FA03F303F00F033033392B04D908B11D
S214005108073301E02733DBB202F8013C01320EF127
S214005118FF335FFA83FEBEF1FF0FE7D1501E11F092
S214005128080F06D00D2302F8013C0A2302F8013BBB
S214005138104611F0400308BF00F8013B10BD000000
S214005148013010F8013C0130202BFAD0013800223B
S21400515809E0303BDBB2092B02D9273B03F00F03EB
S21400516843EA0212013010F8013C2F2BF1D8104602
S214005178704700000130002205E0D30003EB42032D
S2140051885B18A3F1300210F8011C01302F29F4D85F
S21400519810467047C9B2002301E019540133013A9A
S2140051A8FBD270474FF0000C05E01CF801300CF8F5
S2140051B800300CF1010C013AF7D2704700B594465E
S2140051C84FF0000E08E073461A5C5B5C0EF1010EA9
S2140051D89A4201D0012003E0BCF1010CF3D2002072
S2140051E800BD000000B50130013110F8012C11F89F
S2140051F8013C84469A428E4601D001200AE09CF87B
S214005208003001300131002BEFD19EF80030181E17
S21400521818BF012000BD00000130013111F8012C33
S2140052280B4600F8012C13F8013C01300131002B25
S214005238F4D10138704700000246002000E0013033
S214005248835C002BFBD17047F0B5044681B096B25C
S214005258009107F089F9228A618A02EB06038B42DD
S214005268C8BFC2EB0103A768C8BF9EB2E36807EBD6
S21400527806029A42A26038BF354607D3C1EB02033E
S2140052882268A3609B1AC3EB06039DB207F074F965
S21400529839462A4603E00098037801F8013C531E75
S2140052A89AB24FF6FF7301319A42F4D1AE420FD04C
S2140052B8C5EB060321689AB203E00098037801F864
S2140052C8013C531E9AB24FF6FF7301319A42F4D14D
S2140052D807F04AF9238A3344238207F04DF930460B
S2140052E801B0F0BDF0B5054681B096B2009107F062
S2140052F83BF92A8A698A02EB06038B42C8BFC2EBCF
S2140053080103AF68C8BF9EB2EB6807EB06029A4275
S214005318AA6017D3C1EB02032A68AB609B1AC3EBDB
S21400532806039CB207F028F9384600992246FFF78C
S21400533839FFA6420DD0009B286803EB0401C4EB96
S214005348060204E007F018F9009938463246FFF7D7
S21400535829FF07F009F92B8A33442B8207F00CF94A
S214005368304601B0F0BD0000F0B5038A92B282B0B4
S214005378934228BF134604460F464668019343B334
S214005388C26833449342436015D3C6EB0203019ABE
S2140053989DB20368521B9B184360009207F0ECF816
S2140053A88FB131462A463846FFF7FCFE2168009A38
S2140053B807EB050005E007F0DFF827B1019A384645
S2140053C83146FFF7EFFE07F0CFF8238A019A9B1ABB
S2140053D8238207F0D1F8019802B0F0BDF0B5DCB230
S2140053E80F4696B29DF8145007F0BEF8052C04D068
S2140053F8062C13D0042C07D01BE0104B1B6803EBBD
S21400540805135B681C8A15E00C4B39461B68324648
S21400541803EB05135868FFF7A7FF0EE0074B1B685A
S21400542803EB05135B681A689A605A604FF000022F
S2140054381A82002407F0A0F82046F0BD5407002082
S214005448F0B5C7B282B00D461FFA82FE002F6AD1A9
S2140054581FFA8EFE7346CDF804E0002B3CD10A787E
S2140054684B784C1C9A425BD107F07EF8A9783A4BE9
S2140054783A481970C9B2FFF7F1FDDFF8E4C08CF8B6
S214005488000070B1374B1B6803EB001353F80C0C85
S2140054982B79018A4A1D9B18428A934204DD8CF8B0
S2140054A8007007F069F83BE08B1D038221464FF039
S2140054B8050C836811F8012C0CF1FF3C03F8012B4E
S2140054C8C2688360934224BF036883600131BCF1DD
S2140054D8FF3FEED1062424E0214A14785CB90A7806
S2140054E84B789A421CD18E781C48F1B2FFF7B6FD6D
S2140054F80446A8B104E0184B17701E7807F03CF86D
S214005508184B29461B68019A03EB041353F80C0C36
S214005518FFF7E8FE0421044670B201F027FA00E01F
S2140055280024A0B216E0FF2F04D108467146FEF705
S21400553891FA0FE00B4B7A1E1968D2B24FEA021C9A
S2140055480CEB0103187B00925CF801407246294672
S2140055580323A04702B0F0BD59070020E55300001A
S2140055685A0700205407002000B584460CF10102B3
S214005578C8B200E0013212F8013C002BFAD10CF157
S2140055880103C3EB02039AB20AB9002002E061469F
S214005598FFF756FF00BD000000B5024B1978FFF76D
S2140055A8E3FF00BD4D05002010B583B00DF10104E2
S2140055B8C9B22246FFF778FD2046FFF7EDFF03B095
S2140055C810BD000070B5C9B286B016460AB194463A
S2140055D801E00DF10B0C11F0100F04D020230CF88D
S2140055E8013B01F0FB0111EAD07204D02D23C0F173
S2140055F800000CF8013BDFF8E8E000252CE0394A0B
S214005608AEFB02348DE818004FEAD40E2DB9BEF171
S214005618010F0AD111F0020F01D0302303E011F078
S214005628040F02D020230CF8013B8645E7D8B0FBD0
S214005638FEF3DBB203F130020EFB03F30CF8012B8A
S214005648284AC01AAEFB02348DE81800BEF1000FD7
S21400565818BF01254FEAD40E0028E6D1624609E0B5
S2140056682048AEFB00348DE8180030234FEAD40EED
S21400567802F8013C2B1E18BF0123BEF1000F0CBF19
S214005688002303F001030132002BE9D1501E8DB927
S21400569811F0040F04D02023104602F8013C09E05C
S2140056A811F0020F03D0302302F8013C10463023D5
S2140056B800F8013B11F0080F06D003460D2203F848
S2140056C8012B0A224270581C11F0400308BF0370D1
S2140056D826B90DF10B00FFF75FFF002006B070BD7E
S2140056E800CA9A3BCDCCCCCC00B5002382B08DF84E
S2140056F802308DF803308DF804008DF8051001236C
S2140057088DF8072000200DF1020106228DF80630DC
S214005718FFF796FE02B000BD00B540B282B0C9B22F
S21400572888B100238DF803308DF804308DF8050015
S21400573801238DF8071000200DF1030105228DF8CE
S2140057480630FFF77DFE02B000BD000030B58DB212
S2140057580446284601F046F830B100EB0503206001
S2140057686060A060E360658230BD0000F0B5C9B235
S21400577882B005461046009201919FB2FFF76EFC74
S21400578830BB0021FFF76AFC0646F8B1124B1B68CF
S21400579803EB0013A3F110042B8843B1384601F03D
S2140057A821F8606018B12988FFF7D0FF80B16B88B0
S2140057B843B1384601F016F8A06018B16988FFF7BB
S2140057C8C5FF28B1009B2360019B2373304600E089
S2140057D8002002B0F0BD00005407002000B5C0B29B
S2140057E881B0C9B2082806D8DFE800F01605050714
S2140057F81A0505051E00002019E013896846ADF84D
S21400580800304FF00003ADF802301368094A1978E3
S2140058181423FFF7ABFF0AE0104600F075FB06E01E
S214005828104600F017F802E0104600F0DDF801B068
S21400583800BD0000E5530000044BC0B200B5187068
S214005848000100F0CFFF024B186000BD580700208B
S21400585854070020F0B50746017882B02F48FFF7B6
S214005868FDFB002857D100200021FFF7F7FB002892
S21400587850D0431EDBB23846019307F071FF019AF9
S214005888002316010025009322E01C2000F0AAFF42
S214005898044600283ED015B16861054606E0204B50
S2140058A805461B689B1958601E4B1860009806F042
S2140058B8C7FEBA882060A060606062823B7A03B147
S2140058C8A376174B1A68154B9351009B0133009328
S2140058D806F0B4FE009A8242D7DB1C2000F082FF56
S2140058E80546B8B10E4C23689B1998600E4B186095
S2140058F8002006F0ABFEFB88084A6B822368286007
S2140059086860A8609A513A7833441A73019A531C0F
S214005918D8B200E0002002B0F0BD00003559000003
S21400592854070020300A0020340A0020F0B5DCB204
S214005938032C0F4696B29DF8145027D1294B1B68A6
S21400594803EB05139C68C1B1002E47D0228A638AF0
S21400595835469B1A9E4241DA1AB9002006F076FEB2
S214005968A060A06839462A46FFF71CFCA3685B19A6
S214005978A360238A2B44238231E04FF00003208A59
S214005988A168238206F07AFE054628E006F0ECFDBC
S214005998072C02D0082C11D01BE0124B1B6803EB17
S2140059A805135A6800E05269731E9EB24FF6FF73DD
S2140059B89E42F8D11368148A3B600BE0094B3046C8
S2140059C81B6803EB05135C6806F046FE4FF0000301
S2140059D82382002406F0D0FD254600E00025284650
S2140059E8F0BD00005407002030B5417A044602296D
S2140059F837D81D48FFF732FB002832D10021FFF7C1
S214005A082DFB054668B3201D617A174A1C23FFF74D
S214005A18ADFE30B3DFF854C06B1EDDB2DCF80030E4
S214005A2828011B185A681249637A41F8232022B1C4
S214005A38637A51F82320237A1376DCF800300D4970
S214005A481B189A68637A41F8232022B1637A51F8C2
S214005A582320237A1376204607F09CF86B1CD8B2CE
S214005A6800E0002030BD0000815A000054070020E6
S214005A785C070020380A0020F0B5C0B281B0DCB25E
S214005A880F46009096B29DF8185006F06DFD042C4F
S214005A980ED0052C02D0032C67D12AE0364B1B68A3
S214005AA803EB05135868838A002B5ED0058A5DE0F1
S214005AB8314B2A0186B91B6813449C6806F05CFDC6
S214005AC8032239462046FFF70DFC054606F04CFD36
S214005AD8E37D13F0400F42E01B6813445868838A3E
S214005AE8002B42D0013B838239463246FFF73CFC06
S214005AF83FE0002E39D0204B1B6803EB05139C684B
S214005B08A168B7B96268914204D9638AC2EB0102F8
S214005B189B1A02E003D2C1EB020398B202E0238A82
S214005B281BBB608AB04284BFC6EB00039DB21DD87B
S214005B381BE0731E01F8013BE368A160994224BF8D
S214005B482368A36006F018FD394632462046FFF75C
S214005B58C9FB054606F008FDE37D13F0E00F05D106
S214005B682046009907F0A6F800E0002506F004FD98
S214005B78284601B0F0BD00005407002030B591F863
S214005B88282082B012F0030F0D46C4B213D012F0CC
S214005B98010F02D02046112101E02046132108F00B
S214005BA865FAC0B2002876D195F8283043F040034D
S214005BB823F0030330E012F0200F69D1088B20B9D8
S214005BC822F0400381F8283062E0CB6819786B6AC7
S214005BD813F4806F23D012F0040F1CBF22F00403C6
S214005BE885F828301BD195F82AC08C4505D095F83D
S214005BF829308B4213D1012811D042F0040385F8CE
S214005C0828302046614608F031FA2B6801332B60AD
S214005C1895F8283043F0400385F828303BE02046C6
S214005C2808F024FA2B686A6901332B6095F8283047
S214005C3843F0400385F82830EB6801339342EB6065
S214005C4824BFAB68EB602B8B013B9AB2134B2A83BD
S214005C5853F82430588C95F92B30E3B182421AD881
S214005C6895F82B3000248DF8053001238DF8063082
S214005C780020223B0DF1030105228DF803408DF824
S214005C8804408DF80730FFF7DBFB85F82B4002E071
S214005C98204606F033FD02B030BD00006407002041
S214005CA8034BC0B200B553F82010FFF767FF00BDDE
S214005CB87007002000B50A4BC0B253F8202092F8AF
S214005CC8283039B123F0200382F828301146FFF730
S214005CD855FF03E043F0200382F8283000BD00009B
S214005CE8700700207B4BF0B5CFB253F827407A4BAD
S214005CF8616A81B011F4006FC6B253F8275013D00A
S214005D0894F8282012F0040F1CBF22F0040384F82D
S214005D18283010D194F82A30B34204BF42F0040366
S214005D2884F8283000F0D38011F0800F03D094F860
S214005D382930B34201D0002300E001230093636AB0
S214005D4813F0200F1CD0132E09D195F8283043F0F5
S214005D58200385F828306B6801336B60B7E0112E96
S214005D680ED195F8283013F0200F00F0B08023F0FD
S214005D78200385F8283038462946FFF7FFFEA6E0B8
S214005D88236801332360636A13F4805F19D02A8B73
S214005D986B8B9A420CD82B691E702B696A69013383
S214005DA893422B6124BFAB682B612B8B01332B836B
S214005DB895F8283013F0600F03D138462946FFF7C8
S214005DC8DDFE009B002B45D1228B638B93420ED9B8
S214005DD8531C2383E38B0133E38323691E702369F3
S214005DE8626901339342236124BFA3682361616A11
S214005DF811F0600F26D094F8283013F0100F21D138
S214005E08228B238C9A421DD311F0200F0AD095F8C6
S214005E182830384643F0020385F828302946FFF72D
S214005E28ADFE06E038464FF400714FF4005206F017
S214005E3885FC94F8283043F0100384F8283063680B
S214005E4801336360626A48F2800302EA0303002BA8
S214005E5836D03CE0636A13F4807F1ED0E28B002ABB
S214005E682ED0A38B0233A3832369C2EB0302511EF1
S214005E78626901339342236124BFA3682361A36840
S214005E8899423CBF638BC918E38B0B70238B013395
S214005E9823834FF00003E38312E0A38B228B0133A6
S214005EA8A383638B93420BD9531C238323691E70E9
S214005EB82369626901339342236124BFA36823617F
S214005EC894F82B0018B140B2042100F04FFD01B041
S214005ED8F0BD0000640700207007002030B585B2CA
S214005EE82C2000F07FFC60B10446284600F07AFCBF
S214005EF8A06030B100EB05032061E0606361658354
S214005F0800E00024204630BDF0B5054681B0CEB28C
S214005F18017A4148FFF7A2F8074618B116F0040FB1
S214005F2808D176E000200021FFF798F8074608B960
S214005F3800206FE0394B384A1B6816F0020F03EB57
S214005F480713A3F11000009043F8102C08D0E88837
S214005F582C7AFFF7C3FF324B009943F82400886079
S214005F6816F0010F12D0A888FFF7B8FF2A7A2D4B33
S214005F7843F822002B68009A13F4807F506005D0FF
S214005F880369013303614FF0010303832A7A244B24
S214005F9853F822200AB12B685362DFF888E02B7A80
S214005FA85EF8232072B32B7B82F82B302B7A6A7B21
S214005FB85EF823C0AB8802FB03F31B4A83FB02018F
S214005FC84B11ACF820302B7AAA7B5EF823C0AB883E
S214005FD802FB03F3144A83FB02014B11ACF8223090
S214005FE82B7A0C465EF823202B6853622B7A5EF8D1
S214005FF823206B7A82F829302B7A5EF82320AB7A36
S21400600882F82A3000982B7A29460373287A06F0F5
S21400601825FC384601B0F0BD356000005407002066
S21400602870070020640700201F85EB51F0B5DCB22E
S21400603881B0C0B2023C0F46009095B29DF8186039
S21400604806F092FA082C00F26381DFE814F00900E3
S2140060588800AF0072002201610161016101F4004D
S214006068B54917F4805F14BF0B680B684FEA06142F
S21400607815BFE318E3189C685C68002D57D015F028
S214006088800F05D0626A0098294606F057FB4EE056
S21400609815F4806F0CD0626A2946009808F09CF8C0
S2140060A8010A044601F001010098FFF703FE30E1FB
S2140060B815F0010F03D0009808F050F805E015F029
S2140060C8020F02D0009808F02DF815F0040F03D040
S2140060D8009808F005F805E015F0080F02D00098BB
S2140060E807F0E2FF15F0100F03D0636A43F48053FD
S2140060F805E015F0200F03D0636A23F4805363622B
S21400610815F4006F05D0636A84F8297043F4C073E9
S21400611805E015F4805F03D0636A23F4C0736362F6
S21400612815F0400F1CBF07F07F0384F82B30A48CB3
S214006138EFE0814B1B6803EB06135868436A13F0BD
S214006148800F08BF048B00F0E480808B13F4807FF8
S21400615808BF044600F0DD80431C5C08D9E0764B97
S2140061681B6803EB06139C684FB9628B238BC3EB43
S2140061780200A842A8BF84B280F2CB80C8E006F02E
S214006188FBF92A46394604F10800FFF7ABF805463E
S21400619806F0EAF994F8283013F0600F03D1009857
S2140061A82146FFF7EBFC06F0E7F942E0624B3601C2
S2140061B81B689B195C6848F28013626A02EA03034C
S2140061C83BB1A38B1BB906F0D7F90020B1E0013B21
S2140061D8A3832A4604F108003946FFF7C5F80546A2
S2140061E8606A10F0600F24D094F8281011F0100F91
S2140061F81FD0228B638C9A421BD821F0100310F014
S214006208200F84F828300DD04B4B1B689B199968D3
S21400621891F8283043F0010381F828300098FFF7FA
S214006228ADFC06E000984FF480714FF4005206F07B
S21400623885FA28467DE0012D3F494FEA061405D920
S2140062480B6823449868AB1E9DB202E00B68234493
S21400625858687FB9012D81BF374B07601B684760B8
S21400626885BF03EB06135B6840F825701F6088BF80
S2140062785F604DE0AB0000EB0301C35C3A4602F8F2
S214006288013B4B78481C7B70437853708378937037
S2140062983EE02949340155B10B6823449B689A6847
S2140062A81A61DA604FF000021A839A8330E00B68AE
S2140062B81B195A6892F8283013F0100F2DD023F0C7
S2140062C8100382F828300B681B1999684B6A13F07C
S2140062D8200F09D091F8283043F0010381F82830C0
S2140062E80098FFF74BFC06E000984FF480714FF4D7
S2140062F8005206F023FA104B1B681B195A680CE06C
S2140063084B1C13614FF00003D3834FF00103138334
S214006318002406F031F920460BE04FF00003138303
S2140063289383536A916813F4807F1161D160E7D133
S214006338EEE701B0F0BD000054070020C0B24028C8
S21400634898BFA0F1300305D9602894BFA0F13703A1
S214006358A0F13D03D8B27047014B186070470000A3
S214006368800700204FF4CA32002303E00133DBB273
S21400637802F580628242F9D9DBB2092B01D83033A4
S21400638804E0232B01D8373300E03D33D8B2C0B23F
S21400639870470000F0B50D4F81B03B6805460BB955
S2140063A8002010E0012201AC0430002644F8043D29
S2140063B806F06AFB3E6028466946042206F064FB3F
S2140063C800B10096009801B0F0BD00007C070020E0
S2140063D810B5144B0446186881B050B106E08368BF
S2140063E89C4202D1C06820B11AE010300368002B26
S2140063F8F5D10023204669460422009307F0EAF800
S214006408009B13B94FF480600AE0B3F1FF3F01D157
S214006418002005E0044A121B9A4238BF00920098F2
S21400642801B010BD80070020FBFF0300F0B581B067
S21400643806460D4600921F46FFF7CAFF044658B1A7
S214006448441B09D0BC4228BF3C4606EB0500053075
S2140064580099224607F0BEF8204601B0F0BD0000BD
S21400646870B504460D46164660B94FF4C83413E0B6
S214006478002300242B601BE0201D3146012207F074
S214006488A9F815E0FFF7A4FF043020F47E7020F08A
S214006498070000F580602418064B9C42E8D8204682
S2140064A8FFF796FF28600028E6D104F58064F3E736
S2140064B8204670BDFEFF03000A4B00B51A6842B9B5
S2140064C80AE0137900200B700BE093689842F8D026
S2140064D810321368002BF8D10430012207F07AF83E
S2140064E8012000BD8007002000B506F0B3FA00289A
S2140064F814BF4FF0FF30002000BD0000F0B584B098
S21400650884460091174639480AB900686CE0006866
S214006518374B002832D10CF105051D6002A90DF194
S2140065280F02FFF79DFF0446002850D0029B03F594
S2140065388063043323F47E7121F00701A54202919B
S2140065480AD304EB01039D4206D22046FFF7CCFF90
S214006558029BBB423BD2ED18204602A90DF10F0262
S214006568FFF77EFFA8428CBF0023012300280CBF3C
S214006578002303F0010304464BB3D7E71B6803EB7D
S2140065880002A2F5C8339B0A9BB2019302EB0703ED
S214006598A3F5C833013B9B0A9EB29B2E01D8019CEB
S2140065A813E0019B9B2B1FD8C2F580279B26F6E796
S2140065B8A30203F5CA352846FFF70AFF18B1011DDE
S2140065C82846FFF791FF631C9CB2B442F0D1074CF3
S2140065D8074B0099186823683A46C01806F054FA1C
S2140065E8236807EB0300206004B0F0BD7C0700209A
S2140065F8840700200D4B30B51C68054644B90AE0F0
S214006608284603F075FB10B1A06868B903E010349B
S21400661821680029F4D12878FFF790FE9B2828BF28
S2140066289B20800200F5C83030BD0000800700209F
S214006638C0B2022800B504D003280DD0012815D111
S2140066480BE0002006F0ECFF80B16FEA40606FEACE
S2140066585060C0B2002104E0002006F0E1FF28B137
S21400666801210022002306F03FFA01E04FF0FF3038
S21400667800BD000070B584B201200E4695B206F043
S214006688CFFF38B906F0CCFF002808BF412080F0BD
S2140066980300C0B214F4004F1FBF6FEA40636FEAEE
S2140066A85363DBB283F003006104490C32462B4681
S2140066B806F01AFA70BD000070B584B214F4004FE4
S2140066C80E4695B201D1012002E06404640C002055
S2140066D806F0A6FF08B9013804E0214632462B46E4
S2140066E806F080FF70BDC0460F4B4FF000021A80C0
S2140066F80E4B81B019600E4B19600E4B1A7801E0EC
S21400670883B1043003789342FAD1438801EB03003F
S214006718074B186002E0552300F8013B0DF1030310
S2140067289842F8D901B07047880700208C070020E7
S2140067389007002054050020054B1A68104600E014
S21400674801304378552BFBD0801A80B27047000082
S21400675890070020034B1868034B1B68C01A80B2CA
S21400676870470000900700208C070020044B18682C
S214006778044B1B68C01A044B1B88C01A80B27047AB
S214006788900700208C07002088070020F0B5124EDE
S214006798124F33683A8889B202EB03044B1E1C4238
S2140067A818BFC1F100030E4A1CBF23405C1885B20F
S2140067B8126804EB0503934201D300200AE0204642
S2140067C800212A46FEF7E6FC33682046C3EB04039E
S2140067D82B443B80F0BD00008C0700208807002073
S2140067E890070020F0B5104E104F33683A8885B2EF
S2140067F802EB030414F0030F0D4A1CBF24F0030336
S2140068081C1D126804EB0503934201D300200AE01E
S214006818204600212A46FEF7BDFC33682046C3EB17
S21400682804032B443B80F0BD8C070020880700201B
S21400683890070020054B1B8803F00100C0F10000FC
S21400684800F4344080EA530070470000A407002094
S214006858144B154A196813680133136001B31AE01C
S21400686811F8033CBBB1104B1A6851F8083C9A4221
S21400687811D1C37B022B04D00423C37311F8043C44
S214006888037482892AB151F8083C9B1841F8083CE1
S21400689801E001F8032C0C3151F80C0C0028DFD16C
S2140068A8704700009C070020400A0020104B30B5B7
S2140068B81C6840B2DCB10F4B1D6815E01B7883429C
S2140068C811D10CE09D4209D105F04EFE002323723B
S2140068D863720223EB7305F04FFE08E00C3423685E
S2140068E8002BEFD103E014352B68002BE6D130BD22
S2140068F89C070020A0070020194BF0B51D6840B281
S2140069088EB2D7B2002D29D0164B1C6823E01B7810
S21400691883421FD11AE09C4217D105F025FEE37B7F
S21400692823F00203E3732F721FB9A68126B96E728D
S21400693808E0002E08BF01260B4B1B689B196B60EE
S21400694801236B7205F018FE08E00C352B68002B47
S214006958E1D103E014342368002BD8D1F0BD000041
S2140069689C070020A0070020400A0020134B30B5E3
S2140069781D68134B40B21C68C9B21AE01B788342E4
S21400698816D199B97DB911E09C420BD105F0ECFD02
S2140069980C4BA2891B689B186B600023E37305F0F9
S2140069A8EBFD09E00C352B68002BEDD1E17303E015
S2140069B814342368002BE1D130BD00009C0700206A
S2140069C8A0070020400A002030B51C4B82B01D6886
S2140069D82DE0EB7B13F0050F28D005F0C5FDAB893D
S2140069E81BB9EB7B13F0010F1BD12B7CA3B1002442
S2140069F88DF803408DF804402B6800201B788DF82E
S214006A0806408DF805302B7C0DF1030105228DF824
S214006A180730FEF715FD2C74EB7B13F0020308BF56
S214006A28EB7305F0A9FD6B682846984714352B6864
S214006A38002BCED1024B186802B030BDA00700204C
S214006A4894070020F0B5D2B284B0614B00920022C1
S214006A581A60604B01901A605F4B1A7858E05BB278
S214006A68934250D10A4600E02246144614F9013FE4
S214006A78002BF9D1C1EB0203DFB207EB87008000D9
S214006A880430FFF7AFFE534BE41B0026054684464A
S214006A984FF0000E1860029403962BE0019924E04C
S214006AA8227843B29A421FD14B68CCF80040CCF803
S214006AB804300B89ACF808301BB1039A531CDBB2C0
S214006AC803934B89ACF80A308A89ACF80C208B7B88
S214006AD88CF80F30BCF80A300BB993B20BB1731CA4
S214006AE8DEB20CF1140C03E010310C68002CD7D180
S214006AF80EF1010E029B1EF803000028CED1CCF83A
S214006B08000055B956E011F8013F002BFBD10131C2
S214006B180B78002BA3D100274CE0002E2ED006EBD6
S214006B2846008000043080B2FFF75CFE284B1860F1
S214006B38284B1A6819E0518949B14FF6FF739942F4
S214006B4804BF0023538153890121436005E09389DC
S214006B5813B10121436002E0002143680BB1012311
S214006B68437209B140F80C2B14321368002BE2D19B
S214006B7806EB4603164AA0EB83031360039A009BB2
S214006B8802EB0300C0B2FEF757FE039A92B1114B10
S214006B981C680CE023894BB1032001212246FEF72E
S214006BA81DFEA07310B94FF0FF33A3731434236887
S214006BB8002BEFD1094806F0DDFE094B00241C60C7
S214006BC805F0E4FC074B38461C6004B0F0BD000036
S214006BD89C070020A007002054050020A4070020DA
S214006BE8400A002094070020DFF82CC001309CF8EB
S214006BF8033010F8012C1CF8011C03EA02024A4074
S214006C08134201D0002006E0044B0CF1010C0130C1
S214006C189C45ECD101207047060A00200A0A00208D
S214006C28114B00B55FFA80FE186801220146103045
S214006C380378ABB10132082AF9D100204FF0010CD5
S214006C4810310B7813F0010F05D118B10A790379C2
S214006C589A4200D208460CF1010CBCF1080FEFD19D
S214006C6880F800E000BD0000A80700200E4B00B525
S214006C785FFA80FE186800224FF0010C103090F979
S214006C880030002B08DA531CDAB2724504D109B179
S214006C980B3007E0053005E00CF1010CBCF1080FDD
S214006CA8ECD1024800BD0000A8070020E40501005A
S214006CB8054B1A68012100230131137453741032EE
S214006CC80829F8D170470000A8070020F0B5294B1E
S214006CD881B01C6806460091D7B201251034237887
S214006CE8C3B104F10B0031460422FEF767FA88B9EF
S214006CF8601D00990622FEF755FA14232371042313
S214006D08E370237803F03F036FEA43636FEA536345
S214006D1823702CE00135082DE0D13046FFF764FFDC
S214006D2828B3304614490422FEF748FA30B9124808
S214006D3812490422FEF742FAC8B101273846FFF77F
S214006D486FFF0099044606220530FEF72BFA04F179
S214006D580B0031460422FEF725FA14232371237804
S214006D686FEA43636FEA536323700423E37001B04A
S214006D78F0BD0000A80700200D0A0020E405010069
S214006D8800B5002382B08DF802308DF801304378C4
S214006D988DF806108DF8033041238DF80430022351
S214006DA88DF8053083780DF10101002007228DF853
S214006DB80730FEF745FB02B000BD000070B504467C
S214006DC8154606221E46FEF7EDF91B490622A01DAB
S214006DD8FEF7E8F908232373062363731749062288
S214006DE804F10E00FEF7DEF91349062204F1160038
S214006DF8FEF7D8F91249042204F11C00FEF7D2F96E
S214006E082946062204F120000E4DFEF7CBF931463E
S214006E18042204F12600FEF7C5F9287821462A221E
S214006E28FEF70EFB20B1287800210022FEF708FBAB
S214006E380D2000F0EDFF70BDFF0900207CFF00006C
S214006E48050A0020DC070020F0B5C27883788CB0ED
S214006E5843EA0223027943EA0243427943EA02619B
S214006E680B7B082B77D10378427843EA02231B2B47
S214006E7871D90A7D4B7D01F1160743EA0223012BDF
S214006E8802D0022B67D11EE001F11C0433482631DC
S214006E980422FEF793F988B902238DF81A008DF8B4
S214006EA81B300DF1060039463A462346FFF786FFA3
S214006EB8204639460222FFF709FF3DE0082000F089
S214006EC8A7FF012048E001F11C06244826310422C9
S214006ED8FEF774F9002831D1214B01251C681034BF
S214006EE8237833B304F10B0130460422FEF766F923
S214006EF80090F0B9601D06223946FEF753F91423B0
S214006F0823710423E370237813F0400F08D094F914
S214006F1801302BB120460421FFF732FF009B637037
S214006F28237803F03F036FEA43636FEA53632370E3
S214006F3802E00135082DD2D10220C0E730460949C3
S214006F480422FEF73BF90028B8D03046394602221C
S214006F58FFF7BCFEB2E700200CB0F0BD050A002023
S214006F68A8070020EA05010000B500228BB08DF8BE
S214006F78162001228DF8172010F10B0303490DF196
S214006F880200034AFFF71AFF0BB000BDEA0501002E
S214006F98E4050100F0B5444B81B052B21C680646C1
S214006FA84FB20092012523783BB104F10B0031461D
S214006FB80422FEF703F9002848D0082D02D0103422
S214006FC80135F0E73046FFF70FFE58B3304637492D
S214006FD80422FEF7F3F838B9344835490422FEF798
S214006FE8EDF808B1012000E00220FFF719FE31464F
S214006FF80446042200F10B00FEF7D4F82D490622B9
S214007008601DFEF7CFF8022323710423E3702046A1
S214007018FFF7AAFF6770009BA370237843F040032E
S214007028237038E0214822490422FEF7C7F80028D2
S21400703836D01D4B01251C68103423785BB104F14B
S2140070480B001A490422FEF7B9F820B994F9003063
S214007058002B25DA25E00135082DEDD10120FFF7B4
S214007068DFFD12490446042200F10B00FEF79AF8E9
S21400707810490622601DFEF795F8022323710423A3
S214007088E3702046FFF770FF2378677043F04003ED
S2140070982370009BA37041200A210222FFF72CFCD4
S2140070A80024204601B0F0BDA80700200D0A0020E5
S2140070B8E4050100EA050100F0B53F4C90B02368EE
S2140070C8877B002B6FD18020FFF78CFB6FF07E0349
S2140070D82060042200F80B3B3849FEF763F8206866
S2140070E8364905300622FEF75DF856E09DF803306F
S2140070F8002B58D19DF80430012B22D12E4B0121AC
S2140071081C6894F9103004F11000002B14DA237D63
S21400711893B1013BDAB2227572B9237C13F00103EE
S21400712808BF237408D0E37C1BB1013BDBB2E374D1
S2140071385BBB022322742375013110340829E0D181
S2140071482BE0022B2FD11C4B00261C680125237C24
S21400715804F1100013F0400F11D0E37C3BB1013B63
S214007168DBB2E3741BB1FFF7FFFE012607E000233E
S214007178237494F9113013B10321FFF701FE01358A
S2140071881034082DE3D146B103E0FFF7EDFE4123A6
S214007198237441200A21022203E041204FF496611D
S2140071A80122FFF7A9FB384669460522FDF7C2FE0D
S2140071B800289BD110B0F0BDA8070020EA05010002
S2140071C801684FF0000C0A7801EB020301330360F4
S2140071D8002003E01CF8013043EA0020531EDAB210
S2140071E8FF2A0CF1010CF5D17047000000B50A46DD
S2140071F801680B78C9184B1C036003391046042233
S214007208FDF7D0FF00BD00000346104610B500F895
S214007218013B04235370144601300422FDF7C2FFD5
S2140072280634204610BD0000442000B5FFF73EFB9C
S214007238044B00221A70044904220448FDF7B2FFE2
S21400724800BD0000AC070020AF070020050A00209C
S21400725870B5CEB285B2FFF7EDFA0CA318CBA0FB3B
S2140072680312801A02EB5000000A80B2142805EBBD
S214007278000188BFA1F1280314468CBF99B289B2D1
S21400728832464420FFF738FB70BD000021F1D49049
S214007298FFFFFFFF30B51D4C45B294F90030002BB8
S2140072A80CDA102003221A4904F01CFFC0B210F0B2
S2140072B8800F207018BF6FF0010025D1134B4421B2
S2140072C893F9000004F08EFD124B05F07F02002DA6
S2140072D81A7011DB104811490422FDF76FFF58B1E8
S2140072E80D4904220E48FDF75DFF04220A480021D6
S2140072F8FDF750FF012200E002220A4B50201A70C8
S2140073080121FFF7A5FF002030BD00004E05002034
S2140073180D770000AD070020050A0020E4050100EF
S214007328AF070020AC070020C0B2092800B504D07B
S2140073380A2814BF02460B2205E0124B1B68B3F15D
S214007348FF3F1CD00822DFF83CC0DCF80010B9B1BB
S21400735840F21D53994207D9A1F5A2630E3B4FF69A
S214007368FF71CCF8003007E08BB203EB83039B0079
S21400737899B20023CCF800304420FFF7BDFA00206D
S21400738800BD0000C007002030B5CFB004AC002117
S2140073984FF49672C5B22046FDF7FCFE0C22424911
S2140073A82046FDF7FFFEFFF745FA404C2070FFF732
S2140073B841FA6070FFF73EFAA070FFF73BFA2146E5
S2140073C8E0703B4C042205A8FDF7ECFE237813F08A
S2140073D8E00F04D007A837490422FDF7E3FE06228B
S2140073E835490BA8FDF7DEFE06223FA83349FDF710
S2140073F8D9FE012D8DF8025106D002D3EB1E012BC3
S21400740805D940AC033423E040AC03341AE02378B3
S21400741840AA13F0C00F02F1030218BF144604D1A5
S21400742832202749FFF7F0FE0446214B1B7813F05D
S214007438C50F05D1224636202249FFF7E5FE044649
S214007448042D05D0204620490922FDF7ABFE093455
S2140074584FF0FF332370164B0DF1080C1B7813F012
S214007468600F1A4B12D093F900004FF496730093EE
S2140074784423019343221349634604F0EDFC00B20B
S214007488B0F1FF3F0ED1124B1D700BE093F90000D0
S2140074984FF496730093442301930E4943226346A0
S2140074A804F0DAFC4FB030BD88FF0000C8070020A3
S2140074B8AC070020050A0020FF09002082FF000014
S2140074C8AF070020B307002094FF00004E050020F9
S2140074D8AE070020EA05010010B5094C4420FFF766
S2140074E8E5F9042207492046FDF75CFEFFF7E0FBB6
S2140074F8204644214FF0FF32FFF74CFD10BD000038
S214007508050A0020AF07002030B5774DC4B22B78A7
S214007518082B76D007D8022B6DD0042B16D0012B5B
S21400752840F0E0800CE0202B72D003D8102B40F0FF
S214007538D9800EE0402B7ED0802B40F0D380A6E08A
S21400754804232B70694B4FF050021A80062C00F06B
S214007558C780042C14BF00220122072C14BF134630
S21400756842F00103B3B142B10420FFF70DFF604BB0
S214007578DD2193F90000FEF7CFF85B4B02221A7064
S214007588002104225B48FDF705FEDC200121FFF7F9
S2140075985FFEA7E0052C14D157495848524B2022C5
S2140075A81A7002680B689B1A0B60554B1B68D21A38
S2140075B802600920FFF7B8FE4D4BDE2193F9000064
S2140075C816E04A4C0320FFF7DFFE20880321FFF76A
S2140075D83FFE23885B009BB2B3F5A06F238040F282
S2140075E881804FF050032380414BDB2193F9000044
S2140075F8FEF792F876E008232B703C4B4FF05002CB
S2140076081A800120FFF7C0FE384C02212088DEE7EA
S2140076182046FFF789FE002864D0082C62D1402354
S21400762803202B70FFF7B0FE344A13685B0813601C
S214007638334A136027E0082C17D10820FFF774FE9A
S21400764800284FD02D4A2E4913685B083B2B136041
S2140076580B6008D8284A6FF07F032B7013685B0806
S21400766813600B6031E0092030E0062C3AD123483D
S2140076782149202302682B700B689B1A0B60204B4D
S2140076881B68D21A02600920FFF74EFE2AE00B2C70
S21400769822D10B20FFF748FE20B3174B1A68520872
S2140076A81A60174B3B2A1A600FD8022300210422BF
S2140076B810482B70FDF76EFDDC200121FFF7C8FD92
S2140076C80B4BDC2193F9000092E70A20FFF72CFE0B
S2140076D80320FFF759FE05E0062C03D110232B7074
S2140076E8FFF7FAFE30BD0000AC070020B807002000
S2140076F8AD070020050A0020BC070020C4070020AC
S214007708C0070020F0B5B34B40B293F9003082B002
S21400771883421746079CC9B2BDF8202018BF6FF0F1
S214007728070040F05581012940F03C81E32A40F2E9
S2140077383B812378022B40F03781201DA64904227E
S214007748FDF73CFD002840F0328104F110010422C8
S2140077586846FDF727FD04F1EC00A04904226E46B2
S214007768FDF72CFD10B16FF0090031E19C4D2B7828
S214007778102B0FD19B4839460422FDF71FFD002821
S21400778840F01581684698490422FDF717FD002841
S21400779840F00D8104F1F00301932B78102B00F0D4
S2140077A8C38004D8042B0CD0082B04D106E0402B49
S2140077B807D0802B05D06FF0060009E100240025CD
S2140077C843E08A4B00271C68894B1D68894B1E6856
S2140077D8DAE00131062A019131D005D8012A26D0EF
S2140077E833D3032A2ED125E0342A00F0EF8002D8BE
S2140077F8332A27D115E0352A02D0362A22D105E0C9
S2140078084B1C01934D78013301931EE001317548F6
S21400781804220191FDF7C6FC019B01240433019361
S21400782813E001A8FFF7CCFC724B18600DE0724914
S21400783801A801E0714901A8FFF7D8FC05E07049E6
S21400784801A8F9E701A8FFF7BBFC01990A78FF2A07
S214007858BFD184F00103022D18BF43F0010313B112
S2140078686FF00300B4E05E4A1023137069460422E2
S2140078785D48FDF797FC0320FFF786FD614B4FF048
S21400788850021A8050200321FFF7E2FC8AE00131FB
S214007898332B019128D007D8012B13D044D3032BC0
S2140078A813D0062B3DD124E0362B13D005D8342B25
S2140078B800F08C80352B34D11EE03A2B26D03B2B9B
S2140078C82FD128E04C4901A801E04C4901A8FFF750
S2140078D88DFC29E00131434804220191FDF762FC42
S2140078E8019B043301931FE001A8FFF769FC414B95
S2140078F815E0434901A8EAE74A1C01924B78052B94
S21400790852D1531C0193FFF7E7FD0DE001A8FFF7DE
S21400791857FC364B03E001A8FFF752FC344B1860BF
S21400792802E001A8FFF74CFC01990B78FF2BAED1BB
S21400793838E00132352B01920ED003D823B3332B0F
S2140079481FD104E03A2B12D03B2B1AD114E001A821
S214007958FFF736FC064617E0531C01935278062AB2
S21400796828D00133052A08BF012701930CE001A897
S214007978FFF726FC044607E001A8FFF721FC0546AA
S21400798802E001A8FFF71CFC019A1378FF2BD0D160
S214007998164B1C60164B1D60164B1E6017B1062052
S2140079A8FFF7B2FD002013E06FF0050010E06FF05F
S2140079B808000DE00D4B07201C600D4B1D600D4B9D
S2140079C81E60FFF7A1FD4FF0FF3001E06FF00200E8
S2140079D802B0F0BD4E050020C807002082FF000058
S2140079E8AC070020B3070020AF070020C007002020
S2140079F8C4070020BC070020090A00200D0A002042
S214007A08110A0020B807002030B58AB0847B0DF133
S214007A180305204629460522FDF78CFA08B39DF88B
S214007A2806309DF80720412B18D120462946FDF739
S214007A3881FA9DF80330042B07D10B4B187810B148
S214007A48FFF7A2FC06E0042002E0032B02D1052083
S214007A58FFF75AFD044B00221A7002E01046FFF7A3
S214007A6853FD0AB030BD0000AE070020034B00B53A
S214007A78C0B21B680021984700BD0000D40700204C
S214007A88F0B5444AC9B013780646012B02D0032B3A
S214007A987CD10EE0022313703F4B042218603F4B44
S214007AA83F4819603F49FDF77DFB3F4B05221A709A
S214007AB803E0394B1B68834268D140F2111204A8D0
S214007AC80021FDF767FB02AC6FF055030122237215
S214007AD863720027002307A8A272E37223736273F7
S214007AE846E0451C3246002109E00131C7F582739D
S214007AF8621C994241D212F8013C01350B541446D7
S214007B088A5D131E18BF01232E2A0CBF002303F01C
S214007B180103002BE9D14B1E3E2B31D84B1C3B44AE
S214007B289FB2B7F5847F2ED2C1EB050303F8011C7C
S214007B3823782E2B01D1013418E0BBB91B49052246
S214007B482846FDF72FFB642028210122FEF7D4FEE5
S214007B58174B134993F9000007F112039BB20093E1
S214007B6864230193352202AB04F076F926462846AC
S214007B783378002BB5D100200AE06FF0030007E049
S214007B886FF0010004E06FF0020001E04FF0FF30F4
S214007B9849B0F0BDCC070020D8070020D407002045
S214007BA8CD070020110A0020D10700209DFF000005
S214007BB84F05002000B50A480A4902785AB103233F
S214007BC80B70531E0370084B1868084B1968FFF7AC
S214007BD857FF002002E001230B70012000BD0000C3
S214007BE8D1070020CC070020D8070020D4070020A3
S214007BF830B5214A8AB01378847B83B90123137081
S214007C08102003221D4904F06DFA1D4BC0B21870EF
S214007C1840B200282DDB352104F0E4F829E00DF108
S214007C280305204629460522FDF784F908B39DF882
S214007C380630412B16D19DF8072020462946FDF729
S214007C4879F99DF80330032B04D1FFF7B3FF80B111
S214007C580A200CE0042B0CD10A4B06221A70FFF7F8
S214007C68A9FF06E02BB9FFF7A5FF10B10B20FFF719
S214007C78FDFE0AB030BD0000CC070020917C000055
S214007C884F050020D1070020F0B5594B40B293F9B4
S214007C98003084B08342099CCDB2BDF8286028D154
S214007CA8544B1B78012B24D0104653490422FDF769
S214007CB885FAF0B9012D40F09880072E19D9237857
S214007CC8AA2B16D16378621CAA2B12D15378501CA3
S214007CD813F0800F0DD013F07A0F3DD14378411C76
S214007CE813F07F0F08D013F0800F05D00D20FFF794
S214007CF8BDFE4FF0FF3079E04B784A1C002B2BD1A5
S214007D085378511C012B27D14A784B1C00925A1CD9
S214007D185B78CD1D019353780293384B92781C6894
S214007D2803920EE0384621463246FDF747FA002809
S214007D38DFD1A419237813B12E2BDAD1013407EB3F
S214007D4806052F4617F8016B002EEBD12C4829465E
S214007D580522FDF733FA08B10C20C8E7039A029B00
S214007D686C1D42EA0326019A009B42EA032539E085
S214007D780C46237833B103F0C003C02B04F101018D
S214007D88F6D10C46611C04221E48FDF717FA627AE3
S214007D98A37A04F10B01D0B943EA0223042B18D1C5
S214007DA815480422FDF7FEF95DB16420FEF77EFD56
S214007DB8154B01201B68104998470E4B01221A7074
S214007DC813E0124B06221A70FFF7F4FE0DE043EAA2
S214007DD8022301EB030415B16B1E9DB202E00EB13F
S214007DE8731E9EB256EA0502C3D1002004B0F0BD49
S214007DF84F050020CC070020CD070020D80700201C
S214007E089DFF0000A2FF0000D4070020D107002035
S214007E18094AC0B252F8203001330B2842F8203005
S214007E2803D813680133136004E0102802D8136BD4
S214007E380133136370470000E0070020024BC0B20E
S214007E4853F8200070470000E0070020C0B206285C
S214007E5800B506D0112802D0012804D108E00F206A
S214007E6807E0102005E0044A136B0133136302E0B1
S214007E780E20FFF7CDFF00BDE0070020C2B222F0BB
S214007E888003062B00B506D0112B02D0012B04D197
S214007E980BE004200AE0052008E0084BDA69013206
S214007EA8DA611A6801321A6007E0032012F0800FC0
S214007EB801D0831DD8B2FFF7ABFF00BDE007002056
S214007EC800B5002148220248FDF764F900BD00000D
S214007ED8E007002070B5434C97B02378867B002BCC
S214007EE877D1FBF7C5F845238DF848303E4901237E
S214007EF88DF840304A780B780DF1490043EA0223A2
S214007F08ADF842304FF4C063ADF84430ADF84630B3
S214007F180C238DF84F3002314FF000030622ADF8DF
S214007F285030FDF73FF90420032110AAFDF756FC50
S214007F3820704EE09DF80330012B4AD140E0BDF892
S214007F485630BDF8582043EA0242137B082B32D13C
S214007F58537B062B03D12046FEF776FF58BB2046F8
S214007F680DF15A0101F00EFE84B224B3BDF8583064
S214007F78BDF8562042EA0341CB7D062B12D0112BC2
S214007F880BD0012B17D1BDF85A200E31121B01EB6E
S214007F98040092B201F09CFC0DE00E31204604F07D
S214007FA80DF808E0BDF85A200E31121B01EB04004C
S214007FB892B202F0EDFC0B4B69B21878FDF71AF88E
S214007FC815AC01A8214605F0AFFCC5B215F0800F28
S214007FD8B5D0304669460522FCF7ACFF0028A9D183
S214007FE817B070BDDC070020FD09002010B5074C4F
S214007FF894F9000003F07EFA054B93F9000003F0AD
S21400800879FA4FF0FF33237010BD000050050020AA
S2140080185105002030B5104C82B294F90030CDB22C
S214008028B3F1FF3F17D1114610200C4A03F070FA3F
S214008038C0B220701521002240B203F023FA084B84
S21400804800221A70074B08201D707821064A03F094
S2140080585FFA064B187030BD500500201D860000DC
S21400806828080020450800209984000051050020B3
S214008078F0B5DC4BBDF5BC6D1B7881B0C0B2009383
S214008088002800F0AA81022806D802D1D64B187814
S2140080980CE0D64B187803E0272805D9D34B187080
S2140080A8D34B1B78009301E0CF4B1870A0F10A035E
S2140080B81F2B00F29281DFE813F0260029002C001F
S2140080C82F003200350038003B003E0041004400D7
S2140080D820007D0080004A004700900123009001A0
S2140080E890019001900190019001900190019001FB
S2140080F8900190019001F500A800BE490C2462E1A9
S214008108BD4909245FE1BD491B245CE1BC4909243B
S21400811859E1BC49112456E1BB490D2453E1BB493A
S2140081280E2450E1BA490B244DE1BA4913244AE11A
S214008138B9490D2447E1B949092444E1B849092455
S21400814841E1B84912243EE1B74913243BE109ADA1
S214008158043D0F222846B549FDF724F8B44C0DAA6D
S214008168053A207A0021FDF72DFAB24B2C26013469
S21400817800F8016B9C420246F3D1AF4C00212088E0
S214008188000AFDF71FFA024602F8016B0021207864
S214008198FDF718FA2923014601F8013B2E23437000
S2140081A80D234B704A1C0A235370009B023258B2A8
S2140081B8521B1FE0A1490D2405E1A14B09AC186824
S2140081C8043C00F5C830FEF703F99E49054604222C
S2140081D82046FCF7E7FF09AA28460021FDF7F2F932
S2140081E80D23024602F8013B0A234370009B013226
S2140081F858B2121B92B203A9082302F069FA00B219
S2140082080028D4BF00200120E8E08F4A09AE136892
S2140082188E4A5B8C10688A4A043E116840F2B15256
S214008228934228BF13463246FEF700F9884D82B2BD
S2140082382A80002A00F0D180009B03A95FB2384646
S214008248082302F045FA04B2002C18DD7E4B298874
S2140082581A68D38C0B44D384538C7C4A5B1A1FFA57
S21400826883FC774B10681A6840F2B15389189C450E
S21400827838BF63463246FEF7D9F882B20AB92046B6
S214008288ACE02B88384613442B8003A9082302F059
S2140082981FFA00B2A2E001F11F030370A2F12F0338
S2140082A898B284E00DF5BA606A4908220430FCF7F3
S2140082B879FF0DF5BA610DF5BC62033200200C316A
S2140082C8FEF7CEF809AE0022043E07460192029257
S2140082D861E0614801788A4250D3019A02F12F037F
S2140082E89AB240F2B1539A42D5D85C490A2230462F
S2140082F8FCF758FF5A490B2206F10A00FCF752FF12
S21400830806F11502DDF8DC050021FDF75BF906F13C
S2140083181B04054600E0013CAC42FCD8019A06F175
S2140083281B03C3EB02031B192F339BB20C222846F0
S2140083384C490193FCF736FF9DF8E33505F10C042C
S214008348082B02D908238DF8E335474B9DF8E3251B
S2140083580DF5BA6053F8221007300322FCF722FF07
S2140083683846FDF7FFFF0DF5BA618DF8D5050431DF
S21400837820460822FCF716FF05F114060DF5BA612B
S2140083880DF5BC6238460C310332FEF769F8029BDD
S214008398074601330293029BDAB2DDF8DC35002B80
S2140083A897D11AB12C4A13781F331370019882B2EA
S2140083B812B1009B58B21EE7274A13786BB91F23E1
S2140083C82A4913700A2409A822460438FCF7EAFE4C
S2140083D8009A03A950B222460EE7002079B00DF5A0
S2140083E8806DF0BD500500202A0800202C080020CB
S2140083F8510500200C0101001C010100300001009D
S2140084084C000100580001006C0001007C000100CF
S2140084188C00010098000100AC000100BC000100BF
S214008428C8000100D4000100E80001003301010083
S214008438FD090020010A00202E080020FC0001008B
S2140084483808002042010100840800204008002067
S2140084583C080020A8FF00003E0800204601010056
S214008468500101005B0101005805002028010100A9
S21400847830B5054BC0B21C78044D1CB9FFF7F8FDA3
S2140084882C7000E0287030BD2A0800202B08002039
S21400849870B59DB2534B40B293F9003016468342EE
S2140084A8CCB240F09B80504B93F9000002F042F8A3
S2140084B8631E072B05D8DFE803F093072A7793593E
S2140084C8828C4FF0FF308CE0484A137813F0010F87
S2140084D81CBF43F00203137002D10F20FFF7C8FF3A
S2140084E8434C2378012B06D1424B00221A702820D1
S2140084F8FFF7BEFD74E0022B01D1032305E0062B2F
S2140085086ED12920FFF7B4FD0723237068E0384DA5
S2140085182B78012B0AD12820FFF7AAFD84B2002C5D
S2140085285ED10B20FFF7A4FF2C7018E0072B57D15D
S214008538314B4FF000021B683049DA84304B292053
S2140085481A880B689B180B60FFF792FD80B200280C
S21400855846D10B20FFF78CFF4FF000032B70214B02
S21400856893F9000002F0E2FC08203AE0204C237859
S214008578032B0AD1234B24491868FDF70BFF0B2061
S214008588FFF776FF002323700AE0204B197809B11D
S214008598002202E01E4B1A781970D0B2FFF768FD69
S2140085A8124B00221A701BE0114B1B78032B17D1B5
S2140085B8144B314618682A46FDF7A0FF10E00D4A0E
S2140085C813780BB11F3B13700120FFF751FD00B263
S2140085D807E0064B1B7813F0010F01D1022000E0DC
S2140085E8002070BD510500205005002029080020F5
S2140085F8300800203E0800208408002038080020A4
S2140086083C080020400800202D0800202A080020EA
S2140086182B080020F0B5F84B40B293F9003081B033
S21400862883421646C9B240F0DD814B1E072B09D897
S214008638DFE813F020000B0013002A00DA01200000
S214008648D301D5014FF0FF30D4E1EC4B01221A706C
S214008658EB4B00220A201A70C9E1E94B00221A7077
S214008668E84B1B78012B00F0BF81E74B18781A708F
S214008678C0B2ADE1E14A00231370E24A1521137037
S214008688002202F0FFFEAFE1DC4C2378012B13D169
S2140086983046DE4901F02CFB70B1DD4B1B7813F039
S2140086A8010F05D03044092103F038FED94B187065
S2140086B802230C2023709AE1D04F3B78022B1CD162
S2140086C83046D54901F014FBB8B1D14B1B7813F0EE
S2140086D8010F0DD0CF4D30440A212C7803F01EFE32
S2140086E80443E4B22C701CB101230E203B707EE1DB
S2140086F8C24A03230D20137079E1C04B1B78032B65
S21400870840F072813046C54901F0F2FA08B11020EF
S2140087186DE13046C24901F0EBFA002840F050817E
S2140087283046C04901F0E4FA054608B112205EE179
S2140087383046BD4901F0DCFA20B3BC4C237813F070
S214008748010F10D0AC4B93F9000002F0EFFB237832
S21400875813F0020F04D0B64B93F9000002F0E6FBC4
S2140087681020257046E102F04FFEB24B01461880F5
S21400877801232370AE4B002293F9000002F082FE1C
S214008788182034E13046AC4901F0B2FA002840F02F
S2140087982D813046A94901F0ABFA08B1142026E12C
S2140087A83046A74901F0A4FA002840F01F81304659
S2140087B8A44901F09DFA044600282DD03044A24969
S2140087C801F0FCFA002200E00132135C2F2BFBD8E4
S2140087D800EB02042B238354C2EB0400FCF7CAFC0C
S2140087E8944B000285B201221D8000E00132135D21
S2140087F82F2BFBD80023A354601CFCF7BBFC8D4B27
S21400880828441880904991480422FCF7D7FC002891
S21400881840F0EC801920EAE030468D4901F068FA0D
S21400882850B3824E337813F0010115D00F20FFF7AE
S2140088381FFC884B85B21C70337813F0020F02D0E9
S2140088482820FFF715FC2BB2002BD4BF00200120F0
S2140088586C4B01221A70CDE0754B93F90000754BEE
S2140088681A8800911423784902F0F6FF10F0800F5A
S21400887840F0A6800122A0E03046774901F038FA99
S214008888054648B3694D2B7813F001010DD1684BA6
S21400889893F90000674B1A88009114236A4902F07E
S2140088A8DBFF10F0800F40F08B80741D2046FDF72C
S2140088B8A1FE6A4B1860204601F034FA684B514A0C
S2140088C818702B7813F0010F03D003230F201370B2
S2140088D88DE00223137087E03046624901F008FAFB
S2140088E8E8B1741D2046604901F002FA5F4E38B1BF
S2140088F84FF4C8304FF41C31FDF7F6FD35600CE038
S2140089082046FDF777FE0446FDF762FD411D20462A
S214008918A4F5C834FDF7E8FD3460162067E0304655
S214008928534901F0E5F9044658B17379701D2F2BA9
S21400893846D0FDF75FFE4D4BA0F5C83018601720EF
S21400894855E030464B4901F0D3F900283AD0737900
S214008958701D2F2B0BD1354D2B7813F0020F04D03A
S214008968334B93F9000002F0E1FA2C7028E0FDF78B
S21400897841FE3A4B1860FDF72BFD90B12C4B32495F
S21400898893F900002B4B1A881423009402F064FF16
S21400899810F0800F05D11B4A06231370334B1C605A
S2140089A822E0224B1B7813F0010F09D02F4B002230
S2140089B81A602920FFF75CFB0722124B1A7013E097
S2140089C8112014E030462C4901F092F918B11B200A
S2140089D8FFF74EFB08E0152009E0022007E0074BEA
S2140089E81B780BB1022005E0002003E01320FFF7F8
S2140089F83FFB00B201B0F0BD50050020280800205B
S214008A082A080020300800202B080020B4FF0000A9
S214008A184508002044080020BCFF0000C4FF0000F2
S214008A28CCFF0000D4FF0000D8FF00002908002073
S214008A38510500202E080020E0FF0000E8FF000097
S214008A48ECFF0000F4FF000031080020E4050100F8
S214008A58FCFF00003E08002004000100400800203B
S214008A682D0800200C000100140001003808002022
S214008A78180001002000010028000100084B30B54E
S214008A881C685CB1002594F91E0002F033FD013520
S214008A984FF0FF33A3774434042DF4D130BD0000E3
S214008AA848080020F0B5294D83B02C680290019143
S214008AB80092DFB22CBB4FF48870FDF793FE286057
S214008AC840F28C50FDF78EFE214B002618601F4D95
S214008AD8782108201F4A2C6802F01AFDA0772B6818
S214008AE8002293F91E00502102F0CCFC2A680136B9
S214008AF802F14403042E2B60E9D1A2F1CC032B60CB
S214008B0816E0002594F91E30B3F1FF3F0BD178210B
S214008B18104A082002F0FCFCC0B2A077502140B2F0
S214008B28002202F0AFFC0135042D01D04434E9E7F9
S214008B38094B029A1F70094B1A60094B019A1A6072
S214008B48084B009A1A6003B0F0BD000048080020E1
S214008B584C080020CD93000050080020680800202C
S214008B686008002064080020F0B592B28EB09BB270
S214008B7804900D460392029352B9888B0023039003
S214008B88888781F83F3004464FF00001A98305E046
S214008B9891F83F30013381F83F30039C002206925B
S214008BA8AB8B029A0398049905938918C4EB0003C3
S214008BB8049A9BB20A9313440B9395F820300991B4
S214008BC8A7B205F11C01AC830891ADF83670002BEE
S214008BD840F0FB8000220792F2E00B99084610F856
S214008BE8013BA32B0B9040F0E680032A06D8089892
S214008BF803889B1A0380C2EB070395E04B78411C59
S214008C08642B0B910CD005D8442B09D0482B40F088
S214008C18AE8034E0732B03D0762B40F0A88023E098
S214008C28954B1A683AB111F8013C481E732B08BFD9
S214008C380846904707900799002900F0FF80022908
S214008C4805D18E484FF00702ADF83420FFE0079BA9
S214008C58032B05BF0820ADF83400894889481CBF97
S214008C680821ADF83410F2E0874B1C68002C00F0A1
S214008C78E58008460DAA00212B46A04778E0824BDF
S214008C881B68002B00F0DA8095F83F300DF13200B3
S214008C9805EB43039B89022201339EB2FCF782FA56
S214008CA80B9B02330B93BDF83630033BADF83630DA
S214008CB849E095F8403013F0040F05D0BDF834307D
S214008CC8043BADF8343006E0BDF8340020212044DB
S214008CD80422FCF75FFABDF83410099A04310DF146
S214008CE8360389B20093019220460BAA089B03F02C
S214008CF887FB95F8401011F0020F57D10B9A83B2F4
S214008D08C3EB070092B187B2B7F5AF6F19D995F8DC
S214008D183F3005EB4303DE8141F0010385F8403020
S214008D28AB8B043BAB833B1F98B24FE095F83F30C4
S214008D38721E05EB4303DA8141F0010385F84030E3
S214008D4832E0731C9EB2504B0DF132001C6831465F
S214008D580DAA2B46A04704460028AAD10B9B023B27
S214008D680B93BDF836300333ADF8363066E0002096
S214008D780B9B02330B93BDF83630033BADF8363009
S214008D88C8B10DF136030093099BBDF83410019362
S214008D980BAA089B03F034FB80B260B10B9BC0EBB8
S214008DA807000BB187B206E080B20FE001F00803B7
S214008DB885F8403009E0BDF83630013BADF836306E
S214008DC8BDF83620002A7FF408AF384682B20A98E3
S214008DD8069900EB02039EB2AB8B03985B180599C5
S214008DE8C3EB00039CB201EB00031B1BD2F101028C
S214008DF838BF002299B2002C08BF42F00102A983AE
S214008E08002A2DD1029A06EB0407974228DA95F82D
S214008E18403013F0010F23D1AB6968682246C018AA
S214008E281A4B40181968BFB21431891904F0D2FBDE
S214008E38AB8B03979B1BAB830696B1E60B9B023363
S214008E480B93BDF83630033BADF83630B3E70B9BD3
S214008E5802330B93BDF83630033BADF8363090E757
S214008E6895F84030304603F0080385F84030AB8F5D
S214008E781B1BAB870EB0F0BD600800208B010100FD
S214008E889201010083010100640800204C080020BC
S214008E98F0B5D3B23D4A8DB282B0116804462A4670
S214008EA890F91E0001F014FC00B20028D4BF002080
S214008EB801200090002865D094F83E300133DBB2DC
S214008EC8012B84F83E305DD8314BE289D3F800E0B8
S214008ED8A069BEF82230A18B5B1B9EB2D4F814C0E2
S214008EE82282331E18BF012300EB0102944594BF6B
S214008EF8002303F00103002B44D0C1EB0C031B1A1C
S214008F0801939BB2AEF82650B3F5AF6F34BF1D463B
S214008F184FF4AF65AE4238BF354604D3B6F5AF6FEB
S214008F2888BF4FF4AF66A3696068184FC0183968E1
S214008F38A38B1431C0182A4604F04CFB154BA587A2
S214008F481B7813F0010F08D038682A4614302146DB
S214008F583346FFF709FE054602E0A38B2B44A3839E
S214008F68A38F019A93422CBF4FF0080C4FF0000CC9
S214008F7845B1064B6587196894F91E002A4663466C
S214008F8801F0A6FB009802B0F0BD00004C080020D7
S214008F98840800205008002030B50D4D0446286887
S214008FA8372214300B49FCF7FDF84FF03703A3833C
S214008FB80323E37794F91E0029683722082301F073
S214008FC887FB00B20028D4BF0020012030BD000077
S214008FD84C080020B0010100F0B50C46D0B1CB7F9C
S214008FE8022B02D803782F2B01D830230370FDF705
S214008FF801FB0223E3770546FDF7EAF908236061DB
S21400900884F8203040B92A4D4FF4DB73636184F846
S214009018200001E04B685D1F636903F11300B0F59B
S214009028AF6F606103D94FF4AF66002701E086B2E0
S214009038082794F82030082B06D104F1200128468A
S214009048FDF73AFA00B9053D6B1D1A4D63602868AE
S214009058132214301849FCF7A5F8296860682731E8
S214009068A6F1130204F0B6FA6368A683133B63609E
S214009078124B1B7813F0010F0ED0114B28681B6893
S21400908821465B8CB3F5AF6F28BF4FF4AF6314303F
S2140090980022FFF769FD0646094B4FF000021B68E1
S2140090A82046DA8431463A46FFF7F2FEF0BD000065
S2140090B8E30101004C080020680101005008002068
S2140090C884080020F0B504460D46616992B28A42CB
S2140090D8184607D20E23E377EAB1C2EB0107FA2651
S2140090E8626105E00223E377002303700027FB266E
S2140090F862690023AB540020294603F049F90A4B5D
S214009108401B013860611B6830462946224698474E
S214009118FA2E02D16761002004E004F142002146DD
S214009128FFF75AFFF0BD000068080020F0B5C37FBF
S21400913881B0052B05460F4696B20BD19A490A7898
S21400914812B1102200922BE10623C37701230B707D
S21400915880F84120EB7F062B02D900230093C6E057
S21400916800220092C0E090490A7812F0200F02D040
S2140091786B69013B6B6112F0080F10D03B780D2B22
S21400918807D102F0F70312F0040F0B7000F0A98065
S214009198AAE095F84130013385F84130A1E0DFF8C0
S2140091A80CC24FF0000E481C0178DCF800303A7804
S2140091B85B5C9A4240F08A804B1C9CF80420DBB229
S2140091C89A42037040F08480784B03EBCE035B79B9
S2140091D8013B092B6ED8DFE803F0050C163D4D431E
S2140091E843434343704A137843F0480323F002038B
S2140091F834E06D4AB81C137843F004031370FBF789
S214009208B9FF686156E0684C227812F0040F07D060
S21400921895F84130002B00F0B98042F02003237007
S214009228237813F0120F45D06B6995F84120083B58
S2140092389B1A6B615E4BFF201B6800212A469847E5
S21400924830B9237813F0100F02D00923EB7731E0FA
S2140092580A23FBE7544A137843F00203137029E005
S214009268514A137813F0020F24D003F0FD0343F09D
S2140092781003F3E74F4C5049206815221430FBF7CB
S21400928891FF4FF01503AB8316236B610123AB6187
S214009298082385F82030494B15226B6095F91E0087
S2140092A82168082301F014FA009A00B20028C8BF03
S2140092B80122009200210A224148FBF76BFFEB7F50
S2140092C8082B0ED9731E01379EB210E000230370D8
S2140092D80EF1010E0130BEF10A0F0CF1080C7FF4F6
S2140092E863AF731E01379EB2002E7FF43CAFEB7F50
S2140092F80E2B53D12C4B2846394632464BE06C6928
S214009308B44238BFA6B20A2B16D02B6843B9284BEE
S2140093186E611B68FC2039462A4698476C6104E053
S214009328686839463246FDF7E9F82EB16A682B6850
S2140093389A4201D1531D6B606B69C6EB03046B68D8
S2140093486C619B196B60002C2AD1286805F12001F6
S214009358FDF720F8144B1C700223EB772B686C6023
S21400936803B118B1124BFE201B6802E0104BFD201B
S2140093781B6800212A46984728B100202946FFF78F
S2140093882BFE00900CE005F14200F7E7721E791CF0
S21400939892B228462346FFF795FEF2E7002EAED196
S2140093A8009801B0F0BD000054080020B803010082
S2140093B8680800204C080020A1030100A003010053
S2140093C855080020F0B59FB2DFF82C3444B21D686B
S2140093D881B095F91E301646A342C9B20FD044355F
S2140093E895F91E30A3420AD0443595F91E30A3429B
S2140093F805D0443595F91E30A34240F0E6814B1E51
S2140094080B2B47D8DFE813F0300048004E00DC008E
S214009418460030006E000C00460046004B008B00ED
S214009428EB7F002B36D1F54B1B7813F0080F0BD0CB
S214009438F34B1A68B2B16123701E06F8013C9047D8
S214009448012840F0C2810DE013F0020F0AD0EC4B61
S2140094581A683AB16223701E06F8013C9047012844
S21400946800F0B381012318E0AF683FB1E54B1E68F2
S21400947826B10020012100222B46B04700214422B5
S2140094882846FBF787FEAF60AC77204650210022BF
S21400949801F0F8FF0020ACE10223EB77FAE7AB69AE
S2140094A8002BF7D0EB7F032B08BF204600F0848004
S2140094B8AA8BAB699B18AB6103294FF00003AB83FB
S2140094C807D12A8A05F10E00AA8100210422FBF79B
S2140094D861FE4FF0000385F83E30CB4B4FF000029C
S2140094E81B68DA84EB7F032B00F06081012BD1D94F
S2140094F86A69A9698A425DD9C1EB0204B4F5AF6FFF
S21400950801D8082702E04FF4AF640027BE4B1B685B
S2140095185B8C9C4208D9002BBCD01C4604E0012377
S21400952885F83E3001240027AB69AC83B74E63B993
S2140095383068B74913221430FBF734FE6868316880
S21400954813302731A4F1130204E068683168184420
S2140095581431224604F03EF8A84B1B7813F0010F8E
S21400956822D0A94BA94C1B6820685B8C2946B3F50A
S214009578AF6F28BF4FF4AF6314300022FFF7F4FA3A
S21400958808B1044610E095F8403013F0080F01D0F3
S214009598002403E022682023137501244FF00003FB
S2140095A8AB83AB89EB812B82A1B228463A46FFF7FC
S2140095B86FFC1EE195F91E0001F0B8FC082018E1C2
S2140095C86B68EA7F002B40F0F780032A1BD83046EA
S2140095D890490322FBF7F2FD48B130468E49042233
S2140095E8FBF7ECFD002840F0F2800523EB77721CB1
S2140095F8002F00F0EC807B1E16469FB216F8013C42
S21400960801322F2BF4D1EB7F042B1AD9052B40F00F
S214009618D68033782A2B00F0DC803046FCF7EAFF49
S2140096287378044685F84230304600F07BFB2C60A1
S21400963885F820006C600CB901236B6000236B6111
S214009648BDE00622002105F10C00FBF7A3FD3278E9
S214009658BFB28DF80320EB7F032B03D920238DF8A8
S214009668033001E0202A67D1644BE97F1B7895F820
S214009678390013F0040F5FD0032998BF04211FFA9E
S21400968887FE06F1010C4BE00B1F042B46D8DFE8DB
S21400969803F003090F2229001CF8013C0D2B3DD1CD
S2140096A805213BE01CF8013C0A2B36D1062135E0A3
S2140096B81CF8012C0D2A01D107212FE0574B1B5C03
S2140096C8934201D0042104E0431CD8B2142825D9BB
S2140096D80821002022E01CF8013C0A2B1DD1022399
S2140096E8EB7763E01CF8012C00EB05030D2A83F8E2
S2140096F821200DD105F121042046214602F0A2FDC5
S2140097082046072102F00AFE0346002840D113E04F
S214009718431CD8B2172801D948E004210CF1010CE3
S2140097280EF1FF331FFA83FE4FF6FF739E45ABD14B
S21400973885F83900E977ADE6304B1B7813F0020F51
S21400974853D0374B00201B680DF103012A46984773
S2140097580346E8B9344616E07B1E9FB2002F44D075
S2140097683F2914BF00230123262908BF43F001031D
S2140097784BB1631C5C1C1878294B21461B682A468B
S2140097889847034620B914F8011F2029E4D12CE095
S21400979813F1020F0ED0B3F1FF3F07D013F1030FFA
S2140097A81CBF01A800F8013D20D173E62846FFF744
S2140097B8F3FB1EE0002019E0042A7FF66BAE28466D
S2140097C831463A46FFF7B2FC13E0022011E01020BB
S2140097D80FE07378304685F8423000F0A3FA00238D
S2140097E885F820002B606B6026E730462946FFF791
S2140097F8F3FB01B0F0BD0000480800205008002028
S2140098086008002064080020840800204C08002017
S214009818680101007C0101007F0101009A01010036
S2140098286808002030B504468DB284B021462A4622
S214009838002000F0B3F86FEA000080B2030AA370B5
S2140098480023E0700293039304F114000121002220
S21400985880230094019500F011F904B030BD000093
S214009868F0B58EB00DF11604049055B2CFB220466E
S214009878002122225EB2FBF78DFC08238DF81630F5
S2140098888DF81A508DF81C60002104EB010201F1D6
S214009898610301311A291372F7D1214622220020CA
S2140098A800F07CF86FEA000080B2030A8DF81830E2
S2140098B822238DF8190001930498012100223B46C3
S2140098C800940295039600F0D9F800B20EB0F0BDE9
S2140098D8F0B5054696B2002086B00F4632462946B1
S2140098E800F05CF84FF6FF73984254D12B78032BA0
S2140098F838D0082B01D0DBB14DE00024294632468B
S2140099082C70AC70EC70002000F048F86FEA00008D
S21400991880B2030AAB70E870012107F10C00002240
S2140099288023009501960294039400F0A7F832E08D
S2140099388DF812308DF811302B7900208DF8133001
S21400994869238DF8143002238DF8153001238DF81D
S2140099581630AB790DF1110107228DF81730FBF799
S2140099686FFD18E06B78032B15D16B7C112B12D189
S2140099782B7A03F00F0305EB83031A7A93F80AC0D1
S214009988587AD97A40EA022041EA0C2107F11003F6
S214009998022202F045FA06B0F0BDC04630B580B2E5
S2140099A8C4B295B2000A1DE011F8022C00EB0203BF
S2140099B8D8B2904204D2631CDCB20CB9431CD8B2AD
S2140099C8AB1E9DB24FF6FF739D420ED011F8012CC8
S2140099D804EB0203DCB2944204D2431CD8B208B9A2
S2140099E8631CDCB20231002DDED104EB002080B20D
S2140099F830BD00005FFA82FC013001310AE010F841
S214009A08012C11F8013C01301A430131FF2A01D01C
S214009A18002007E00CF1FF335FFA83FCBCF1FF0F70
S214009A28EDD101207047000030B5C37884780D4624
S214009A3844EA03240379042244EA0344437905F1FB
S214009A480C0044EA036423780B70A3788B70E378E1
S214009A58CB70637A4B7204F10C011034FBF7A2FB4F
S214009A6805F1100021460422FBF79CFB287800F03D
S214009A780F0080001438C0B2143030BDF0B58AB07C
S214009A88DFB2BDF84030CCB2D6B29DF944109DF98D
S214009A98482005460093FDF77DFA08B9013864E0CA
S214009AA8411D06220DF10600FBF77CFB3049062215
S214009AB803A8FBF777FB2F4902220DF11200FBF7EC
S214009AC871FB45238DF81430009B2B4903F11402D3
S214009AD813128DF816300B888DF817208DF819306C
S214009AE81A0A01330B808DF81820002305A90A22CC
S214009AF800208DF81A308DF81B308DF815608DF81B
S214009B081C708DF81D40FFF749FF1C490422FFF71B
S214009B1845FF29460422FFF741FF6FEA000080B29E
S214009B28030A8DF81F001549042208A88DF81E3070
S214009B38FBF738FB2946042209A8114DFBF732FB30
S214009B482046FEF783F928780DF106012222FBF756
S214009B5877FC50B10F99009A2878FBF771FC2878A3
S214009B6800210022FBF76CFC00B20AB0F0BD000032
S214009B78FF090020B80401006C080020050A002030
S214009B88DC070020F0B582B00091C27883780446DE
S214009B9843EA0223027943EA0243427943EA02602F
S214009BA8437B002B40F099802278637842EA0321B1
S214009BB80D2940F29280212940F38F80837B00F1A3
S214009BC80E0603F0F003402B40F08780B378F27857
S214009BD802EB032292B2A1F10E039A4201927CDCB8
S214009BE800F11E0528463E490422FBF7E7FAE8B1CD
S214009BF828463C490422FFF7FDFEB8B9707A40F0C3
S214009C088000FEF73BF9737A012B66D1E378A078DB
S214009C18354940EA03202379062240EA034063795F
S214009C2840EA0360FBF7CAFA18B156E0707AFEF706
S214009C3825F9337803F00F039B00143BDDB2282D7B
S214009C484BD82378627843EA0223223B9D4244DCC1
S214009C58E378A1782A4641EA0321237906F114001D
S214009C6841EA0341637905F1140741EA03612231A9
S214009C78FBF798FAE378A178002041EA03212379D4
S214009C88BAB241EA0341637941EA03610E31FFF74C
S214009C9885FE4FF6FF7398421FD106F10C0528463D
S214009CA812490422FBF78AFA70B1E378A1782846AD
S214009CB841EA03212379022241EA0341637941EA12
S214009CC803610631FDF702F8B37913F0200F04D1CB
S214009CD8019B009A3846138000E0002002B0F0BDD1
S214009CE8050A0020090A0020FF090020EA050100ED
S214009CF800B5002286460EE012F80EC09C4509D034
S214009D08602B01D9203B02E0402B09D92033DBB277
S214009D189C4505D10132535C90B2002BECD100E093
S214009D28002000BD70B500210CE00B1E18BF0123F3
S214009D38202A14BF002303F001037BB92E2A08BF8C
S214009D48012101300278B2F13F0318BF01231F2A10
S214009D5894BF002303F00103002BE6D189B1013834
S214009D68437801382E2BFBD1074D861C002004466D
S214009D782968701CFFF7BCFF20B9601C043508284A
S214009D88F5D10824204670BD5805002070B50A464F
S214009D980646441C032514F8010C4021FBF712FC68
S214009DA82E2300F8013B013415F1FF350246F2D1A7
S214009DB8F0780021FBF706FC70BD0000F0B5002225
S214009DC804460D46002701E00134013226782E2E7F
S214009DD8FAD8032AD4BF00230123002A08BF43F079
S214009DE801036BB92370C2EB0400FBF7C3F9013714
S214009DF8032F287004F8016B03DC01350022E5E721
S214009E0800242046F0BD000070B50A460646441CED
S214009E18052514F8010C4121FBF746F92D2300F817
S214009E28013B013415F1FF350246F2D17079012164
S214009E38FBF73AF970BD0000F0B5002282B0044680
S214009E480F46002601E00134013225782F2DFAD876
S214009E58022AD4BF00230123002A08BF43F00103C7
S214009E680BB1002416E02370C2EB0400FBF768F978
S214009E7802AA02EB06030136052E03F8060C04F8C0
S214009E88015B01DC0022E0E738460DF102010622FC
S214009E98FBF788F9204602B0F0BDC04610B503228D
S214009EA804460A49102002F01DF9094BC0B2187082
S214009EB840B20028B8BF4FF0FF3005DB054B8921BC
S214009EC81C6001F08FFF002010BD0000E19E00001E
S214009ED85205002070080020F0B587B00C9D02924D
S214009EE89FB2AB7846B213F0800F5ED113F0780FAE
S214009EF85BD12B79002B58D16B79012B55D12B7B55
S214009F08202B52D105F10F014FF0000C11F8022C4E
S214009F1811F8013C413A413B03A843EA02130CF806
S214009F2800300CF1010C0231BCF1100FEED1204BC1
S214009F381968FFF7DDFE002206E0202C35D1013235
S214009F4800EB02030F2B30DC03AB9B18C45C002C21
S214009F58F3D16FF07A03AB700123EB711549042235
S214009F68EC706C71AC7105F13200FBF71BF9062337
S214009F7885F837301049042285F8364085F8394088
S214009F8885F8384005F13A00FBF70CF93E220092B6
S214009F98A5F10803304602993A46019401F05CFFA1
S214009FA800B2003818BF012000E0002007B0F0BD5E
S214009FB870080020BA040100050A002010B5084BF6
S214009FC8C4B293F9000000F0B1FF064B01221A70E4
S214009FD8054B20461B6800219847082010BD000046
S214009FE8530500207408002078080020F0B5854B3B
S214009FF8D1B01B78053B0A2B0CD8DFE813F00D0010
S21400A008210028002C003700460061006500B300D8
S21400A018B300DA000020F3E00DF1160420467A4972
S21400A028FBF7FAF8794B00211B6801209847014690
S21400A03807A80138FBF7F0F82046FBF7FDF83DE0E7
S21400A0480DF116007249FBF7E7F80A24B7E06F4BE4
S21400A05806201B6802E06D4B07201B680021984706
S21400A0680DF11601002202F085F827E00DF116041E
S21400A07868492046FBF7D0F8644B00211B6802208D
S21400A088984701460DF122000CE00DF116046249CE
S21400A0982046FBF7C1F85D4B00211B680320984754
S21400A0A8014608A8FBF7B8F82046FBF7C5F80DF1F7
S21400A0B8020380B21B183E221A75013084B27EE075
S21400A0C856490DF1160077E00DF116064F4F30464B
S21400A0D85349FBF7A1F83B6800210320984704463C
S21400A0E821460DF11A00FBF797F82046FBF7A4F86F
S21400A0F8041DA4B206EB04004A49FBF78DF83B683A
S21400A1080021042098470B340546A4B2294606EBDE
S21400A1180400FBF781F82846FBF78EF82418A4B24B
S21400A12806EB04004049FBF777F83B68002102205D
S21400A138984708340546A4B206EB04002946FBF700
S21400A1486BF82846FBF778F82418A4B23619304678
S21400A1583649FBF761F80234354B4FF00002A4B2DB
S21400A1681A802CE0324B51A91B88052021F8023DA5
S21400A178264B1B6898470146BDF842010DF11603A9
S21400A18850B918462B49FBF747F81E4B0E220324F6
S21400A1984FF0080C1A7018E0B0F5967F34BF0446E6
S21400A1A84FF4967422461846FAF7FCFF4FF0000C58
S21400A1B807E021490DF11600FBF72EF804244FF0AE
S21400A1C8080C104B1B780D2B0CD00DF1020101EB7F
S21400A1D804020D231375631C9BB2C9180A220133A7
S21400A1E80A759CB2154B0DF1020193F90000224640
S21400A1F8634600F06DFA00B20028D4BF00200120A4
S21400A20851B0F0BD74080020C00401007808002092
S21400A218C8040100D4040100E4040100F0040100AD
S21400A228F8040100000501000C0501002CF20000EE
S21400A23882080020180501002800010053050020A8
S21400A24830B5C0B21D4D022881B0287004D004284D
S21400A25829D0012823D118E0194C94F9000000F001
S21400A26865FE002394F9000019221649009301F0B0
S21400A278F3FA10F0800F16D1032353204FF416710B
S21400A28801222B70FCF738FB0DE05320FCF70EFB81
S21400A2980D4B08201B680021984700240AE0FFF7AA
S21400A2A8A5FE044600E0002453204FF41671012250
S21400A2B8FCF722FB204601B030BD000074080020E1
S21400A2C8530500207D0800207808002010B50446B5
S21400A2D808B900200FE0014611F8012B4378303A00
S21400A2E892B203EB0213303B4A789BB202EB03129E
S21400A2F8303A90B28C1C364B1B78043B0B2B65D837
S21400A308DFE803F0060B17252D393E4A4F51595EF4
S21400A318B0F5087F5AD1052008E0B0F5147F55D16E
S21400A3282C4B1B7813F0010F1DD00620FFF788FF73
S21400A3384DE0B0F54D7F04D16378562B46D1072003
S21400A348F4E740F20153984240D10E2021E0B0F5E0
S21400A3584D7F3BD16378552B38D10820E6E740F28D
S21400A3683523984201D10920E0E740F23553984258
S21400A3782CD10D200DE0B0F5147F27D10A20D5E7A3
S21400A388B0F5147F01D10B20D0E7B0F5AA6F1DD128
S21400A3980F20FFF713FE1AE0B0F5557F16D10C20F4
S21400A3A8C4E798B905E088B90B4A138803F596738D
S21400A3B813800D20BAE7B0F5147F07D10F20B5E754
S21400A3C840F22123984201D10120AFE7002010BDBA
S21400A3D8740800207C0800208208002000B51FFAB8
S21400A3E883FC1F4B40B293F90030C9B2834232D186
S21400A3F84B1E082B2FD8DFE803F015070D24301D59
S21400A408212E05000A2012E0164B1B78032B24D1B8
S21400A418042010E0134B1B780B2B1ED90020FFF7E7
S21400A42855FF1AE00F4B1B78012B03D90C20FFF7BA
S21400A438C5FD13E00120FFF703FF0FE0FFF7D6FD89
S21400A4480CE0BCF1020F98BF4FF0FF3006D910465B
S21400A458FFF73CFF02E0022000E0002000BD0000FD
S21400A4685305002074080020F0B5154C054694F9ED
S21400A47800301646002BCFB20CDA10207821114A8D
S21400A48801F046F8C0B210F0800F207018BF4FF0E9
S21400A498FF3013D10C4B1B78012B88BF6FF00100DF
S21400A4A80CD8294604220948FAF77CFE084B0220F5
S21400A4B81E60084B1F70FFF7C3FE0020F0BD0000AB
S21400A4C853050020E5A30000740800207D0800203E
S21400A4D8780800207C08002000B5094B8AB01B7855
S21400A4E8807B5BB10DF103010522FAF723FD28B145
S21400A4F89DF8063013B90B20FFF760FD0AB000BDC3
S21400A50874080020054B40B21A68C3B2122B01D952
S21400A518002002E0342303FB002070478808002050
S21400A52800B540B2FFF7EEFF08B9FF2001E090F84B
S21400A538280000BD00B540B2FFF7E4FF08B1038B62
S21400A548438300BDC9B20723402930B5054680F8C5
S21400A5582F3080F828102ED006D804290FD02029AE
S21400A56830D0022934D115E090292BD002D8802982
S21400A5782ED127E0A02925D0B02929D126E005F13B
S21400A5882A0290F93100AB8AEC680621A0474FF002
S21400A5980402AA832869F0B100234374037400F107
S21400A5A83503036043604FF000038381C373038160
S21400A5B8438183730FE04FF03C038383002380F8C6
S21400A5C82F3008E0012385F82F3001E0028B428304
S21400A5D84FF00303AB8330BD30B504680546A64686
S21400A5E81EF8013B0022023B5FFA83FC0B78002032
S21400A5F8CCEB0303013B0B70614604E01302025DDB
S21400A6089BB243EA02024B1ED9B20130FF29F5D1AC
S21400A6180EEB0C0310462B6030BD000010B54FF44F
S21400A628007482B001908DF8001018E08DF80030A4
S21400A638019B13F8012B013A0193072A15D8DFE886
S21400A64802F00E040A0A1414140A01A86946FFF751
S21400A658C3FF044603E001A86946FFF7BDFF9DF85F
S21400A6680030013BDBB2FF2BE0D1204602B010BD24
S21400A67810B540B28CB2FFF745FFC48310BD00008A
S21400A68870B5844681B00D46164661460422002001
S21400A6989CB2FFF783F929460422FFF77FF90222C6
S21400A6A80A49FFF77BF9230A0DF1020102228DF809
S21400A6B802308DF80340FFF771F931462246FFF75E
S21400A6C86DF96FEA000080B201B070BD1C0501008C
S21400A6D8F0B540B287B00491059094B2DDB2FFF7AA
S21400A6E811FF074610B94FF0FF3071E0C38A049A8D
S21400A6F81B0A02F8013BC38A04994B70838A511CD3
S21400A7081B0A5370838A4B700369023182680BB147
S21400A7189B8900E0C38C02EB0300030E0A4602F88E
S21400A728013B030C4B70511C030A53704870FB79AD
S21400A7384A1C5370FB88511C4B707B684A1C1B0ACA
S21400A74853707B68511C4B7097F829304A1C13F0DD
S21400A758020F02F1020102D06023537004E0502376
S21400A76853703B681B193B6097F829300A4645EA40
S21400A778030302F8013BFB8B14341B0A4B70FB8B5C
S21400A788511C4D1C53706A1C0023561C4B70A4B2F7
S21400A7986B705370737007F12A0319460693A5F178
S21400A7A8100223460B48FFF76BFF030A06F8023C25
S21400A7B86870542397F82E2004990293059B0091FD
S21400A7C803930698062180230194FFF757F900B2F1
S21400A7D807B0F0BD050A002000B5022386B080F851
S21400A7E829108DF8143004238DF8153005238DF8BC
S21400A7F81630513B8DF8173069460422002390F92D
S21400A8083100FFF765FF06B000BD000000B585B053
S21400A81869460022002390F93100FFF759FF05B07A
S21400A82800BD000070B544B220468DB2FFF76AFE40
S21400A838294606462046FFF71BFF102386F82930D0
S21400A8483046FFF7E3FF70BD042310B5044680F8D2
S21400A8582930FFF7DBFF20460221FFF773FE04F1DD
S21400A8682A02A38A94F931000121E468A04710BDA2
S21400A878838B00B513B1013B83830CE090F82F302F
S21400A8883BB1013B80F82F304FF003038383012050
S21400A89802E0FFF7D9FF002000BD000000B55FFA10
S21400A8A883FE037B1FFA82FC13F0010F01D1002000
S21400A8B812E04279037943EA0223827943EA0243A3
S21400A8C8C279084643EA0263013363444B6081F861
S21400A8D829E0FFF79BFF012000BD00002B4B70B559
S21400A8E804461868237B9B0803F00103002814BF5E
S21400A8F81E4643F00106002E47D100F56A7500F59E
S21400A9087470042202300C31FAF74CFC6278237813
S21400A91843EA0223AB82A378E27885F82E6043EAFE
S21400A9280223EB82237B13F0100318D0627A237A73
S21400A93843EA0223A27A43EA0243E27A43EA02633C
S21400A948AB60042385F829306279237943EA022329
S21400A958A27943EA0243E27943EA02630EE0AB6077
S21400A968142385F829306279237943EA0223A279E9
S21400A97843EA0243E27943EA026301336B60034B1E
S21400A988186800F56A70FFF741FF70BD8808002058
S21400A998F0B504468CB097B201F10C00009122463F
S21400A9A810313B460290FFF76BFE002840F0B48259
S21400A9B8224612F8011B637843EA0123ADF81C30DF
S21400A9C8531C591C52785B7843EA0223ADF81E30B4
S21400A9D84B1C5A1C49785B7843EA0123511C527871
S21400A9E8481C42EA03224B7843EA02230893431C96
S21400A9F841785A1C5B7843EA0123511C5278481C5C
S21400AA0842EA03224B7843EA02230993431C42781E
S21400AA18591C5B7843EA0223ADF828304B1C4A7869
S21400AA28591C5B7843EA0223ADF82A304B1C4A7857
S21400AA38591C5B7843EA0223ADF82C304B1C4A7845
S21400AA48591C04915B7843EA0223BDF82820ADF828
S21400AA582E30930A03F03C03132B069340F25C82D5
S21400AA68BB4200F259823C2B00F25682DFF8AC3427
S21400AA781E68002E00F0998002F01703022B14BF00
S21400AA8800230123FF22039301920024F28ABDF8D3
S21400AA981E30E5B29A4225D196F82830032B0DD100
S21400AAA8039BFBB1BDF81C000299B082042206F194
S21400AAB82A00FAF777FB86F8315022E2039919B193
S21400AAC8402B04BFEDB20195B28ABDF81C309A42FD
S21400AAD808D106F12A0002990422FAF76FFB00282B
S21400AAE800F00F820134122C01D03436CEE7019ADA
S21400AAF850B2002859DBFFF705FD0646022106F18D
S21400AB082A04FFF71FFD06212246002396F9310086
S21400AB18F568A847BDF81C302046B382029904227F
S21400AB28FAF740FB019886F83100EAE1BDF82810EC
S21400AB3811F004050BD030460221FFF703FD96F905
S21400AB483100B38AF46806F12A020121C5E1049AA5
S21400AB580132202C059200F05E810DD8042C00F0FE
S21400AB68C68103D8032C40F0D78114E0082C4CD0BB
S21400AB78102C40F0D18120E1802C00F08A8103D887
S21400AB88402C40F0C98178E1A02C00F09381B02CCD
S21400AB9840F0C2815DE0082196F9310006F12A02EC
S21400ABA8B38AF468A047022804D107A80099FFF7DB
S21400ABB895FEB1E1042800F0AF8186F8305006987B
S21400ABC84FF00003A0F11401F384C9B20598FFF70B
S21400ABD825FD0821B0843046FFF7B4FC089BD04812
S21400ABE801337360CF4B01781B6843F2D4020B44E1
S21400ABF802FB03F301310170B36030461221FFF700
S21400AC08EBFDB3680133336086E111F0100F00F0F6
S21400AC1883813268099B934240F07E8111F0020FCF
S21400AC28089A08D0531C7360102386F829303046DB
S21400AC38FFF7ECFD03E073689A4240F06D8110233D
S21400AC4886F8293033683046B360B021FFF77AFCBF
S21400AC58D1E011F0020F11D011F0100F0ED0089BA2
S21400AC6872680133934240F057813268099B9342D9
S21400AC7840F05281102386F829308EE0B368D6F863
S21400AC8800C0634501F010032FD0002B00F044816C
S21400AC98002386F8213086F82030099B06F12A0220
S21400ACA8634596F93100F4680DD1B3600321B38A81
S21400ACB8A04710F0080F054610D1738C23BB052358
S21400ACC886F8203020E0C3EB0C030A219BB2A0478D
S21400ACD810F0080F08BF40F0200515D0BDF8283042
S21400ACE813F0010F00F01881B7E063B1002386F86F
S21400ACF8213086F8203096F9310006F12A02B38A08
S21400AD08F4680B21A047002506998F421CD9726863
S21400AD18089B9A4218D17F1A102386F8293002EB2E
S21400AD2807037360059B96F9310003EB0102143A9A
S21400AD380421BBB2F468A047054315F0180F0BD0E2
S21400AD487368DB1B7360E7E015F0200F03D17268A9
S21400AD58089B9A4200D10125BDF8283013F0010F50
S21400AD681FD096F9310006F12A02B38AF468052145
S21400AD78A04728B911233046A02186F8293004E0D8
S21400AD88102386F8293030469021FFF7DBFB7368DE
S21400AD98013373603368013333603046FFF736FD9E
S21400ADA8BAE015F0010F05D1102386F82930304691
S21400ADB8FFF72CFD3046B02175E001F01203122B88
S21400ADC821D1099A33689A4240F0A680089B0698D3
S21400ADD80133A0F114017360B260C9B20598FFF799
S21400ADE81DFCB021B0843046FFF7ACFB86F829403E
S21400ADF83046FFF70BFD96F93100B38AF46806F182
S21400AE082A02022169E011F0100F00F08580304612
S21400AE18FFF71AFD80E001F01103112B13D10999F1
S21400AE28336899420FD10698089BC0EB0702013396
S21400AE3892B29B1873601023B16086F829303046AA
S21400AE48FFF7E4FC2DE0069907A8C1EB070292B2CB
S21400AE5831461023FFF722FD10B13046802122E04C
S21400AE68BDF8283013F0100F56D0099A33689A4266
S21400AE7852D130464021B26015E0069B07A8C3EBC6
S21400AE88070292B231461023FFF708FD002843D088
S21400AE9807E011F0100F09D0099A33689A423BD19F
S21400AEA8B26030460421FFF74DFB35E00698C0EB4C
S21400AEB807021FE011F0100F11D0099A33689A4262
S21400AEC82AD1B26030460221FFF73CFB96F93100E2
S21400AED8B38AF46806F12A020621A0471CE0069900
S21400AEE807A8C1EB070292B23146112306E0069B7B
S21400AEF8C3EB070292B207A831461023FFF7CEFC31
S21400AF080AE0094B1E6096F82840BDF82A00022C75
S21400AF1870843FF60BAE48E60CB0F0BD88080020FB
S21400AF288C080020400A00208408002030B545B26E
S21400AF382846FFF7E7FA044600283AD090F8283063
S21400AF48202B38D009D8042B35D001D8032B02E0A3
S21400AF58082B0DD0102B2CD110E0802B2BD002D82C
S21400AF68402B26D127E0A02B25D0B02B21D10AE0F4
S21400AF788368013383600368013309E020460221B1
S21400AF88FFF7E0FA17E0826803689A420AD1531C72
S21400AF9823601123204684F82930FFF737FC204623
S21400AFA82021EDE790F8303043F0010380F8303088
S21400AFB801E04FF0FF35284630BD0000F0B540B23E
S21400AFC8BDF5B66DDBB202910390019397B2FFF719
S21400AFD899FA0590002800F0128290F82830B02BD5
S21400AFE840F00D8205696DB940F62830FBF7FAFB8C
S21400AFF8002800F004820546059805F1350305612A
S21400B0082B606B60019911F0080F11D06B892A89A3
S21400B0181A4402EB0703B3F52F6FDCBFC2F52F63A4
S21400B02898B240F3ED81029A137885F83430E6E159
S21400B03805F53266029805F135030536069304963B
S21400B04808B900242CE06B892A8968689B18C3F520
S21400B0582F639BB2BB4234BF1E463E46049900EBA4
S21400B06806038B4213D3C0EB0104A4B2224602990E
S21400B078FAF798F8029AC4EB06039FB214440698A7
S21400B08821463A46FAF78EF8069B6B6004E002996A
S21400B0983246FAF787F837466B683446DB196B6032
S21400B0A8019E16F0020F00F0828016F0800F55D130
S21400B0B8EA7B002A00F0A381AB7B9A4203D9022BD5
S21400B0C801D80133AB73BAB2002A3AD0AB899B1ABF
S21400B0D821E0B3F816C02B89059A5B1A2B812B68DA
S21400B0E85B182B60AB895B1AAB8193685B1893601F
S21400B0F8EB7B013BEB736B7C0133DBB2032B6B748E
S21400B10801D900236B746A7C2B7C9A4226D0C1EB4B
S21400B1180003CCEB030398B200B36B7C05EBC303C8
S21400B128998A8842D5D219E005EBC102D28AAB8942
S21400B1389B1AAB814B1CDBB2032B6B7401D9002323
S21400B1486B74697C2B7C8B42EED1AB892A68D2184B
S21400B1584FF000032A60AB81EB732B812B68049EAB
S21400B1686C89B34228BFA3F52F634FF0000228BFAF
S21400B1782B606A81002C6DD195F93430002B00F0D5
S21400B18835818DF8AB258DF8AC2595F834300DF55E
S21400B198B4618DF8AD3501238DF8AE350020223B1D
S21400B1A80B3105228DF8AF35FAF74AF91EE10198FA
S21400B1B810F0040F4BD010F0400F02D100260021EB
S21400B1C821E02B7C05EBC3039C8A1B7E3EE02B7C90
S21400B1D8013BDBB2FF2B2B7401D103232B7436B94A
S21400B1E82B7C05EBC3031B7E13F0200F05D02B7CAE
S21400B1F8012205EBC3035A7601362B7C05EBC30305
S21400B2089B8A0B4499B2EB7B013BDBB2FF2BEB73BB
S21400B218DDD14FF000020023EB732A81AA819EB18C
S21400B2286B8900240B446B8102E044EA00039CB25D
S21400B238013EC0F0E2800398002100224423FFF775
S21400B248BDFE0028F1D1D8E00C4601230193002C5E
S21400B25800F0CC80EA7BAB7B9342C0F0C780032A21
S21400B26800F2C4806B89059E23446B81B4F5AF6FEA
S21400B27834BF23464FF4AF639CB2B18C059B8C4217
S21400B2885A8C059E86BF0C4627464FF4AF6796F83D
S21400B2983030944284BF1446274613F0020F2868BD
S21400B2A80BD1B2EB510F08D24FF0050143F0020361
S21400B2B80024B18386F8303004E0059A23F00203B0
S21400B2C882F83030059E0199738C1B1B73842B897A
S21400B2D800EB03060498864228BFA6F52F661B19BE
S21400B2E82B816B891B1B11F0200F6B8103D010A9D3
S21400B2F822460C393AE0039800F01EFB0028F6D0E8
S21400B30810A90D394FF0000C00221EE03378FF2BF1
S21400B3180CD17B1E9A421ADA4FF0FF3301F8013B34
S21400B328531C9AB20CF101031FFA83FC16F8013B72
S21400B3380B70631E9CB20498069B864228BF1E4666
S21400B348531C9AB2BA4202D20131002CDED16B8964
S21400B358234414466B8111E016F8013B01F8013CC2
S21400B368069B04980131864228BF1E46531E9AB291
S21400B3784FF6FF739A42EFD14FF0000C08A9013937
S21400B388082303982246CDF800C0FFF7A1F90199D3
S21400B39880B203B2A342C8BF204611F0040EDDF8FF
S21400B3A800C021D12B7CA1B205EBC30399822B7C6C
S21400B3B8032205EBC3035A762B7C019A05EBC303DD
S21400B3C8A3F816C02B7C05EBC3031A76AB89C918FD
S21400B3D8EB7BA9810133EB732B7C0133DBB2032BA8
S21400B3E82B7488BF85F810E080B209E06B89234487
S21400B3F86B81019B13F0100F01D0204600E000205F
S21400B4080DF5B66DF0BD000010B51C4C238843B989
S21400B4184CF200032380FBF70DFA800800F5404045
S21400B4282080B4F800C00CF1010398B2144B2080B9
S21400B438D3F800E015E0B0F5404F38BF4FF4404071
S21400B4487246002192F82830022B02D9D38A83420A
S21400B45805D04B1C99B2122909D03432F2E7431CA6
S21400B46898B28445E7D1054B1880002004E0034BCA
S21400B4781880604508BF002010BD00008E08002018
S21400B48888080020F0B589B281B046B200913046EF
S21400B49897B2FFF737F8054608B9002627E090F870
S21400B4A8283013F0070F08BF4FF0FF361FD00323CE
S21400B4B8002480F8283080F83040042200F12A0062
S21400B4C80021F9F767FE009B4FF00002EB824FF071
S21400B4D8FF33AA82AC6085F829202B606C6085F85B
S21400B4E82F201FB940F2B453EB8300E0EF833046B9
S21400B4F801B0F0BD10B544B22046FFF703F808B90E
S21400B508002403E000213422F9F744FE204610BD4B
S21400B518F0B589B281B01646C7B2009162B3184C2E
S21400B528236863B94FF47770FBF75CF91223206041
S21400B538142180F8D93301225420FBF7DDF924685A
S21400B548002294F82830D5B273B920460021342258
S21400B558F9F720FE012384F8283084F82E70009B23
S21400B56868B2E660238309E00132122A02D16FF03E
S21400B578010003E03434E4E74FF0FF3001B0F0BDDB
S21400B58888080020F0B5807B91B0009050E19DF8C7
S21400B59807301BB1412B40F04B810BE1AC4B002729
S21400B5A81B6803F1340515F80C3CA5F13406202B6E
S21400B5B800F0E78009D8082B00F0C380102B00F0B5
S21400B5C8C080042B40F0EB80CFE0802B00F0D980C1
S21400B5D803D8402B40F0E380DEE0A02B00F0D180BB
S21400B5E8B02B40F0DC8015F8043C13F0010F19D09E
S21400B5F855F8342C55F82C3C9A4213D1531C45F870
S21400B608343C112305F80B3C3046FFF7FFF830466C
S21400B6182021FEF797FF15F8043C23F0010305F8F0
S21400B628043CBCE015F8143CD3B1013BDBB205F88A
S21400B638143C002B40F0B38015F8132C854B042AD5
S21400B6489B5C05F8143C02D8531C05F8133C35F8E7
S21400B658203C55F8284C06F12A0238460C2119E0F9
S21400B66835F81A2CC2B955F8343C3046013345F83B
S21400B678343C112305F80B3CFFF7C8F83046202168
S21400B688FEF760FF35F8203C55F8284C06F12A02EC
S21400B69838460521A04782E04FF6FF739A4202D04B
S21400B6A8531E25F81A3C15F8043C13F0020F25D152
S21400B6B855F8342C55F82C3C9A423FD035F8183CAF
S21400B6C8E3B155F8241C002938D04A7C4FF0030C07
S21400B6D80B7C9A4202D1CB7B042B2FD101EBC20004
S21400B6E8437E1BB1013BDBB243763BB10132032AF2
S21400B6F8C8BF0022BCF1010C20D3E9E715F8053CC9
S21400B708002B00F09F8055F82C2C55F8343C55F843
S21400B718284C9B1A45F8342C9BB238460721002241
S21400B728A047002800F08E804FF0020325F8183C4A
S21400B73815F8053C013B05F8053C30E035F8183CA3
S21400B74816E03046FFF794F848B315F80C3C102B73
S21400B75806D14FF002033046022125F8183C01E0D6
S21400B76830461221FFF738F819E035F8183C1BB1B7
S21400B778013B25F8183C12E030460221FEF7E2FEAF
S21400B7880DE03046FFF774F848B1112305F80B3C76
S21400B7983046FFF73BF802E03046FFF769F8013716
S21400B7A83435122F7FF4FFAE542014210122FBF704
S21400B7B8A3F83DE0264E9DF80820009829463468F0
S21400B7C8F9F7B8FB9DF80430032B23D0042B2FD1B0
S21400B7D89DF80530342203FB02F104EB010090F8D3
S21400B7E82830102B03D10221FEF7F6FF20E0C568AB
S21400B7F855B18268635890F931009B1A62509BB223
S21400B80807210022A84713E0306800F56A70FEF7A3
S21400B818FDFF0DE09DF80520342302FB0343DC689A
S21400B82834B193F9310003F12A0209219B8AA04713
S21400B83801AD009829460522F9F77CFB00287FF41D
S21400B848A6AE03E03046FEF7FFFFA8E711B0F0BD4E
S21400B858880800201E050100F0B584B09EB2BDF829
S21400B868243040B292B202910390019200930746A8
S21400B878FEF748FE0546002846D026B9FFF7C4FD61
S21400B8880646002840D095F8283013F0030F0ED14E
S21400B89813F0440F38D028460221FEF753FE95F9D8
S21400B8A8310005F12A02AB8AEC680621A04705F1AB
S21400B8B82A0002990422F9F775FC019BEE82AB82F6
S21400B8C8002385F83030009B13B940F2B45300E0EB
S21400B8D8009BEB830F48104B01781B6843F2D40299
S21400B8E80B4402FB03F301310170AB6001332B609C
S21400B8F8039B2846022185F83130FEF76DFF28465F
S21400B9081021FEF71FFE01E04FF0FF37384604B05F
S21400B918F0BD00008C080020400A0020054B42B20B
S21400B928186810B905E0002003E090F90A30934241
S21400B938F9D170479008002000B540B2FFF7EEFF37
S21400B948838813F4906F0CBF0020012000BD000010
S21400B95800B54FF0FF3381B08DF801308DF8021036
S21400B9688DF803200DF101010322212390F90A0026
S21400B978FFF724FB01B000BD30B540B20D46FFF717
S21400B988CDFF0446002840D00A2D3ED8DFE805F053
S21400B998060E181C2024282C30343A00FB210122DD
S21400B9A8FFF7D6FFA38843F0100306E0FC21012228
S21400B9B8FFF7CEFFA38843F040030120A38025E0CD
S21400B9C8838843F020031FE0838823F020031BE0CE
S21400B9D8838823F0840317E0838843F0040313E086
S21400B9E8838843F400630FE0838823F4006306E04B
S21400B9F8838843F4806307E0838823F480631B040A
S21400BA081B0C01E04FF00003A380002030BD0000AF
S21400BA18F0B5174C5BB281B00093236887B28DB23D
S21400BA2896B233B91020FAF7DDFE4FF0FF332060E8
S21400BA3883724FF0FF30FFF771FF044610B94FF0DE
S21400BA48FF3012E029460B4A1020FFF761FDA0726E
S21400BA58069BE7802360009B2681237340B2394605
S21400BA683246FFF70FFD94F90A0001B0F0BD00005A
S21400BA7890080020A5BA000030B545B22846FFF762
S21400BA884DFF044640B12846FFF734FD0023E37215
S21400BA98A3804FF0FF33A37230BD0000F0B547B265
S21400BAA884B038460092CCB29EB2FFF737FF054600
S21400BAB810B94FF0FF3070E1631E092B00F25A816F
S21400BAC8DFE813F01F00190059008A00310038001B
S21400BAD879000A0058014900C37A002B40F04C81CF
S21400BAE8046808213846009AA047022800F04481D6
S21400BAF80123EB723EE102230468C3720221384632
S21400BB0814E0A74BC1881B6838461A89FFF7BAFCA9
S21400BB180023EB724FF00002AA802C6838460121F9
S21400BB28009A3346A0472C6838460521009A3346C3
S21400BB38A04732E104680621009A33463846A047F3
S21400BB480023EB72AB80964BE9881B6838461A8947
S21400BB58FFF798FC0EE1007B18B140B20421FAF713
S21400BB6805FF3846002132460223FFF727FA002849
S21400BB7800F000812EE0007B18B140B20421FAF7ED
S21400BB88F5FE0021002202233846FFF717FA0321A4
S21400BB98041E18BF0124002200232D683846A84733
S21400BBA844EA000010F0080F00F0F7803846FFF768
S21400BBB8BDF90820F1E03846002100220423FFF7EB
S21400BBC8FDF9002800F0D68038460021002282239E
S21400BBD8FFF7F4F90120E0E0828840F6040302EA61
S21400BBE80303042B02D100210191B9E04FF6FF634D
S21400BBF8009C02EA0303B6B202F4807100220396A0
S21400BC0883800294019273E0237819B1FF2B40F0E9
S21400BC18B58065E0FF2B5CD1731E01349EB24FF4ED
S21400BC28807165E0012E4CD9FB3B601C032B48D87D
S21400BC38DFE803F02F3D021A0378012B0FD112F02C
S21400BC48100F04D042F0010323F010031FE012F097
S21400BC58010F04BF42F00103AB8003D095E0002B30
S21400BC6840F09180FB2123E00378012B40F08B8085
S21400BC7803F57E4303F5FE73013302EA030312F06D
S21400BC88400FAB807FD04FF6BE7302EA0303AB804B
S21400BC987BE003785BB92846FD210022FFF758FEB3
S21400BCA8AB8843F0800323F00103AB8004E0FE2159
S21400BCB802782846FFF74CFE002866D0012201923B
S21400BCC863E0731C02999EB24FF0FF3301F8013B04
S21400BCD8029114F8013B029A02F8013B029206E030
S21400BCE802994FF0FF3301F8013B0134029100211D
S21400BCF8039A531E9BB20393039A4FF6FF739A4216
S21400BD0882D1AB88B6B241EA0303AB80002E27D0B7
S21400BD1813F0010F24D013F0200F0FD000990B78E2
S21400BD28082B03D11F493846032211E03A2B0BBFD4
S21400BD3800991D4938463846012209E032463846F9
S21400BD4800990123FFF73AF9019A0243019207E0A6
S21400BD580123FFF733F9019B002818BF012301933D
S21400BD6804212C683846009A3346A047019941EAD0
S21400BD78000012E0002010E002200EE0AA8812F070
S21400BD88040F9ED14EE7FC2192E7039AB31E9EB29B
S21400BD98531E9BB202340393A9E704B0F0BD00001B
S21400BDA8900800202405010018EE00000C4B1A68C5
S21400BDB81FFA80FC8AB100211379C8B2022B04D17D
S21400BDC8D388634501D140B209E00131042902D184
S21400BDD86FF0120003E00C32EEE76FF013007047C6
S21400BDE8940800200D4B40B21A680428D4BF0023DC
S21400BDF80123002A08BF43F0010389B213B16FF08C
S21400BE080C000AE011B96FF00D0006E000EB4003E5
S21400BE1802EB830302221A71D98070479408002027
S21400BE28F0B580B282B01F468EB2D5B2FFF7BEFF1D
S21400BE3840B200280CDB074B00EB400219680023D1
S21400BE480093019351F82240334629463A46A047C4
S21400BE5802B0F0BD94080020F0B58AB047B206914B
S21400BE681E4694B2BDF83C109DF94020414B042F65
S21400BE78059104921D68C8BF6FF00C0077DC069821
S21400BE883D490422F9F79AF908B90F386FE014B952
S21400BE986FF00F006BE007EB470305EB83000379B1
S21400BEA8022B18BF6FF0100061D1C28812B96FF06C
S21400BEB811005CE0059901F108039BB2B3F5B86F71
S21400BEC834BF1D464FF4B865130A324602F8013BE4
S21400BED8C388511C7370230A53704B1C4C705A1C31
S21400BEE8290A0791ECB25970511C547000234A1C59
S21400BEF84B70511C08915370037A13F0010F2AD027
S21400BF081E4904220020FDF749FD06990422FDF784
S21400BF1845FD1B490222FDF741FD079A0DF1260152
S21400BF288DF8262002228DF82740FDF737FD31468A
S21400BF382A46FDF733FD6FEA000080B228B900F5FF
S21400BF487E4000F5FF70013000E080B20899030AD1
S21400BF5801F8013C0870049A069802921121002202
S21400BF688023009601950397FDF788FD00B20AB076
S21400BF78F0BD000094080020E4050100050A002032
S21400BF88270501000C4B10B51A6844B2042CD4BF20
S21400BF9800230123002A08BF43F0010313B16FF002
S21400BFA80C0008E004EB440002EB800000210C22A1
S21400BFB8F9F7F0F8204610BD94080020F0B585B2D1
S21400BFC801EB05030C46495D9CB002915A1C5B7850
S21400BFD80593531C92F801C05A1C5878531C591CD8
S21400BFE852785B7843EA0226072E72D94A1C0492D6
S21400BFF8497840EA0C2006915378571C0793FFF7B8
S21400C008D5FEC0B241B20029039020DA04F1100030
S21400C01831490422FDF7EEFC00285AD103230021FB
S21400C028062209A88DF822308DF82330F9F7B2F8E1
S21400C038214605F108020DF12A00F9F7B3F805F1D3
S21400C048100189B20DF12200FDF7ECFB41E0234B0D
S21400C05801371A6801EB410302EB83052B7A13F0CC
S21400C068020F26D00799069A51EA022121D0042207
S21400C07804F110010020FDF791FC042204F10C01E4
S21400C088FDF78CFC02221649FDF788FC330A0222CB
S21400C0980DF16E018DF86E308DF86F60FDF77EFC41
S21400C0A8049B3246991FFDF779FC4FF6FF739842BA
S21400C0B80FD1039904F10C0248B2059C0299009727
S21400C0C844EA0123A6F1080189B201912C680121EE
S21400C0D8A0471CB0F0BD0000090A00209408002004
S21400C0E827050100F0B5174C0D462368C6B2D7B22F
S21400C0F81BB93020FAF776FB2060226815B96FF076
S21400C1080A001DE013790BB9002010E00C321379F1
S21400C1180BB901200BE00C3213790BB9022006E0AC
S21400C1280C32137913B16FF00B0009E003200123DA
S21400C13813714FF000035671D3801772156040B222
S21400C148F0BD000094080020C0B2192898BF00F17E
S21400C158410303D9332803D800F14703D8B207E0D0
S21400C1683D2801D8031FF9E73E2814BF2F202B20AF
S21400C17870470000F0B50E4681B00AB9009206E096
S21400C1880092C41C00274EE0009B01330093009ADF
S21400C198135C262BF8D8F4E714F8030C3546800809
S21400C1A8FFF7D2FF05F8010B14F8033C009A03F0DA
S21400C1B803031B01012A07F1020711D014F8020C29
S21400C1C8B51C43EA1010FFF7BFFF707014F8023C66
S21400C1D8009A03F00F039B000334022A06D119E0E5
S21400C1E81846FFF7B1FF70706E1C1AE014F8040CBE
S21400C1F8023743EA9010FFF7A7FFB07014F8040C54
S21400C20800F03F00FFF7A0FFF070009B0436033BEA
S21400C218009308E01846FFF797FF05F8010B01376B
S21400C2282E46314607E0009A002AB5D1F9E73D23A5
S21400C23801F8013C0137013117F0030FF7D13846F2
S21400C24801B0F0BD30B501304FF0000C00250024D9
S21400C2584FF0000E3BE0DAB22B2A14BF002301236E
S21400C2682F2A08BF43F00103CBB9A2F13003DBB293
S21400C2784A2B2BD8392A01D8131D03E0602A04D983
S21400C288A2F147035FFA83FE0BE05A2A1ED8402A1B
S21400C29888BFA2F14103F5D83D2A17D11EE04FF01A
S21400C2A83F0E0EEB8C1C022D0ED94FEA1C43012CB8
S21400C2B801F8013B0FD84FEA1C2301F8013B54B99B
S21400C2C801F801CB002501E06B1CDDB2013010F847
S21400C2D8013C0D2BBFD126230B7030BD631C0EEB23
S21400C2E88C1CDCB2DFE70000013001314FF0000C97
S21400C2F80EE010F8013C934201D001200DE00CF14D
S21400C30801035FFA83FC01300131BCF1080F03D04A
S21400C31811F8012C262AECD10020704730B5CCB293
S21400C328024614F0080F0CBF3A200D20114600E014
S21400C33801310B780BB18342FAD114F0040F02D006
S21400C3483A2B17D11BE026230B70154614F0010F65
S21400C35806D00E4B114618680E30FFF7C5FF48B9D1
S21400C36814F0020F09D0094B294618681630FFF753
S21400C378BBFF10B14FF0FF3006E0002004E0262394
S21400C38801F8013B0D46E1E730BD0000DC06002061
S21400C39810B58C4610B90846012400E000249CF825
S21400C3A800300130421E2B2B01D120231DE0252B07
S21400C3B817D19CF801200CF10103303A03F1010C67
S21400C3C85B78D2B2303B092AD9B202D9D31F03F020
S21400C3D80F02092902D9CB1F03F00F0141EA021305
S21400C3E803E0262B01D82CB123B10CF1010C00F880
S21400C3F8013CD4E7002302F8013B104610BD0000BC
S21400C408F0B582B08DB207991E460C881168631E77
S21400C4181FFA83FC01EB05030090043B01EB0C00BC
S21400C42883421746C5EB000E23D900EB0503089A8E
S21400C438043B934212D22A1F92B20CEB02031FFA55
S21400C44883FC04EB0203079C8018238033889644F9
S21400C4581344C2F10002338001920CE0C1EB0003E2
S21400C468181D3388CCEB0303043B338000233B6062
S21400C4783EE000230193032D15D90EF104018842EE
S21400C48801D1002208E0C5EB0C0304339AB203E09E
S21400C49811F8013D00F8013D531E9AB24FF6FF739E
S21400C4A89A42F5D111E001EB050062460438F8F728
S21400C4B879FE3C680099043C20462A46F8F772FE46
S21400C4C86419C5F104003C6012E03C682A46043C46
S21400C4D8204600996419F8F765FE3C60079C2A1FF9
S21400C4E8238892B29B1A2380338801989B1A33803C
S21400C4F802B0F0BD0F4B43F820200F4A00F11F038F
S21400C50800EA020213EA200338BF0346002AC9B22B
S21400C5184FEA631C05DA013A6FEAC2626FEAD26232
S21400C528013201239340054A42F82C30044BC1548B
S21400C53870470000400000201F00008000E100E077
S21400C54800E400E0074B00221A6002F1804202F580
S21400C558143202F57E720432136883F00103136006
S21400C568704700000C00004072B6024A1368013398
S21400C57813607047D4090020034A1368013B136010
S21400C58803B962B670470000D4090020074A084B72
S21400C5981A60084A4FF00053DA63074A136843F0F4
S21400C5A8E0631360054B07221A6070479F25260034
S21400C5B814E000E065DB000020ED00E010E000E09D
S21400C5C8074B20221A6040F0010020331860044B05
S21400C5D81B6813F0200FFAD0024B186880B2704719
S21400C5E80080044030800440074B89B2196020223E
S21400C5F82C3B1A6040F0030020331860034B1B687E
S21400C60813F0200FFAD070472C80044000800440B6
S21400C61881B04FF6FF73009306E0009B013B009342
S21400C628009B0BB9012005E0034B1B6813F0010FB4
S21400C638F3D1002001B070473880044004207047CA
S21400C648014B53F820007047E8090020014B186892
S21400C65870470000E40900200649074A0B684FF0B7
S21400C668000052F823200133032BC8BF0023108094
S21400C6780B607047D8090020E809002030B584B25E
S21400C688091BA4F10E0301F8023C1B1201F8013C39
S21400C6984D1EFFF7BDFF08B100200DE0691EA31C64
S21400C6A898B20A68054B04281A6002D90431031F99
S21400C6B8F6E7034B01221A6030BD000010800440E4
S21400C6C838800440C0B2012800B507D002D302283B
S21400C6D80DD107E0064A0520062106E0054A062091
S21400C6E8062102E0044A21200621FFF703FF00BDC9
S21400C6F825D70000E1D600009DD600007047000050
S21400C708C0B210B1012816D10AE021B10A4A13684E
S21400C71823F002030EE0084A136843F0020309E018
S21400C72821B1054A136823F0010303E0024A13689F
S21400C73843F0010313607047FC73004030B58DB2B8
S21400C74815F4C05FC4B274D015F4006F2DD014B1C0
S21400C758012C26D113E0404A136843F008031360FF
S21400C768A2F57622A2F53E620C3A136843F002035D
S21400C7781360A2F58E72136843F0020310E0364A7F
S21400C788136843F008031360A2F57622A2F53E620A
S21400C7980C3A136823431360A2F58E72136823437A
S21400C7A8136020460021FFF7ABFF15F4805F40D0EA
S21400C7B8012C17D002D3022C3BD126E0264A136858
S21400C7C843F001031360A2F57822A2F5DF520C3A73
S21400C7D8136843F008031360A2F58E72136823F0FB
S21400C7E8080325E01C4A136823431360A2F5782241
S21400C7F8A2F5DF520C3A136843F080031360A2F5E3
S21400C8088E72136823F0800312E0134A136843F00D
S21400C81801031360A2F57822A2F5DF520C3A1368DA
S21400C82843F040031360A2F58E72136823F04003AA
S21400C838136040F2011305EA030313B120460121F1
S21400C84806E040F2022305EA03031BB12046002156
S21400C858FFF756FF30BD000008E10F40C0B2C2B275
S21400C868012A30B50D4608BF6C4C07D038BF6C4C53
S21400C87804D36C4B022A0CBF1C4600240023012854
S21400C88823631ED002D3022867D140E0664A1368A5
S21400C89843F001031360C03A136823F001031360E2
S21400C8A8136823F001031360BC32136843F00103D6
S21400C8B81360C03A136823F001031360A2F57822C8
S21400C8C83FE0594A136843F008031360C03A1368F8
S21400C8D823F008031360136823F008031360BC32C0
S21400C8E8136843F002031360C03A136823F0020388
S21400C8F81360A2F57622A2F54262043A136843F062
S21400C9080C031360FC32136843F00C0324E0464A19
S21400C918136843F040031360C03A136823F04003DB
S21400C9281360136823F040031360BC32136843F0A7
S21400C93804031360C03A136823F004031360A2F5D7
S21400C9485622A2F5E152043A136843F00303136033
S21400C958FC32136843F0030313602B6813F0400F90
S21400C96804D04FF4C0510022FFF7E8FEEB7A0B2BF9
S21400C97828D8DFE803F00C1014181C2024272A2DCA
S21400C98806091B22082325E00D22242322E042F66E
S21400C998B0022B231EE041F2584215231AE040F657
S21400C9A82C220B2316E040F21652052312E040F222
S21400C9B88B2203230EE040F2451221230AE0D922F7
S21400C9C8012307E0A222312304E05122182301E0C4
S21400C9D8362210236262A3622B6813F0060208BF91
S21400C9E8E26206D013F0040F01D0022300E006230B
S21400C9F8E3622B6813F0100F1EBFE36A43F00803C8
S21400CA08E3622B6813F0010FE36A14BF43F0400398
S21400CA1843F06003E3620123236330BD00D0004087
S21400CA2800C0004000E0004008E10F40074B1A60D5
S21400CA38043B1960064A40F0244343F48403136019
S21400CA48034B1B680342FBD17047000004D00F401D
S21400CA5808D00F4030B520F47E740D4624F0070445
S21400CA68084B002202201A602146FFF7DFFFB5F5C3
S21400CA78806F04D904F58064A5F58065F0E700208A
S21400CA8830BD00000C00004070B520F00304236899
S21400CA981546001B4E1C17E0C100FF228A4023EAF9
S21400CAA8020216F8013C8B40032842EA030309D128
S21400CAB8012021461A46FFF7B9FF65B154F8043F2E
S21400CAC8002000E001300136013DE5D20120214674
S21400CAD81A46FFF7ABFF002070BD000000B54FF404
S21400CAE80061FFF7B7FF00BDF0B5C0B282B09EB2D6
S21400CAF8552310F0800F00928FB28DF8073001D1C1
S21400CB08002502E000F07F00012510F0400F0AD053
S21400CB184FF4C030FFF7E2FF4FF4C430FFF7DEFFF4
S21400CB284FF4C03405E0022814BF4FF4C0344FF465
S21400CB38C4347EB94DB1B4F5C03F14BF4FF4C0300D
S21400CB484FF4C430FFF7CAFF19E02046FFF7C6FFC8
S21400CB58AFB11BE004EB0700009932460230FFF73E
S21400CB6893FF20460DF107010122FFF78DFF6DB9EF
S21400CB78601C0DF107010122FFF786FF06E020463C
S21400CB880DF107010122FFF77FFFF1E7002002B051
S21400CB98F0BD000030B5417A0546CAB22AB13E4B10
S21400CBA8012A0CBF1C46002400E03C4C002931D169
S21400CBB83B4A08201368042143F002031360C03A76
S21400CBC8136823F002031360136823F0020313604C
S21400CBD8BC32136843F480531360C03A136823F4D6
S21400CBE880531360A2F57822A2F54262043A1368CD
S21400CBF843F00C031360FC32136843F00C03136015
S21400CC08103A136843F00C031360264B01221A608F
S21400CC18254A30E0224A25201368042143F0010300
S21400CC281360C03A136823F001031360136823F0F7
S21400CC3801031360BC32136843F480431360C03AA0
S21400CC48136823F480431360A2F57822A2F5E15214
S21400CC58043A136843F0C0031360FC32136843F0C9
S21400CC68C0031360103A136843F0C00313600F4BF9
S21400CC7801221A600E4AFFF73DFC28881023322846
S21400CC88236206D0B0F5C87F01D1052302E0182339
S21400CC9800E03123E36030BD00100240000002408F
S21400CCA808E10F401C000240B9D500001C100240E5
S21400CCB895D50000C9B2CAB232B1304B012A0CBFB2
S21400CCC89C464FF0000C01E0DFF8B4C0436813F848
S21400CCD8012B8275C2684360934224BF0368436091
S21400CCE8436813F8012BCCF80020C26843609342CF
S21400CCF824BF03684360DCF8003013F0010F1BD034
S21400CD08837D012B01D1072300E00B23CCF80430E8
S21400CD186FF03F03C375038A4268033B0382194BCF
S21400CD2853F8211012F8013B0B76C36842609A420A
S21400CD3824BF0368436020E0436813F8012BCCF84F
S21400CD4808204360837D012B01D1072300E00323DD
S21400CD58CCF804300123CCF810304268C3689A42F5
S21400CD6828BF0368827D28BF43604023C375038AB3
S21400CD789B1A013B013A03828275704700100240F5
S21400CD88000002405C0700201E4A012330B51360ED
S21400CD981D4B00201A6805E022B11C4B01301B68A9
S21400CDA822F8023B1A4B1B6813F4807FF4D0DFF896
S21400CDB864C0DFF854E0BCF80010CEF80020012963
S21400CDC8154D0CD8154A164C136823F48033136097
S21400CDD8012323602B6898470023236011E02B6803
S21400CDE81BB14B1EACF8003003E0A2EB4003CEF8B4
S21400CDF800300C4B1B6813F00F0F02D10A4B0122B0
S21400CE081A6030BD0C800340D009002048800340DB
S21400CE184C800340CC090020C809002000E10F40E0
S21400CE28D40900201480034028800340F0B5037915
S21400CE3883B0012B064600F0FA8003D3022B40F09D
S21400CE484F8246E1C27901239340DDB2002D00F0FF
S21400CE5847828379062B08D8DFE803F0090C0F12FF
S21400CE6815180400DFF87C4412E0002410E0DFF810
S21400CE7878440DE0DFF874440AE0DFF8744407E00D
S21400CE88DFF8704404E0DFF8704401E0DFF86C4433
S21400CE98082B00F22582DFE803F0050E172029325A
S21400CEA83B444D00DFF85834DFF858C403EB8207DC
S21400CEB80020012147E0DFF85034DFF850C403EBC8
S21400CEC88207012002213EE0DFF84434DFF844C43C
S21400CED803EB82070220042135E0DFF83C34DFF854
S21400CEE83CC403EB8207032008212CE0DFF830342B
S21400CEF8DFF830C403EB82070420102123E0DFF8B4
S21400CF082834DFF828C403EB82071E2020211AE005
S21400CF18DFF81C34DFF81CC403EB82071F2040210F
S21400CF2811E0DFF81434DFF814C403EB820720207E
S21400CF38802108E0DFF80834DFF808C403EB82072E
S21400CF4836204FF4807133688BB9737A082B0ED06D
S21400CF58636923EA05036361002B40F0C18103F18E
S21400CF68604303F56043022203F5C073B7E1F64A4F
S21400CF7813680B431360C03A136823EA010313606F
S21400CF88636A6FEA05010B4063626368A2680B4038
S21400CF986360D4F820312B43C4F82031337A012B50
S21400CFA810D902EA0103A360337A042BE36802D19E
S21400CFB82B43E36015E00B40E360337A2269032BCA
S21400CFC809D00BE0E3680B40E36042EA0503A36080
S21400CFD8337A226913B942EA050301E002EA01033B
S21400CFE82361737A022B09D0082B0CD0012B13D19E
S21400CFF8D4F814312B43C4F814310DE0D4F81831A2
S21400D0082B43C4F81831D14B1B6813F0020F0AD112
S21400D018CF4B10221A6006E0256271796246FFF748
S21400D02869FA33683B6063692B43636158E1847A25
S21400D038032C00F355814FF4803202FA04FCC549EC
S21400D04802F180420B6802F56E2243EA0C030B607D
S21400D05802F58272230303F180451368022C43EA23
S21400D0680C0305F54035136001DD232002E063005C
S21400D07803F11300B74A136823EA0C0313603368F6
S21400D08853B1B54B717953F82420FFF733FAB34BF5
S21400D098326843F824200123AB61F38813F0020FAB
S21400D0A801D0022300E001236B60F388328913F075
S21400D0B8010F14BF4CF25033322302FB03F3AB626A
S21400D0C8F38813F0080F01D0212300E00123EB605A
S21400D0D806E1036913F4801F0DD0A14B00221A60E5
S21400D0E802F1804202F57E2202F58072136823F46C
S21400D0F880331360F4E013F4804F0FD0816969B170
S21400D108828A06E0974B1B681AB121F8023B531E29
S21400D1189AB2954B1B6813F4807FF3D0316911F4EB
S21400D128805C40F0DD8011F4004F00F0D2808F4A1A
S21400D1388F48136843F480331360A2F54622A2F59D
S21400D14880721368F56823F00103B76813600368F4
S21400D15823F00F02874B026001EA0303002B69D015
S21400D16811F4403F2BD033698DF804C003F44033E4
S21400D178B3F5003FCDF800C007D0B3F5403F06D062
S21400D188B3F5803F06D1032302E0022300E0042320
S21400D1988DF8083001238DF8063002238DF8053007
S21400D1A804238DF80730684608238DF80930FFF702
S21400D1B83DFE6F4A136843F0040313603BE011F02A
S21400D1C8404313D0B3F1004F09D0B3F1404F0AD013
S21400D1D8B3F1804F08BF42F0010302D02BE042F0C3
S21400D1E80203036027E042F00303FAE711F0005F4A
S21400D1F818BF42F00503F4D111F048631BD0B3F111
S21400D208806F0ED003D8B3F5000F14D106E0B3F143
S21400D218006F09D0B3F1406F0DD108E042F0060365
S21400D228DFE742F00703DCE742F00803D9E742F0FD
S21400D2380903D6E70260B27D4F4B00211A604FF013
S21400D248000E002400204FF0010C47EA05031CEAF4
S21400D258030F14D01CEA050F0BD010F0010F0ED1E7
S21400D2688B0001229A40144342089A404EEA020E66
S21400D27804E08B0010FA03F34EEA030E0131072888
S21400D2884FEA4C0C01D00130DFE749B34B1E9B0038
S21400D29806229A40394B44EA0202C3F800E00433F7
S21400D2A81A607179364A0E20FFF724F93268354B32
S21400D2B81A60354BB28A1A80B269344B1A60284A0B
S21400D2C8136843F001031360083A136843F0010338
S21400D2D81360336913F0100F02D02D4B01221A6029
S21400D2E803B0F0BDFC630240FC430040FC53004022
S21400D2F8FC630040FC730040FC430240FC530240C1
S21400D30898080020A1DE0000B808002051DE0000C2
S21400D318D808002005DE0000F8080020B9DD000067
S21400D328180900206DDD00003809002021DD000006
S21400D33858090020D5DC00007809002089DC0000A8
S21400D348980900203DDC000008E10F4000E100E0FD
S21400D3581C54004044E00F40F0050100B8090020C6
S21400D36808800340488003404C80034000E10F409B
S21400D37814800340000083EC308003404080034064
S21400D38891CD0000C8090020CC090020D009002053
S21400D398288003400C4A136843F00803136002F120
S21400D3A85A4202F53D02094B02F58A6201321A60BA
S21400D3B800224FF080431A6002F1804208320223AE
S21400D3C8136003231360FEE700E10F40000C0040E3
S21400D3D87047000070470000704700007047000064
S21400D3E87047000070470000704700007047000054
S21400D3F87047000081B000EB80000090009B013B66
S21400D4080093009BB3F1FF3FF8D101B070470000CE
S21400D418164A174B1749C2EB030003E011F8013C04
S21400D42802F8013C144B0132034401319A42F5D10B
S21400D438124A134B1349C2EB030003E011F8013CF0
S21400D44802F8013C104B0132034401319A42F5D1EF
S21400D4580E4A0F4BC2EB030102E0002302F8013C20
S21400D4680C4B01320B449A42F7D170471C0500203A
S21400D4787C050020780601001D0500200820000015
S21400D488BCE2000008200000092000007C050020FF
S21400D498440A00207D0500204FF0000E7AE270470F
S21400D4A8D0F800D0D0F804F070470000F0B592F934
S21400D4B817300E46002B1446C7B2957D35DA314A2A
S21400D4C8DDB16B1EA37552F82710B2688B6803F897
S21400D4D8012B8B60A37D0BB9052300E0092373603D
S21400D4E8284B53F82700038A826801330382C368EF
S21400D4F89A4224BF0368836042E052F82720938A42
S21400D508107E0133938250B172B61F4B40B21A6830
S21400D518042101321A60F9F729FAFFF72DF8238A51
S21400D528002B29D13561E5752AE09DB16B1E9375F0
S21400D538536813F8012B8A606360A37D0BB9052333
S21400D54800E0012362687360E3689A4224BF236898
S21400D558636015E0138A7BB90B61107ED37578B1CA
S21400D56872B6094B40B21A68042101321A60F9F7FC
S21400D578FDF9FFF701F803E020463946FFF79AFB66
S21400D588F0BD00005C070020D4090020054B0122EE
S21400D5981A60054B00B55A6801200449FFF786FF54
S21400D5A800BD00001C100240380A0020001002408F
S21400D5B8054B01221A60054B00B51A68002004497D
S21400D5C8FFF774FF00BD00001C000240380A002068
S21400D5D800000240034600B508461946F7F7E2FD84
S21400D5E800BD000070B5C0B289B2022814BF4FF45F
S21400D5F8C0304FF4C43040189EB2851C07E0541C57
S21400D608284611460122FFF7E5FF01352246731E1C
S21400D6189EB24FF6FF739E42F1D1002070BD000007
S21400D62810B581B0C4B202224FF4C0300DF1020129
S21400D638FFF7D0FF9DF80230002C0CBFFF245524BE
S21400D648552B05D19DF80330A34201D1012011E0E6
S21400D65802224FF4C4300DF10201FFF7BBFF9DF81C
S21400D6680230552B05D19DF80330A34201D1022084
S21400D67800E0002001B010BD054B01211B6800B575
S21400D68881EAD30101F001010020F8F713FB00BD81
S21400D698FC43004010B516E0236813F0100F08D0BE
S21400D6A80B4B10221A60443B18680221C0B2F8F7E8
S21400D6B819FB236813F0200F05D0054B20221A60AB
S21400D6C80220F8F7EDFA034C2368002BE4D110BDCE
S21400D6D844E0004040E0004010B516E0236813F030
S21400D6E8100F08D00B4B10221A60443B1868012113
S21400D6F8C0B2F8F7F7FA236813F0200F05D0054BE9
S21400D70820221A600120F8F7CBFA034C2368002B76
S21400D718E4D110BD44D0004040D0004010B516E01B
S21400D728236813F0100F08D00B4B10221A60443BE6
S21400D73818680021C0B2F8F7D5FA236813F0200F4E
S21400D74805D0054B20221A600020F8F7A9FA034CEA
S21400D7582368002BE4D110BD44C0004040C0004000
S21400D768634A70B51368418843F0A0431360C03A13
S21400D7781368064623F0A043136002F1404202F500
S21400D78808025C4B02F5364237321A60C37A027BCF
S21400D7981B0443EA0263427A1343827A11F0080FA5
S21400D7A843EA0223544A1360827B437B43EA0223FC
S21400D7B8524A136001D0162200E00622504B11F0A0
S21400D7C8200F1A6001D01C2200E018224D4B1020B2
S21400D7D81A60FEF7F5FE04041820FEF7F1FE4A4B21
S21400D7E8044324F00F049C4240F08080708810F0B8
S21400D7F8040F23D03E49454A0B6843F020030B60CC
S21400D808136823F020031360136823F020031360C3
S21400D8180B6843F080530B60136823F08053136043
S21400D828A2F55822A2F54262083A136843F00C03A0
S21400D8381360FC32136843F00C03136010F0030FF8
S21400D84808BF4FF490510ED010F0020F0CBF002105
S21400D8584FF4005110F0080F05D0002914BF4FF4FC
S21400D86804514FF4807110F4807F18BF41F4804152
S21400D8780020FEF7B9FEB388254A1380023300E07D
S21400D888631C9CB214F0030FFAD1224D2046F8F719
S21400D898A9FF214B45F8040B9D42F7D1F0881F4D90
S21400D8A8023080B2F8F79EFF1D4B02301860002346
S21400D8B82B6003F1804303F590235F241C60194A0C
S21400D8C82A200121FEF716FE88204FF4A0612C605E
S21400D8D8FEF78AFE0B480A4902680B6822F0100217
S21400D8E843F0010342F001020B60026070BD0000C5
S21400D8F808E10F4024800440148004401880044047
S21400D9080C8004400880044030720E0048E00F4047
S21400D918F8090020E8090020F809002004800440DF
S21400D928E4090020EDDE000000B50378FC2B13D1D7
S21400D9380E4B1A680E4B53F8222013889BB10B70B7
S21400D9481B0A4B70931C1A0A8B70CA7000201A0C9C
S21400D9581B0E0A714B7108E0F82B01D1012000E07C
S21400D9681120FAF755FA4FF0FF3000BDD80900200D
S21400D978E8090020064B10B51C682388038013B9F5
S21400D98841F27B230380F8F755FF208010BD000086
S21400D998E009002010B5594B81B00DF102021A605B
S21400D9A8574A136823F480031360136843F400632C
S21400D9B81360136823F0F06323F47C731360136812
S21400D9C843F0C07343F460731360136823F4005382
S21400D9D81360136843F4800313604A4B1B6813F004
S21400D9E8400FFAD0464A136823F400631360464B88
S21400D9F84FF000521A60454BD360454B1361454BB8
S21400DA085361454B9361454B1363454B9360454BB8
S21400DA189363454BD3624032444B1360444B9A425F
S21400DA2801D00432F8E7FFF7F3FC424A424913688C
S21400DA3843F020031360C03A136823F020031360F2
S21400DA48B832136843F008031360C03A136823F02B
S21400DA5808031360394B4FF480720B6003F11453BC
S21400DA6803F54C1303F5F65307331A6002F10E72EA
S21400DA7802F5862202F558724FF080431A6002F1CA
S21400DA887852A2F57012A2F55052583A0223136043
S21400DA980323136003F18043002209331A600A60E7
S21400DAA8F5F762F9264B31221A60264B1C686CB9CA
S21400DAB825482649F8F718FE254826490622F8F785
S21400DAC8C1FFF8F781FF04460028FAD022680AB991
S21400DAD81E4905E0204B1868904701460028E7D005
S21400DAE86068F8F701FEA068E1680622F8F7AAFF62
S21400DAF8F8F76AFF04460028FAD0E7E7E0090020AE
S21400DB0860E00F4050E00F4008ED00E0D9D3000079
S21400DB18DDD30000E1D30000E5D30000E9D3000020
S21400DB28EDD30000F1D30000F5D30000F9D30000D0
S21400DB38EC00002008E10F40000C004051E5CC1A2C
S21400DB4840E10F40940700202C050100440A0020FD
S21400DB58440501003405010098070020074B4FF0E4
S21400DB68007200B51A6072B6054A1368013313606E
S21400DB78F8F76EFEFEF700FD00BD000004ED00E0BD
S21400DB88D4090020074B012200B51A6072B6064A6F
S21400DB98136801331360054BDB689847FEF7ECFC07
S21400DBA800BD000024300340D4090020B809002036
S21400DBB8074B012200B51A6072B6064A136801338D
S21400DBC81360054B9B689847FEF7D6FC00BD00001F
S21400DBD824200340D4090020B8090020074B01225E
S21400DBE800B51A6072B6064A136801331360054B0F
S21400DBF85B689847FEF7C0FC00BD00002410034091
S21400DC08D4090020B8090020074B012200B51A6085
S21400DC1872B6064A136801331360054B1B689847AB
S21400DC28FEF7AAFC00BD000024000340D40900202B
S21400DC38B809002030B50D4C802512E013681D4247
S21400DC480AD00B4B1D6072B60A4A1368013313607C
S21400DC58E3699847FEF790FC074B043C6D089C4226
S21400DC6803D0064A1368002BE8D130BD9809002077
S21400DC781CD40340D40900207809002018D4034097
S21400DC8830B50D4C802512E013681D420AD00B4BA8
S21400DC981D6072B60A4A136801331360E369984731
S21400DCA8FEF76AFC074B043C6D089C4203D0064A04
S21400DCB81368002BE8D130BD780900201C74024098
S21400DCC8D4090020580900201874024030B50D4CBD
S21400DCD8802512E013681D420AD00B4B1D6072B6F1
S21400DCE80A4A136801331360E3699847FEF744FC51
S21400DCF8074B043C6D089C4203D0064A1368002B69
S21400DD08E8D130BD580900201C640240D409002020
S21400DD18380900201864024030B50D4C802512E002
S21400DD2813681D420AD00B4B1D6072B60A4A136868
S21400DD3801331360E3699847FEF71EFC074B043C63
S21400DD486D089C4203D0064A1368002BE8D130BD04
S21400DD58380900201C540240D40900201809002065
S21400DD681854024030B50D4C802512E013681D4249
S21400DD780AD00B4B1D6072B60A4A1368013313604B
S21400DD88E3699847FEF7F8FB074B043C6D089C428E
S21400DD9803D0064A1368002BE8D130BD18090020C6
S21400DDA81C440240D4090020F80800201844024009
S21400DDB830B50D4C802512E013681D420AD00B4B77
S21400DDC81D6072B60A4A136801331360E369984700
S21400DDD8FEF7D2FB074B043C6D089C4203D0064A6C
S21400DDE81368002BE8D130BDF80800201C740040EA
S21400DDF8D4090020D80800201874004030B50D4C0F
S21400DE08802512E013681D420AD00B4B1D6072B6BF
S21400DE180A4A136801331360E3699847FEF7ACFBB8
S21400DE28074B043C6D089C4203D0064A1368002B37
S21400DE38E8D130BDD80800201C640040D409002072
S21400DE48B80800201864004030B50E4C802513E052
S21400DE5813681D420BD00C4BE1691D6039B172B6D0
S21400DE680A4A1368013313608847FEF785FB084B98
S21400DE78043C6D089C4203D0064A1368002BE7D181
S21400DE8830BD0000B80800201C540040D40900200B
S21400DE98980800201854004030B50D4C802512E034
S21400DEA813681D420AD00B4B1D6072B60A4A1368E7
S21400DEB801331360E3699847FEF75EFB074B043CA3
S21400DEC86D089C4203D0064A1368002BE8D130BD83
S21400DED8980800201C440040D40900207808002038
S21400DEE81844004030B5574B82B01D68A3E013684D
S21400DEF813F0190F00F08880136813F018001ED06E
S21400DF0800238DF804308DF803304E238DF8053045
S21400DF1801238DF806300A3B8DF80730136813F096
S21400DF28080F1CBF6FF007038DF8073072B6464A15
S21400DF38002013680DF10301013313605CE0434BC6
S21400DF48D3F800E0424B53F82E10424B1A680B8861
S21400DF581BB34E238DF8053001238DF806303E4C52
S21400DF680A3B8DF804008DF803008DF80730236807
S21400DF7843F01003236072B6334A0DF103011368A9
S21400DF880020013313600522F7F75AFAFEF7F4FA71
S21400DF98236823F01003236033E0931E0B602F4B97
S21400DFA812041B88120C9A4282BFC3EB02000B8035
S21400DFB81A468C4698BF0020264B042A1B684CF845
S21400DFC8043F08D804E0234B04281B6805D9043806
S21400DFD80028F8D101E0043AEEE70EF101031B4AE7
S21400DFE8032B136001DD0023136072B6164A1C4922
S21400DFF813680020013313600522F7F721FAFEF7AD
S21400E008BBFA184B19221A60164C236813F0060F31
S21400E01808D0154B4FF000021B681A821A689A60DF
S21400E02806232360236813F0400F04D08820FEF7E9
S21400E038C7FA402323600B4A13682B427FF457AF76
S21400E04802B030BD04800440D4090020DC0900205A
S21400E058E80900201080044008800440F8090020E1
S21400E0681506010000800440340A0020C0B20128CA
S21400E078C9B208BF094807D038BF094804D3094BB6
S21400E08802280CBF18460020836913F0800F01D1C0
S21400E098012001E0016000207047000000D0004029
S21400E0A800C0004000E00040C0B2012808BF094890
S21400E0B807D038BF084804D3084B02280CBF1846B8
S21400E0C80020836B23F020038363036B23F48073A1
S21400E0D80363704700D0004000C0004000E00040E6
S21400E0E8C0B2C2B2012A10B508BF0B4C07D038BF61
S21400E0F80A4C04D30A4B022A0CBF1C460024FEF71F
S21400E108E1FA20236364A36B43F02003A363236B25
S21400E11843F48073236310BD00D0004000C0004065
S21400E12800E00040C0B2012808BF094807D038BF41
S21400E138084804D3084B02280CBF18460020836BF7
S21400E14823F010038363036B23F4007303637047A1
S21400E15800D0004000C0004000E00040C0B2C2B29C
S21400E168012A10B508BF0B4C07D038BF0A4C04D399
S21400E1780A4B022A0CBF1C460024FEF7A3FA1023FB
S21400E1886364A36B43F01003A363236B43F4007329
S21400E198236310BD00D0004000C0004000E00040EF
S21400E1A8054B01211B6800B581EA931101F00101B6
S21400E1B80220F7F77FFD00BDFC430040054B012118
S21400E1C81B6800B581EAD31101F001010120F7F7B9
S21400E1D871FD00BDFC43004010B589B211F00C0F6C
S21400E1E883B0C4B225D011F004031CBF254B53F8E6
S21400E1F8243000220093244B1B5D8DF80630234BF9
S21400E20813F804E0224B185DD1B24B1C013250FAC9
S21400E21803FCF9D101238DF80930684604238DF8EC
S21400E22807108DF808308DF805E08DF804C0FEF765
S21400E238FDFD184B1A68144B195D01238B401A42D2
S21400E24813D0062911D8DFE801F00406080A0C0ED8
S21400E2581200114B0CE0114B0AE0114B08E0114B71
S21400E26806E0114B04E0114B02E0002008E0104BDA
S21400E278074A1B68125D134208BF4FF48070F4D13A
S21400E28803B010BD000601000C0601000F060100D1
S21400E2981206010008E10F40FC430040FC53004012
S21400E2A8FC630040FC730040FC430240FC53024001
S20800E2B8FC630240BC
S21400E2BC3C62723E3C62723E486572652069732011
S21400E2CC74686520726571756573746564206D7508
S21400E2DC6C7469706C69636174696F6E20746162CA
S21400E2EC6C653A3C62723E3C62723E003C62723E28
S21400E2FC3C62723E4368616E67652076616C75653C
S21400E30C7320616E6420636C69636B2067656E6551
S21400E31C7261746521213C62723E3C62723E000062
S21400E32C3C7472207374796C653D6261636B6772C2
S21400E33C6F756E642D636F6C6F723A77686974656F
S21400E34C3E3C74682077696474683D36303E000045
S21400E35C3C74723E3C7468207374796C653D6261E3
S21400E36C636B67726F756E642D636F6C6F723A7742
S21400E37C686974652077696474683D36303E0000C1
S21400E38C3C74682077696474683D36303E00000043
S21400E39C3C2F74723E3C2F74683E00003C2F746811
S21400E3AC3E00000056312E332E3031310000000076
S21400E3BC6261636B67726F756E642D636F6C6F72E0
S21400E3CC3A000000726564200000000067726179F4
S21400E3DC002D202D202DD4E07F0E00003C68746D9F
S21400E3EC6C3E3C686561643E3C7469746C653E5377
S21400E3FC572055706C6F6164206661696C65643C6F
S21400E40C2F7469746C653E3C2F686561643E3C6293
S21400E41C6F6479206267636F6C6F723D2366663932
S21400E42C30303020746578743D23303030303030E6
S21400E43C20746F706D617267696E3D33206D61720A
S21400E44C67696E6865696768743D333E3C63656EE4
S21400E45C7465723E3C74642076616C69676E3D74BC
S21400E46C6F7020636C6173733D683E3C666F6E74B0
S21400E47C20636F6C6F723D236666303030302073CD
S21400E48C74796C653D666F6E742D73697A653A3374
S21400E49C3070783E3C62207374796C653D276D73E2
S21400E4AC6F2D626964692D666F6E742D776569676A
S21400E4BC68743A6E6F726D616C273E266D69637276
S21400E4CC6F3B5461736B65723C2F666F6E743E3C8B
S21400E4DC2F693E3C2F623E3C2F74643E3C62723E7B
S21400E4EC3C2F74643E3C746420616C69676E3D6CB2
S21400E4FC6566743E3C62723E3C62723E536F72724C
S21400E50C79206275742075706C6F61642068617315
S21400E51C206661696C65642E3C2F666F6E743E3C9B
S21400E52C62723E3C62723E3C6120687265663D6A71
S21400E53C6176617363726970743A686973746F722A
S21400E54C792E6261636B28293E52657475726E3C37
S21400E55C2F613E3C2F626F64793E3C2F68746D6C65
S21400E56C3E0000003C68746D6C3E3C686561643E21
S21400E57C3C6D65746120687474702D657175697670
S21400E58C3D7265667265736820636F6E74656E7433
S21400E59C3D31303B55524C3D304D656E752E687492
S21400E5AC6D3E3C7469746C653E4C4D3353585858EC
S21400E5BC582053572055706C6F616465643C2F74FB
S21400E5CC69746C653E3C2F686561643E3C626F64A2
S21400E5DC79206267636F6C6F723D2366666666664B
S21400E5EC6620746578743D233030303030302074BB
S21400E5FC6F706D617267696E3D33206D617267690D
S21400E60C6E6865696768743D333E3C63656E746519
S21400E61C723E3C74642076616C69676E3D746F70F4
S21400E62C20636C6173733D683E3C666F6E7420634A
S21400E63C6F6C6F723D2366663030303020737479A1
S21400E64C6C653D666F6E742D73697A653A333070FF
S21400E65C783E3C62207374796C653D276D736F2D24
S21400E66C626964692D666F6E742D77656967687468
S21400E67C3A6E6F726D616C273E266D6963726F3BE6
S21400E68C5461736B65723C2F666F6E743E202D2042
S21400E69C5357205570646174653C2F693E3C2F625D
S21400E6AC3E3C2F74643E3C62723E3C2F74643E3C8F
S21400E6BC746420616C69676E3D6C6566743E3C6282
S21400E6CC723E3C62723E53572055706C6F616420EC
S21400E6DC7375636365737366756C2E20546865205A
S21400E6EC4C4D3353585858582074617267657420D3
S21400E6FC77696C6C206E6F77207265736574206119
S21400E70C6E6420737461727420746865206E65770D
S21400E71C2070726F6772616D2E20506C6561736528
S21400E72C2077616974203130732E2E2E3C2F626F49
S21400E73C64793E3C2F68746D6C3E00000D0A0A48E6
S21400E74C656C6C6F2C20776F726C642E2E2E204CA2
S21400E75C4D335336393635204556414C0D0A00009C
S21400E76C4144432056616C7565733A0D0A000000EF
S21400E77C3D3D3D3D3D3D3D3D3D3D3D000D0A53611E
S21400E78C6D706C652D00000066617669636F6E2E89
S21400E79C69636F0009007800202017005D0A0000EE
S21400E7AC000041444D494E002020755461736B6542
S21400E7BC7226755461736B6572204E756D62657248
S21400E7CC20310000000000501401030000005573B7
S21400E7DC6572206E616D6500000000000000000090
S21400E7EC00000000005061737320776F72640000A5
S21400E7FC4D794164647265737340755461736B65CF
S21400E80C722E636F6D000000000000000000006DAB
S21400E81C61696C2E70726F76696465722E636F6DAB
S21400E82C00000000000000000000000000000000D7
S21400E83C000000006D795F646F6D61696E2E636F0A
S21400E84C6D000000454B5F4C4D3353363936352042
S21400E85C546573740000000048656C6C6F21210DC4
S21400E86C0A5468697320697320616E20656D61694E
S21400E87C6C206D6573736167652066726F6D2074AE
S21400E88C686520454B5F4C4D3353363936352E0D67
S21400E89C0A4920686F7065207468617420796F75FA
S21400E8AC2068617665207265636569766564207498
S21400E8BC686973207465737420616E642068617671
S21400E8CC652066756E207573696E672074686520A2
S21400E8DC755461736B6572206F7065726174696EC6
S21400E8EC672073797374656D207769746820696E18
S21400E8FC7465677261746564205443502F495020C8
S21400E90C737461636B2E0D0D0A52656761726473C6
S21400E91C20796F757220454B5F4C4D335336393624
S21400E92C3521210094E700000700000097E900005D
S21400E93C7E04000000000000000000000000000044
S21400E94C000000001800000000000000C0A8000333
S21400E95CFFFFFF00C0A80001C0A80001436F6D6D4B
S21400E96C616E64206C696E6520626C6F636B6564A7
S21400E97C0D0A0000436F6E6E656374696F6E2074CB
S21400E98C696D6564206F75740D0A00000001000146
S21400E99C00101000000100200068040000160000A3
S21400E9AC00280000001000000020000000010020DD
S21400E9BC000000000000000000130B0000130B000A
S21400E9CC000000000000000000FFFFFFFFFFFFFF3D
S21400E9DCFFFFFFFFFFFFFFFFFFFFFFFFFFFFFFFF36
S21400E9ECFFFFFFFFFFFFFFFFFFFFFFFFFFFFFFFF26
S21400E9FCFFFFFFFFFFFFFFFFFFFFFFFFFFFFFFFF16
S21400EA0CFFFFFFFFFFFFFFFFFFFFFFFFFFFFFFFF05
S21400EA1CFFFFFFFFFFFFFFFFFFD7DBDDFF919CA291
S21400EA2CFF5F6F77FF5F6F77FF5F6F77FF5F6F77C5
S21400EA3CFF5F6F77FF5F6F77FF5F6F77FF5F6F77B5
S21400EA4CFF919CA2FFFFFFFFFFFFFFFFFFFFFFFFF3
S21400EA5CFFFFFFFFFFA5AEB3FF5F6F77FF5F6F771C
S21400EA6CFF5F6F77FF5F6F77FF5F6F77FF5F6F7785
S21400EA7CFF5F6F77FF5F6F77FF5F6F77FF5F6F7775
S21400EA8CFF5F6F77FFFFFFFFFFFFFFFFFFFFFFFF3D
S21400EA9CFFA5AEB3FF5F6F77FF5F6F77FF87939926
S21400EAACFFD7DBDDFFFFFFFFFFFFFFFFFFFFFFFFD3
S21400EABCFFFFFFFFFFFFFFFFFFFFFFFFFF5F6F770D
S21400EACCFF5F6F77FFFFFFFFFFFFFFFFFFD7DBDD6B
S21400EADCFF5F6F77FF5F6F77FFAFB7BBFFFFFFFF81
S21400EAECFFFFFFFFFFFFFFFFFFEBEDEEFFAFB7BB38
S21400EAFCFFC3C9CCFFFFFFFFFFFFFFFFFF5F6F7772
S21400EB0CFF5F6F77FFFFFFFFFFFFFFFFFF919CA2EA
S21400EB1CFF5F6F77FF879399FFFFFFFFFFE1E4E549
S21400EB2CFF919CA2FFFFFFFFFFD7DBDDFF5F6F7738
S21400EB3CFF879399FFFFFFFFFFFFFFFFFF5F6F77D6
S21400EB4CFF5F6F77FFFFFFFFFFFFFFFFFF5F6F7734
S21400EB5CFF5F6F77FFD7DBDDFFFFFFFFFF7D8A913F
S21400EB6CFF879399FFFFFFFFFFD7DBDDFF5F6F7714
S21400EB7CFF879399FFFFFFFFFFFFFFFFFF5F6F7796
S21400EB8CFF5F6F77FFFFFFFFFFFFFFFFFF5F6F77F4
S21400EB9CFF5F6F77FFFFFFFFFFE1E4E5FF5F6F7737
S21400EBACFF879399FFFFFFFFFFD7DBDDFF5F6F77D4
S21400EBBCFF879399FFFFFFFFFFFFFFFFFF5F6F7756
S21400EBCCFF5F6F77FFFFFFFFFFFFFFFFFF5F6F77B4
S21400EBDCFF5F6F77FFFFFFFFFFD7DBDDFF5F6F7712
S21400EBECFF879399FFFFFFFFFFD7DBDDFF5F6F7794
S21400EBFCFF879399FFFFFFFFFFFFFFFFFF5F6F7716
S21400EC0CFF5F6F77FFFFFFFFFFFFFFFFFF5F6F7773
S21400EC1CFF5F6F77FFFFFFFFFFD7DBDDFF5F6F77D1
S21400EC2CFF879399FFFFFFFFFFD7DBDDFF5F6F7753
S21400EC3CFF879399FFFFFFFFFFCDD2D4FF5F6F775F
S21400EC4CFF5F6F77FFFFFFFFFFFFFFFFFF5F6F7733
S21400EC5CFF5F6F77FFFFFFFFFFD7DBDDFF5F6F7791
S21400EC6CFF879399FFFFFFFFFFD7DBDDFF5F6F7713
S21400EC7CFF879399FFFFFFFFFF879399FF5F6F77DF
S21400EC8CFF919CA2FFFFFFFFFFFFFFFFFF5F6F7769
S21400EC9CFF5F6F77FFFFFFFFFFD7DBDDFF5F6F7751
S21400ECACFF879399FFFFFFFFFFD7DBDDFF5F6F77D3
S21400ECBCFF879399FF9BA5AAFF5F6F77FF5F6F7720
S21400ECCCFFD7DBDDFFFFFFFFFFFFFFFFFF5F6F7769
S21400ECDCFF5F6F77FFFFFFFFFFD7DBDDFF5F6F7711
S21400ECECFF879399FFFFFFFFFFD7DBDDFF5F6F7793
S21400ECFCFF879399FF5F6F77FF5F6F77FFAFB7BBA9
S21400ED0CFFFFFFFFFFFFFFFFFFFFFFFFFF5F6F77BA
S21400ED1CFF5F6F77FFFFFFFFFFD7DBDDFF5F6F77D0
S21400ED2CFF5F6F77FF5F6F77FF5F6F77FF5F6F77C2
S21400ED3CFF5F6F77FF5F6F77FFAFB7BBFFFFFFFF1E
S21400ED4CFFFFFFFFFFFFFFFFFFFFFFFFFF5F6F777A
S21400ED5CFF5F6F77FFFFFFFFFFD7DBDDFF919CA206
S21400ED6CFF5F6F77FF5F6F77FF5F6F77FF69788066
S21400ED7CFF9BA5AAFFE1E4E5FFFFFFFFFFFFFFFFF8
S21400ED8CFFFFFFFFFFFFFFFFFFFFFFFFFFFFFFFF82
S21400ED9CFFFFFFFFFFFFFFFFFFFFFFFFFFFFFFFF72
S21400EDACFFFFFFFFFFFFFFFFFFFFFFFFFFFFFFFF62
S21400EDBCFFFFFFFFFFFFFFFFFFFFFFFFFFFFFFFF52
S21400EDCCFFFFFFFFFFFFFFFFFF000000000000003B
S21400EDDC0000000000000000000000000000000022
S21400EDEC0000000000000000000000000000000012
S21400EDFC0000000000000000000000000000000002
S21400EE0C0000000000000000000000002A000000C7
S21400EE1C202D2000656E61626C65640D0A00000092
S21400EE2C64697361626C65640D0A00004C414E2087
S21400EE3C7370656564200000444843505F53455228
S21400EE4C564552000A0D53657269616C206E756DDD
S21400EE5C6265723A20000000536F667477617265C3
S21400EE6C2076657273696F6E2000000044657669C3
S21400EE7C6365206964656E74696669636174696F3D
S21400EE8C6E3A20000A0A0D000A0D3D3D3D3D3D3D03
S21400EE9C3D3D3D3D3D3D3D3D3D3D3D3D3D0A0D0031
S21400EEAC0A0D506172616D65746572207365740A23
S21400EEBC0D0000000A0D54656D702E2050617261B5
S21400EECC6D65746572207365740A0D000A0D5061C9
S21400EEDC72616D657465722076616C7565203D2077
S21400EEEC000000000A0D4E6F2076616C696420707D
S21400EEFC6172616D657465727320617661696C61AF
S21400EF0C626C650A0D0000000A0D4F726967696E27
S21400EF1C616C20706172616D6574657273207265C8
S21400EF2C73746F7265640A0D000000000A0D46616A
S21400EF3C63746F727920706172616D65746572733B
S21400EF4C20726573746F7265640A0D000A0D506149
S21400EF5C72616D657465727320696E76616C696436
S21400EF6C617465640A0D00000A0D4E6577205061C9
S21400EF7C72616D65746572732076616C6964617418
S21400EF8C65640A0D000000000A0D436F6E66696723
S21400EF9C75726174696F6E2073617665640A0D0014
S21400EFAC415250207265736F6C7574696F6E207366
S21400EFBC7461727465640A0D000000000D0A4950F5
S21400EFCC2061646472657373203D20000D0A4D4108
S21400EFDC432061646472657373203D20000000005A
S21400EFEC0D0A5375626E6574206D61736B203D203F
S21400EFFC000000000D0A44656661756C742067613C
S21400F00C7465776179203D2000000000656E6162B2
S21400F01C6C65000064697361626C65000D0A496E6C
S21400F02C76616C6964207377697463680D0A0000F6
S21400F03C0A0D53797374656D206D656D6F7279204A
S21400F04C7573653A0A0D00003D3D3D3D3D3D3D3D29
S21400F05C3D3D3D3D3D3D3D3D3D3D0A0D0000000026
S21400F06C467265652068656170203D2000000000D2
S21400F07C2066726F6D2000000A0D556E7573656400
S21400F08C20737461636B203D200000000D0A5468E9
S21400F09C65206465766963652068617320626565C2
S21400F0AC6E206F7065726174696E6720666F722071
S21400F0BC0000000042616420706F7274206E756DE3
S21400F0CC6265720D0A0000000D0A506F727420649F
S21400F0DC6972656374696F6E3A2000004F55545020
S21400F0EC55540D0A00000000494E5055540D0A00A8
S21400F0FC496E76616C696420706F72740D0A00003C
S21400F10C506F727420697320696E7075740D0A00E6
S21400F11C506F72742073746174653A20000000009E
S21400F12C310D0A00300D0A000D0A3F3F0D0A230070
S21400F13C0A0D427965204279650A0D004D4143203F
S21400F14C6D6179206E6F74206265206D6F646966E0
S21400F15C69656421210D0A000D0A45746865726E96
S21400F16C657420537461746973746963730D0A0053
S21400F17C0D0A415250205461626C6520636F6E74A8
S21400F18C656E74733A0000000D0A49502061646481
S21400F19C726573733A200000204D4143206164640D
S21400F1AC726573733A2000000D0A456E640D0A00F2
S21400F1BC496E636F72726563742064617461206C4F
S21400F1CC656E6774680D0A000D0A53657269616C8A
S21400F1DC20636F6E66696775726174696F6E0D0A6F
S21400F1EC0000000042617564203D2000696E766167
S21400F1FC6C69642100000000370000003800000035
S21400F20C20426974730D0A00207061726974790D5E
S21400F21C0A0000002073746F7020626974287329CA
S21400F22C0D0A0000466C6F7720636F6E74726F6CFD
S21400F23C20000000486967682077617465722000BA
S21400F24C250D0A004C6F77207761746572200000DC
S21400F25C0D0A5365637572697479207365747469E5
S21400F26C6E67730D0A0000005465726D696E616CF2
S21400F27C206D656E75206C6F67696E004654502065
S21400F28C7365727665720000574542207365727618
S21400F29C6572000057454220736572766572206170
S21400F2AC757468656E7469636174696F6E000000CE
S21400F2BC54454C4E455420736572766572000000BA
S21400F2CC20202054656C6E657420706F7274206EEE
S21400F2DC756D626572203D2000000000496E636FFC
S21400F2EC7272656374204C414E2073706565640DB4
S21400F2FC0A000000496E636F727265637420736552
S21400F30C7269616C2073706565640D0A00000000FC
S21400F31C496E636F7272656374207061726974797A
S21400F32C0D0A0000496E636F727265637420737405
S21400F33C6F7020626974730D0A000000496E636F6B
S21400F34C727265637420666C6F7720636F6E74726E
S21400F35C6F6C0D0A000000000A0D415250207265B9
S21400F36C736F6C7665640A0D000000000A0D41523E
S21400F37C50207265736F6C7574696F6E2066616968
S21400F38C6C65640A0D00000050494E472072657388
S21400F39C706F6E73652066726F6D2000556E6B6EA7
S21400F3AC6F776E2050494E4720726573706F6E7380
S21400F3BC650D0A0020202020204D61696E206D65A9
S21400F3CC6E750000204C414E20636F6E6669677543
S21400F3DC726174696F6E000020202053657269613B
S21400F3EC6C20636F6E6669672E00000020496E7095
S21400F3FC75742F4F7574707574206D656E7500007E
S21400F40C20202041646D696E2E206D656E7500009F
S21400F41C20202053746174732E206D656E75000069
S21400F42C4D41430031000000436F6E66696775728C
S21400F43C65204C414E20696E74657266616365008A
S21400F44C32000000436F6E666967757265207365DF
S21400F45C7269616C20696E74657266616365000022
S21400F46C33000000476F20746F20492F4F206D65C6
S21400F47C6E75000034000000476F20746F206164C6
S21400F48C6D696E697374726174696F6E206D656EEA
S21400F49C7500000035000000476F20746F206F76F3
S21400F4AC6572766965772F737461746973746963B2
S21400F4BC73206D656E75000068656C70000000004A
S21400F4CC446973706C6179206D656E752073706518
S21400F4DC63696669632068656C7000007175697491
S21400F4EC000000004C6561766520636F6D6D616E83
S21400F4FC64206D6F6465000075700000676F207483
S21400F50C6F206D61696E206D656E75007365745F36
S21400F51C64686370000000003C656E61626C652F69
S21400F52C64697361626C653E204448435000000079
S21400F53C7365745F69705F61646400005365742062
S21400F54C4950206164647265737300007365745F60
S21400F55C69705F6D61736B0053657420495020733E
S21400F56C75626E6574206D61736B00007365745FF5
S21400F57C69705F67776179005365742064656661AE
S21400F58C756C742067617465776179007365745F58
S21400F59C6574685F7370656564000000536574205D
S21400F5AC4C414E207370656564202831302F313005
S21400F5BC302F4155544F290073686F775F636F6E19
S21400F5CC6669670053686F77206E6574776F726B29
S21400F5DC20636F6E66696775726174696F6E000082
S21400F5EC73686F775F636F6E6669675F6F000000A6
S21400F5FC53686F77206F726967696E616C206E65F1
S21400F60C74776F726B20636F6E6669677572617460
S21400F61C696F6E0073617665000000005361766555
S21400F62C20636F6E66696775726174696F6E20749D
S21400F63C6F20464C4153480076616C696461746572
S21400F64C0000000056616C69646174652074656D19
S21400F65C706F7261727920636F6E6669672E2069AF
S21400F66C6E20464C4153480070696E6700000000DF
S21400F67C50696E6720746573742049502061646409
S21400F68C7265737300000000617270202D610000BB
S21400F69C5265717565737420415250207461626CAA
S21400F6AC65000000617270202D64000044656C6576
S21400F6BC746520415250207461626C650000000035
S21400F6CC7365745F62617564000000005365742096
S21400F6DC73657269616C2062617564207261746511
S21400F6EC000000007365745F73746F700000000098
S21400F6FC5365742073746F7020626974732028319C
S21400F70C2F312E352F3229007365745F626974733E
S21400F71C0000000053657420646174612062697493
S21400F72C732028372F3829007365745F7061720058
S21400F73C5365742070617269747920284556454E5D
S21400F74C2F4F44442F4E4F4E452900007365745F6F
S21400F75C666C6F770000000053657420666C6F77DC
S21400F76C20636F6E74726F6C2028584F4E2F525455
S21400F77C532F4E4F4E4529007365745F6869676852
S21400F78C5F7761746572000053657420666C6F77E2
S21400F79C207374616C6C20282529205B312E2E3941
S21400F7AC395D00007365745F6C6F775F77617465A5
S21400F7BC7200000053657420666C6F772072657358
S21400F7CC7461727420282529205B312E2E39395D00
S21400F7DC0000000053686F772073657269616C20B7
S21400F7EC636F6E66696775726174696F6E00000090
S21400F7FC7365745F6464720053657420706F727402
S21400F80C2074797065205B312E2E345D205B3C694C
S21400F81C3E7C3C6F3E0000006765745F646472005B
S21400F82C47657420646174612064697265637469E9
S21400F83C6F6E205B312E2E345D00000072656164A5
S21400F84C5F706F72740000005265616420706F7296
S21400F85C7420696E707574205B312E2E345D00003A
S21400F86C77726974655F706F7274000053657420EC
S21400F87C706F7274206F7574707574205B312E2ED9
S21400F88C345D205B302F315D0000000053617665DF
S21400F89C20706F72742073657474696E6720617360
S21400F8AC2064656661756C74000000007365745F97
S21400F8BC667470003C656E61626C652F646973617A
S21400F8CC626C653E204654502073657276657200F5
S21400F8DC7365745F74656C6E657400003C656E6170
S21400F8EC626C652F64697361626C653E2054656C4E
S21400F8FC6E65742073657276696365007365745FF4
S21400F90C776562003C656E61626C652F6469736135
S21400F91C626C653E205745422073657276657200B0
S21400F92C7365745F7765625F6175746800000000CC
S21400F93C3C656E61626C652F64697361626C653ED2
S21400F94C205745422073657276657220617574681F
S21400F95C656E7469636174696F6E000053686F77C7
S21400F96C20636F6E66696775726174696F6E0000EE
S21400F97C72656A65637400005265736574206E6FF9
S21400F98C6E2D7361766564206368616E67657300BF
S21400F99C726573746F726500526573746F7265204E
S21400F9AC666163746F72792073657474696E6773BD
S21400F9BC0000000072657365740000005265736584
S21400F9CC7420646576696365000000006970737462
S21400F9DC6174000053686F772045746865726E65B5
S21400F9EC7420737461746973746963730000000027
S21400F9FC725F697073746174000000005265736501
S21400FA0C742045746865726E6574207374617469CD
S21400FA1C737469637300000075705F74696D6500BC
S21400FA2C53686F77206F7065726174696E672074A7
S21400FA3C696D65006D656D6F7279000053686F7740
S21400FA4C206D656D6F72792075736500082008004F
S21400FA5CA0FC00000F070000C0F30000F4FC000040
S21400FA6C140F0000D0F30000A8FD0000160C0000D8
S21400FA7CE4F3000038FE00000F080000F8F3000066
S21400FA8C98FE0000110C00000CF4000028FF00008B
S21400FA9C110700001CF400006D0000002CF40000A0
S21400FAAC0000000004090000546F74616C2052784A
S21400FABC206672616D6573000000005278206F76C8
S21400FACC657272756E7300000000000000005278BC
S21400FADC2041525000000000000000000000000012
S21400FAEC0052782049434D500000000000000000F2
S21400FAFC0000000052782055445000000000000022
S21400FB0C0000000000000052782054435000000013
S21400FB1C00000000000000000000527820636865BA
S21400FB2C636B73756D206572726F727300527820FA
S21400FB3C6F746865722070726F746F636F6C73008D
S21400FB4C466F726569676E205278204152500000ED
S21400FB5C000000466F726569676E20527820494334
S21400FB6C4D5000000000466F726569676E20527833
S21400FB7C205544500000000000466F726569676EA1
S21400FB8C205278205443500000000000546F7461DB
S21400FB9C6C205478206672616D657300000000411D
S21400FBAC52502073656E74000000000000000000C8
S21400FBBC000049434D502073656E74000000000031
S21400FBCC00000000005544502073656E7400000061
S21400FBDC00000000000000005443502073656E7453
S21400FBEC00000000000000000000004F7468657202
S21400FBFC206576656E7473000000000000003130DE
S21400FC0C00000031303000004155544F0033303086
S21400FC1C000000003630300000000031323030007A
S21400FC2C0000323430300000003438303000000031
S21400FC3C3936303000000031343430300000313981
S21400FC4C3230300000333834303000003537363040
S21400FC5C3000003131353230300032333034303011
S21400FC6C004F444400004556454E004E4F4E45004E
S21400FC7C31000000312E3500320000004E4F4E454C
S21400FC8C000000005254530000000000584F4E0075
S21400FC9C0000000030F4000034F400000004000003
S21400FCAC4CF4000050F40000000500006CF400005A
S21400FCBC70F400000006000080F4000084F40000DD
S21400FCCC00070000A0F40000A4F4000000090000E7
S21400FCDCC4F40000CCF4000000000000E8F40000BF
S21400FCECF0F400000200000004F5000008F5000027
S21400FCFC000D000018F5000024F5000007010000B8
S21400FD0C3CF5000048F500000401000058F5000022
S21400FD1C64F500000402000078F5000084F500008D
S21400FD2C0403000098F50000A8F500000406000087
S21400FD3CC4F50000D0F5000004050000ECF500004A
S21400FD4CFCF50000040A000020F6000028F600006F
S21400FD5C0306000044F6000050F600000305000001
S21400FD6C74F600007CF600000400000094F6000018
S21400FD7C9CF6000004070000B0F60000B8F6000081
S21400FD8C04080000C4F40000CCF4000000000000DE
S21400FD9CE8F40000F0F400000200000004F5000097
S21400FDAC08F50000000D0000CCF60000D8F60000A8
S21400FDBC05000000F0F60000FCF60000050100004F
S21400FDCC14F7000020F700000502000034F70000CE
S21400FDDC3CF700000503000058F7000064F700002D
S21400FDEC0504000084F7000094F7000005150000D9
S21400FDFCB0F70000C0F7000005160000C4F50000C0
S21400FE0CE0F700000511000020F6000028F60000C0
S21400FE1C03060000C4F40000CCF400000000000050
S21400FE2CE8F40000F0F400000200000004F5000006
S21400FE3C08F50000000D0000FCF7000004F80000B8
S21400FE4C0102000024F800002CF80000010B000052
S21400FE5C48F8000054F80000010400006CF800009C
S21400FE6C78F800000105000020F6000098F8000065
S21400FE7C010C0000C4F40000CCF4000000000000EC
S21400FE8CE8F40000F0F400000200000004F50000A6
S21400FE9C08F50000000D0000B8F80000C0F80000DF
S21400FEAC07020000DCF80000E8F80000070000007D
S21400FEBC08F9000010F90000070300002CF90000F8
S21400FECC3CF9000007050000C4F5000068F90000C6
S21400FEDC0602000020F6000028F6000003060000CC
S21400FEEC7CF9000084F90000030700009CF9000070
S21400FEFCA4F9000003020000C0F90000C8F90000D5
S21400FF0C01000000C4F40000CCF400000000000067
S21400FF1CE8F40000F0F400000200000004F5000015
S21400FF2C08F50000000D0000D8F90000E0F900000C
S21400FF3C04040000FCF9000008FA0000040B0000A2
S21400FF4C24FA00002CFA0000010A000040FA000017
S21400FF5C48FA000001010000C4F40000CCF40000D4
S21400FF6C00000000E8F40000F0F4000002000000BE
S21400FF7C0001080006046382536335010101060084
S21400FF8C123456780000800037070103060C333A0B
S21400FF9C3B000001000100010001000020302E484B
S21400FFAC544D0D0A00000000555345522000000029
S21400FFBC5041535320000000737973740000000006
S21400FFCC7369746500000000505744005041535646
S21400FFDC000000006E6F6F70000000004357440076
S21400FFEC5459504520000000504F52542000000039
S21400FFFC4C4953540000000053544F52200000004C
S21401000C44454C45200000002A2E2A0053495A45E7
S21401001C200000005245545220000000515549540E
S21401002C000000003232302057656C636F6D65201E
S21401003C4C4D335378787878204654502E0D0A0060
S21401004C323236204F4B2E0D0A000000333331204E
S21401005C456E74657220706173732E0D0A00000074
S21401006C323330204C6F67204F4B2E0D0A000000A8
S21401007C353330204C6F67204241442E0D0A000068
S21401008C31353020446174612E0D0A003231352031
S21401009C554E495820547970653A204C380D0A0053
S2140100AC3535302044656E6965642E0D0A000000F6
S2140100BC32353720222F220D0A0000003230302034
S2140100CC4F4B2E0D0A000000323530204469722049
S2140100DC6368616E6765642E0D0A00003432352044
S2140100EC426164206461746120706F72740D0A0041
S2140100FC3235302044656C204F4B2E0D0A00000023
S21401010C35303020576861743F2E0D0A0000000010
S21401011C323231204279650D0A0000002D722045DD
S21401012C6D7074790D0A00323237205041535620C7
S21401013C4D4F44452028323133202D727778727713
S21401014C78727778203120353032203530322020C5
S21401015C4A616E20312032303038200048545450D9
S21401016C2F312E3020323030204F4B0D0A0D0A0025
S21401017C474554504F535464697361626C656463AC
S21401018C6865636B656473656C65637465644175FA
S21401019C74686F72697A6174696F6E3A2042617322
S2140101AC69632000485454502F312E30203430319E
S2140101BC0D0A5757572D41757468656E74696361DE
S2140101CC74653A204261736963207265616C6D3D9A
S2140101DC755461736B65720D0A0D0A003C68746D7B
S2140101EC6C3E3C686561643E3C7469746C653E7536
S2140101FC5461736B6572204E6F2066696C653C2F7B
S21401020C7469746C653E3C2F686561643E3C626F34
S21401021C6479206267636F6C6F723D236666393052
S21401022C303020746578743D2330303030303020D7
S21401023C746F706D617267696E3D33206D617267A4
S21401024C696E6865696768743D333E3C63656E74B8
S21401025C65723E3C74642076616C69676E3D746FA2
S21401026C7020636C6173733D683E3C666F6E7420E0
S21401027C636F6C6F723D236666303030302073745A
S21401028C796C653D666F6E742D73697A653A333099
S21401029C70783E3C62207374796C653D276D736F84
S2140102AC2D626964692D666F6E742D776569676852
S2140102BC743A6E6F726D616C273E755461736B6523
S2140102CC723C2F666F6E743E202D204572726F72D3
S2140102DC203430343C2F693E3C2F623E3C2F7464F4
S2140102EC3E3C62723E3C2F74643E3C746420616CEE
S2140102FC69676E3D6C6566743E3C62723E3C62722A
S21401030C3E54686520726571756573746564206604
S21401031C696C6520686173206E6F74206265656E0A
S21401032C20666F756E64206F6E2074686520736529
S21401033C727665722E20506C6561736520636865F4
S21401034C636B20746861742068746D6C2066696CCC
S21401035C65732068617665206265656E206C6F61D9
S21401036C64656420636F72726563746C792E3C628B
S21401037C723E3C2F666F6E743E3C2F74643E3C2F6F
S21401038C74723E3C2F626F64793E3C2F68746D6CC0
S21401039C3E0000002A485454502F312E3020313064
S2140103AC3020636F6E740D0A0D0A000008040100FC
S2140103BC09010000140401000F02000024040100CE
S2140103CC04030000280401000E0400003804010098
S2140103DC1405000050040100180600006C0401000E
S2140103EC0A07000078040100210800009C040100A3
S2140103FC09090000A80401000F0A0000626F756E5F
S21401040C646172793D000000436F6E74656E742DE5
S21401041C4C656E6774683A000D0A0D0A436F6E746C
S21401042C656E742D547970653A20000045787065B8
S21401043C63743A203130302D636F6E74696E756556
S21401044C000000006170706C69636174696F6E2FD7
S21401045C6F637465742D73747265616D00000000B2
S21401046C746578742F706C61696E00006170706CC5
S21401047C69636174696F6E2F782D7777772D666F48
S21401048C726D2D75726C656E636F64656400000029
S21401049C696D6167652F6769660000006170706C35
S2140104AC69636174696F6E2F7064660008000001E1
S2140104BC5180000045484C4F2000000041555448DF
S2140104CC204C4F47494E00004D41494C2046524F57
S2140104DC4D3A203C000000005243505420544F3AF1
S2140104EC203C00004441544100000000546F3A2067
S2140104FC000000000D0A5375626A6563743A2000A9
S21401050C0D0A46726F6D3A20000000000D0A2E008F
S21401051C000605060C181C3C0820080011000000FB
S21401052C01005866000000000157414554616D44B6
S21401053C6453464E730000001C060100FD4E00007D
S21401054C000000000400010024060100C170000038
S21401055C450001000000000028060100DD7E0000B9
S21401056C3C000100000000002C0601008DB50000C7
S21401057C450002000000000030060100B131000009
S21401058C450002000000000034060100117A00004C
S21401059C2500FFFF000000003C060100F97B00006F
S2140105AC250001000000000040060100E1A4000047
S2140105BC2500FFFF0000000048060100E94D000081
S2140105CC2500FFFF000000000000000000000000F6
S2140105DC0000000000000000000000000000FFFF0B
S2140105ECFFFFFFFF11DC0000E5DB0000B9DB0000BC
S2140105FC8DDB000081D60000C5E10000A9E10000FA
S21401060C00000003030308804000004501FC0000C5
S21401061C57646F6700000000415250004574680033
S21401062C5443500061707000444843500000000071
S21401063C644E5300534D5450000000006D61696EBA
S21401064C74656E616365000048544D004A5047005E
S21401065C47494600435353004A53000042494E0053
S21001066C5458540049434F003F3F3F00E4
S214010678746573745F6E616D6540746573742E631B
S2140106886F6D000000000000000000000000000080
S214010698000000000000000000FFC0A8006600007F
S2140106A8FFFFFFFFFFFFFFFF0100000054060100E8
S2140106B8580601005C060100600601006406010098
S2140106C8680601006C060100700601007406010048
S80400D99D85
